:10A01B00543100543200543300543400543500543E
:10A02B0036005631004631004632004633004D3182
:10A03B000053540053460053560053300053310025
:10A04B005332005333004831004330004331005347
:10A05B0045462D476D624820203534382E3034204C
:10A06B00205265762E20332E33002020002D3E000B
:10A07B003C2D00504320636F6E6E65637465640006
:10A08B0048454154455220204F4E004845415445C8
:10A09B0052204F464600413A0054313D00256400A2
:10A0AB003B0054333D0056313D0053543D002C00D2
:10A0BB0053463D0053563D0053303D3534382E301A
:10A0CB003420563D0053313D0053323D00256C6426
:10A0DB000053333D0048313D004552523D313B006A
:10A0EB004552523D303B00413A4552523D004331BF
:10A0FB003D000D00737065656400746C75667400CB
:10A10B006972006865697A006765626C00332E338B
:01A11B000043
:10005E0078167C397D017BFF7AA179187E007F04AA
:10006E001230069002FC74FFF0A374A0F0A3741B70
:10007E00F090030874FFF0A374A0F0A3741EF09028
:10008E00031474FFF0A374A0F0A37421F090032066
:10009E0074FFF0A374A0F0A37424F090032C74FFEB
:1000AE00F0A374A0F0A37427F090033874FFF0A3AC
:1000BE0074A0F0A3742AF090034474FFF0A374A00C
:1000CE00F0A3742DF090035074FFF0A374A0F0A36E
:1000DE007430F090035C74FFF0A374A0F0A374333B
:1000EE00F090036874FFF0A374A0F0A37436F09040
:1000FE00037474FFF0A374A0F0A37439F09003801E
:10010E0074FFF0A374A0F0A3743CF090038C74FF02
:10011E00F0A374A0F0A3743FF090039874FFF0A3C3
:10012E0074A0F0A37442F09003A474FFF0A374A023
:10013E00F0A37445F09003B074FFF0A374A0F0A385
:10014E007448F09003BC74FFF0A374A0F0A3744B3A
:10015E00F09003C874FFF0A374A0F0A3744EF09057
:10016E0003D474FFF0A374A0F0A37451F09003E0D5
:10017E0074FFF0A374A0F0A37454F09003EC74FF1A
:10018E00F0A374A0F0A37457F0E490000CF090016B
:10019E00FAF0900202F07B0190391304F0A3743947
:1001AE00F0A37411F012C27512C1D612C2C412C2DB
:1001BE00BAE49000B3F0D2137B0190398A04F0A315
:1001CE007400F0A374B4F0A3E4F0A304F07B107DEC
:1001DE00067C0C7F501295C912C15012BE7290024D
:1001EE0017123338E47B0CFAF9F8900217E0FCA3EF
:1001FE00E0FDA3E0FEA3E0FF1232719001EAEEF003
:10020E00A3EFF0E47B0CFAF9F8900217E0FCA3E000
:10021E00FDA3E0FEA3E0FF123271CCE8CCCDE9CD18
:10022E00CEEACECFEBCFE47B05FAF9F81231E690A9
:10023E000152EEF0A3EFF0903913E0F9A3E0FAA328
:10024E00E090398AC9F0A3EAF0A3E9F0A3E4F0A3A1
:10025E007402F07B107D257C0C7F501295C9EF64E3
:10026E00014E600690390FE004F0903911E0FFA3C3
:10027E00E09039D0CFF0A3EFF0E4900223F012C259
:10028E00CE12BC571200037D057C007F057E001246
:10029E00B8A17BFF7AA0795A12C18190C060E4F0B8
:1002AE00900209F0C2057F0412C1FEC2057F08123A
:1002BE00C1FED20FE4900220F09000B7F09002033E
:1002CE00F0F5FD7F8012C299E4339036DEF0900295
:1002DE001BE4F0A37403F0900212E4F0A37405F093
:1002EE0090020AE4F0A37402F0E4900207F0A3F087
:1002FE009001EFF0A3F0900210F0A3F09036D2F040
:10030E00A37414F0900007E4F0A37414F090390D68
:10031E00E4F0A37414F09000B1E4F0A37414F0E4CC
:10032E009001FEF0A3F090022104F0A3746AF09005
:10033E00022AE4F0A37409F0E4900001F0A3F09017
:10034E000000F0900214F0A3F07F32FEFDFC12BF0D
:10035E00569036CEE0645A6041E4900204F07B0180
:10036E0090399504F0A37402F0A37404F0A3E4F0A2
:10037E00A304F07B107D087C0C7F50128D9712B277
:10038E00FC903904EEF0A3EFF07003EE64017003FD
:10039E00120000E4903904F0A3F090398A7401F051
:1003AE00A37402F0A37426F0A3E4F0A304F07B1070
:1003BE007D077C0C7F501295C990398A7401F0A389
:1003CE007403F0A374F8F0A3E4F0A304F07B107DA3
:1003DE00047C0C7F501295C99003F8E0FFC3940083
:1003EE004006EFD394084005E49003F8F0900226FF
:1003FE00E0FFC3648094804008D3EF648094814012
:10040E0005E4900226F0E49001FCF0A3F09036CEC5
:10041E00E0645A60030204E77B0190398A04F0A37A
:10042E007402F0A37404F0A3E4F0A304F07B107D37
:10043E00087C0C7F501295C990398A7401F0A37410
:10044E0036F0A374C9F0A3E4F0A37402F07B107D20
:10045E00097C0C7F501295C990398A7401F0A374EF
:10046E0036F0A374C7F0A3E4F0A37402F07B107D02
:10047E00117C0C7F501295C990398A7401F0A374C7
:10048E0036F0A374CBF0A3E4F0A37402F07B107DDE
:10049E00137C0C7F501295C990398A7401F0A374A5
:1004AE0002F0A3741DF0A3E4F0A304F07B107D15FD
:1004BE007C0C7F501295C990398A7401F0A3743662
:1004CE00F0A374BDF0A3E4F0A304F07B107D177CC1
:1004DE000C7F501295C902060C90398A7401F0A354
:1004EE007436F0A374BDF0A3E4F0A304F07B107D8A
:1004FE00057C0C7F501295C99036BDE0FFC3648019
:10050E009481403BD3EF6480949050337B017A36D4
:10051E0079BD90394FE4F0A37411F012BD74903987
:10052E008A7401F0A37402F0A3741DF0A3E4F0A387
:10053E0004F07B107D157C0C7F501295C98021E450
:10054E009036BDF09036C7F0A37404F0A3E4F0A388
:10055E0074D2F0A3E4F0A37414F090021D7432F080
:10056E009039957401F0A37436F0A374C9F0A3E426
:10057E00F0A37402F07B107D097C0C7F50128D97D6
:10058E009039957401F0A37436F0A374C7F0A3E408
:10059E00F0A37402F07B107D117C0C7F50128D97AE
:1005AE009039957401F0A37436F0A374CBF0A3E4E4
:1005BE00F0A37402F07B107D137C0C7F50128D978C
:1005CE009039957401F0A37402F0A3741DF0A3E4A6
:1005DE00F0A304F07B107D157C0C7F50128D97904C
:1005EE0039957401F0A37436F0A374BDF0A3E4F052
:1005FE00A304F07B107D177C0C7F50128D97128A0E
:10060E00AE9036C7E0FFA3E09036EDCFF0A3EFF04B
:10061E009036C9E0FFA3E09036EFCFF0A3EFF09055
:10062E0036CBE0FEA3E0FF9036F1EEF0A3EFF090B4
:10063E0036CDE09036F3F0E4900000F0900214F026
:10064E00A3F0127B1C9036CBE0FFA3E09000B8CF56
:10065E00F0A3EFF0D2147F017E0012BEBFC21412BF
:10066E000003438710E4F5FFD2057F0812C1FE9008
:10067E0036CE745AF0D202C203903925740AF0E4D1
:10068E0090390BF0A3F012C25FC299C298D2AC900F
:10069E003926E0FF9036CFE07003A3E06F700302BF
:1006AE0007689036D0E0903926F030020302075AE0
:1006BE0020040E90390CE004F0700690390BE00423
:1006CE00F030040E90390CE024FFF090390BE0343A
:1006DE00FFF020041790390CE02410FF90390BE046
:1006EE003400FE7D047C0012B8A1801590390CE018
:1006FE002412FF90390BE03400FE7D047C0012B80A
:10070E00A17BFF7AA0797512C18190390BE0FEA30F
:10071E00E0FFC39404EE94004002D204D3EF9400A1
:10072E00EE94005002C204EF2411FFE43EFE7D045D
:10073E007C0012B8A120040B7BFF7AA0797812C13D
:10074E008180097BFF7AA0797B12C181903925E0E7
:10075E0014F0E07005740AF0D202A202300301B365
:10076E00400302085220020302080E1262097D079E
:10077E007C007F037E0012B8A1900000E0FFC364EE
:10078E0080948040339003F8E075F00CA4248CF52F
:10079E0082E43438F583EF3395E0FE75F003EF1203
:1007AE003375EE75F003A42583F583E0FBA3E0FA21
:1007BE00A3E0F912C18180449003F8E075F00CA417
:1007CE002429F582E43438F583C083C0829000007A
:1007DE00E0FF3395E0FEC3E49FFFE49EFED082D09F
:1007EE008375F003EF123375EE75F003A42583F5D0
:1007FE0083E0FBA3E0FAA3E0F912C181A202920307
:10080E002002411200037D067C007F0E7E0012B88E
:10081E00A17BFF7AA0797E12C1817D027C007F0FC1
:10082E007E0012B8A1900204E0B4010B7BFF7AA007
:10083E00798B12C18180097BFF7AA0799612C181D2
:10084E00A202920320023A9036D1E0FF900204E019
:10085E006F602E7D027C007F0F7E0012B8A1900289
:10086E0004E0B4010B7BFF7AA0798B12C181800961
:10087E007BFF7AA0799612C181900204E09036D166
:10088E00F030021B12B2FC903904EEF0A3EFF04EE2
:10089E006010903904E0FEA3E0FF12B6F880031258
:1008AE00AA9F201203021439E490391AF0D2019053
:1008BE003925740AF0C20278547C017D017BFF7ADF
:1008CE00A079A1123665E490021EF09001ECF09032
:1008DE003909F0A3F090021F7401F090390AE02458
:1008EE00BBF582E43400F583E0FF64436006903983
:1008FE001AE02FF0EF6443705690390AE014FF129D
:10090E004DFC903910EFF09001ECE0B415279039C2
:10091E0010E0FF129320903907EEF0A3EFF090391C
:10092E001AE06F7001EE700690021FF080079002C1
:10093E001FE04401F09001ECE0B41405E490021FB6
:10094E00F0903909E4F0A37496F0E49001ECF043D2
:10095E00871090390AE004F07006903909E004F02F
:10096E00C390390AE09496903909E094005003023E
:10097E0008E3E4903909F0A3F0903909E0FEA3E012
:10098E00FFC39496EE940040030211C0EF4E7038F0
:10099E00E024BBF582E43400F583E0FFB457069003
:1009AE00021E7457F0EFB4520690021E7452F0EF0E
:1009BE0064576014EF6452600F90021E7455F090ED
:1009CE003909E4F0A37496F090021EE0FF645760BC
:1009DE0005EF6452703390390AE024BBF582E4349B
:1009EE0000F583E0FF643A6004EFB43B2390390ACC
:1009FE00E0FF124DFC903910EFF024FFFEE434FFBF
:100A0E00903909F0A3CEF0800790021FE04402F067
:100A1E0090021FE030E0030211AF9001ECE01233C0
:100A2E00A10A5D010B30020B84030C07070CD00CDE
:100A3E000DA20D0E1B0E0E960F0EEB100F67110F63
:100A4E00E01210C213119014119F15000011AC90FA
:100A5E00021EE06457704890390AE004FF1293209A
:100A6E00903907EEF0A3EFF0C3EE64809480402F30
:100A7E00903907E0FEA3E0FF9428EE648094804056
:100A8E0017D3EF940EEE64809481500C9036EFEEF7
:100A9E00F0A3EFF0D211800790021FE04408F0900F
:100AAE00021EE06452707390392A74FFF0A374A092
:100ABE00F0A374A4F07B017A01795412BB869039AD
:100ACE009374FFF0A374A0F0A374A8F09000B1E0AB
:100ADE00FEA3E0FF7C007D0A12310D903996EEF0F8
:100AEE00A3EFF07B017A39791B123D1490392A74E9
:100AFE0001F0A37439F0A3741BF07B017A017954D1
:100B0E0012BB8690392A74FFF0A374A0F0A374ABC5
:100B1E00F07B017A01795412BB86E49001ECF0026D
:100B2E0011AC90021EE06457704490390AE004FF45
:100B3E00129320903907EEF0A3EFF0C3EE64809489
:100B4E0080402B903907E0FEA3E0FFEE6480948096
:100B5E004015D3EF9405EE64809480500A9036EDE4
:100B6E00EEF0A3EFF0800790021FE04408F0E4904F
:100B7E0001ECF00211AC90021EE0645270739039D9
:100B8E002A74FFF0A374A0F0A374ADF07B017A0178
:100B9E00795412BB8690399374FFF0A374A0F0A31E
:100BAE0074A8F0900200E0FEA3E0FF7C007D0A1224
:100BBE0030B8903996EEF0A3EFF07B017A39791BBD
:100BCE00123D1490392A7401F0A37439F0A3741BEA
:100BDE00F07B017A01795412BB8690392A74FFF0AA
:100BEE00A374A0F0A374ABF07B017A01795412BB0D
:100BFE0086E49001ECF00211AC90021EE064577096
:100C0E004690390AE004FF129320903907EEF0A3C4
:100C1E00EFF0C3EE64809480402D903907E0FEA380
:100C2E00E0FF9405EE648094804015D3EF943CEE83
:100C3E0064809480500A9036F1EEF0A3EFF08007B6
:100C4E0090021FE04408F090021EE06452706B9018
:100C5E00399374FFF0A374A0F0A374A8F09000B8B9
:100C6E00E0FFA3E0903996CFF0A3EFF07B017A3945
:100C7E00791B123D1490392A74FFF0A374A0F0A3CF
:100C8E0074B1F07B017A01795412BB8690392A74C3
:100C9E0001F0A37439F0A3741BF07B017A0179542F
:100CAE0012BB8690392A74FFF0A374A0F0A374AB24
:100CBE00F07B017A01795412BB86E49001ECF002CC
:100CCE0011AC90021EE064526003020D9A90392A14
:100CDE0074FFF0A374A0F0A374B5F07B017A0179D0
:100CEE005412BB8690399374FFF0A374A0F0A374D2
:100CFE00A8F09036C9E0FFA3E0903996CFF0A3EFAD
:100D0E00F07B017A39791B123D1490392A7401F067
:100D1E00A37439F0A3741BF07B017A01795412BBD2
:100D2E008690392A74FFF0A374A0F0A374B9F07BF7
:100D3E00017A01795412BB8690399374FFF0A37433
:100D4E00A0F0A374A8F09036C7E0FFA3E090399608
:100D5E00CFF0A3EFF07B017A39791B123D14903955
:100D6E002A7401F0A37439F0A3741BF07B017A018D
:100D7E00795412BB8690392A74FFF0A374A0F0A3A5
:100D8E0074ABF07B017A01795412BB86E49001ECCE
:100D9E00F00211AC90021EE06452706990392A7410
:100DAE00FFF0A374A0F0A374BBF07B017A01795419
:100DBE0012BB8690399374FFF0A374A0F0A374A8AD
:100DCE00F09036CDE0FF903996E4F0A3EFF07B0182
:100DDE007A39791B123D1490392A7401F0A37439B3
:100DEE00F0A3741BF07B017A01795412BB86903903
:100DFE002A74FFF0A374A0F0A374ABF07B017A0108
:100E0E00795412BB86E49001ECF00211AC90021EF4
:100E1E00E06452706B90392A74FFF0A374A0F0A3B3
:100E2E0074BFF07B017A01795412BB8690399374AA
:100E3E00FFF0A374A0F0A374A8F09036CBE0FFA34C
:100E4E00E0903996CFF0A3EFF07B017A39791B123F
:100E5E003D1490392A7401F0A37439F0A3741BF079
:100E6E007B017A01795412BB8690392A74FFF0A364
:100E7E0074A0F0A374ABF07B017A01795412BB8697
:100E8E00E49001ECF00211AC90021EE06452704549
:100E9E0090392A74FFF0A374A0F0A374C3F07B0101
:100EAE007A01795412BB8690392A7401F0A37439F1
:100EBE00F0A37416F07B017A01795412BB86903937
:100ECE002A74FFF0A374A0F0A374ABF07B017A0137
:100EDE00795412BB86E49001ECF00211AC90021E24
:100EEE00E06452706CFF900000E0B4FF027F02904D
:100EFE00399374FFF0A374A0F0A374A8F0A3E4F0E8
:100F0E00A3EFF07B017A39791B123D1490392A74C4
:100F1E00FFF0A374A0F0A374D0F07B017A01795492
:100F2E0012BB8690392A7401F0A37439F0A3741B96
:100F3E00F07B017A01795412BB8690392A74FFF046
:100F4E00A374A0F0A374ABF07B017A01795412BBA9
:100F5E0086E49001ECF00211AC90021EE064527037
:100F6E006990399374FFF0A374A0F0A374A8F09065
:100F7E00000CE0FF903996E4F0A3EFF07B017A3994
:100F8E00791B123D1490392A74FFF0A374A0F0A3BC
:100F9E0074D4F07B017A01795412BB8690392A748D
:100FAE0001F0A37439F0A3741BF07B017A0179541C
:100FBE0012BB8690392A74FFF0A374A0F0A374AB11
:100FCE00F07B017A01795412BB86E49001ECF002B9
:100FDE0011AC90021EE0645260030210BA7B0CFA50
:100FEE00F9F8900217E0FCA3E0FDA3E0FEA3E0FFFA
:100FFE00123271CCE8CCCDE9CDCEEACECFEBCFE438
:10100E007B05FAF9F81231E6ECC0E0EDC0E0EEC077
:10101E00E0EFC0E0E47B0CFAF9F8900217E0FCA3D5
:10102E00E0FDA3E0FEA3E0FF123271E47B3CFAF98F
:10103E00F81231E6D0E0FBD0E0FAD0E0F9D0E0F8DB
:10104E00EF2BFFEE3AFEED39FDEC38FC9039937440
:10105E00FFF0A374A0F0A374D8F0A31233387B0171
:10106E007A39791B123D1490392A74FFF0A374A0BB
:10107E00F0A374DCF07B017A01795412BB869039AF
:10108E002A7401F0A37439F0A3741BF07B017A016A
:10109E00795412BB8690392A74FFF0A374A0F0A382
:1010AE0074ABF07B017A01795412BB86E49001ECAB
:1010BE00F00211AC90021EE06457704E90390AE0B7
:1010CE0004FF129320903907EEF0A3EFF0C3EE6405
:1010DE008094804035903907E0FEA3E0FFEE6480F7
:1010EE009480401FD3EF9401EE648094805014EFEF
:1010FE0064014E700790021604F0800EE490021602
:10110E00F0800790021FE04408F090021EE0645247
:10111E00706990399374FFF0A374A0F0A374A8F0D3
:10112E00900204E0FF903996E4F0A3EFF07B017A91
:10113E0039791B123D1490392A74FFF0A374A0F074
:10114E00A374E0F07B017A01795412BB8690392AA0
:10115E007401F0A37439F0A3741BF07B017A01794A
:10116E005412BB8690392A74FFF0A374A0F0A374B6
:10117E00ABF07B017A01795412BB86E49001ECF05E
:10118E00801CE49001ECF0903909F0A37496F08085
:10119E000DE49001ECF0903909F0A37496F04387BA
:1011AE001090390AE004F07006903909E004F0025C
:1011BE000987C2129001FAE004F0E0C3949640024F
:1011CE00E4F0E49001F2F090021EE0645760030236
:1011DE0012BBA3E0D39400401F90392A74FFF0A3F2
:1011EE0074A0F0A374E4F07B017A01795412BB86EB
:1011FE00E4900204F00212BB90392A74FFF0A3743B
:10120E00A0F0A374EBF07B017A01795412BB8690A7
:10121E0036EFE0FFA3E09036C9CFF0A3EFF09036A3
:10122E00EDE0FFA3E09036C7CFF0A3EFF09036F1DC
:10123E00E0FEA3E0FF9036CBEEF0A3EFF09000B807
:10124E00EEF0A3EFF0900216E0900204F0903995C4
:10125E007401F0A37436F0A374C9F0A3E4F0A37480
:10126E0002F07B107D097C0C7F50128D9790399582
:10127E007401F0A37436F0A374C7F0A3E4F0A37462
:10128E0002F07B107D117C0C7F50128D979039955A
:10129E007401F0A37436F0A374CBF0A3E4F0A3743E
:1012AE0002F07B107D137C0C7F50128D9790021EE6
:1012BE00E0B45703D38001C3500302136B90021F97
:1012CE00E0D39400500302136BE4903909F0A3F0BD
:1012DE0090390AE02454F582E43401F583E4F043B6
:1012EE00871090390AE004F07006903909E004F096
:1012FE00903909E07004A3E0649670D478547C01B0
:10130E007D017BFF7AA079F212366590399374FFD6
:10131E00F0A374A0F0A374A8F090021FE0FF903920
:10132E0096E4F0A3EFF07B017A39791B123D14900D
:10133E00392A7401F0A37439F0A3741BF07B017A7F
:10134E0001795412BB8690392A74FFF0A374A0F071
:10135E00A374ABF07B017A01795412BB86E4903909
:10136E001AF0903909F0A3F090390AE02454F5826E
:10137E00E43401F583E0FF600690391AE02FF0EFB8
:10138E006003021416903909F0A37496F090399305
:10139E0074FFF0A374A0F0A374A8F090391AE0FFC4
:1013AE00903996E4F0A3EFF07B017A39791B123D68
:1013BE001490392A74FFF0A374A0F0A374F9F07B93
:1013CE00017A01795412BB8690392A7401F0A37404
:1013DE0039F0A3741BF07B017A01795412BB86900D
:1013EE00392A74FFF0A374A0F0A374ABF07B017ADA
:1013FE0001795412BB867B017A017954123D1A7B16
:10140E00FF7AA079FD123D1A43871090390AE00445
:10141E00F07006903909E004F0C390390AE0949612
:10142E00903909E094005003021376300232903660
:10143E00D1E0FF900204E06F60267D027C007F0801
:10144E007E0012B8A1900204E0B401077F3112B9F8
:10145E002B80057F3012B92B900204E09036D1F02C
:10146E0030023D900227E0FEA3E0FF9000B8E06E50
:10147E007003A3E06F60297D027C007F127E001254
:10148E00B8A19000B8E0FEA3E0FF7D037C0012A29D
:10149E001D9000B8E0FFA3E0900227CFF0A3EFF07D
:1014AE0030024490390DE0FEA3E0FF9000B1E06EF3
:1014BE007003A3E06F60307D047C007F0F7E00120E
:1014CE00B8A19000B1E0FEA3E0FF7C007D0A1231CE
:1014DE000D7D037C0012A21D9000B1E0FFA3E090F1
:1014EE00390DCFF0A3EFF0E490000CF0900000E087
:1014FE00FD700790000CE04401F0900204E07006CD
:10150E0090000C7407F02002030215BA903906E021
:10151E006D70030215BA7D077C007F037E0012B842
:10152E00A1900000E0FFC36480948040339003F8E4
:10153E00E075F00CA4248CF582E43438F583EF3397
:10154E0095E0FE75F003EF123375EE75F003A425EA
:10155E0083F583E0FBA3E0FAA3E0F912C181804496
:10156E009003F8E075F00CA42429F582E43438F5E4
:10157E0083C083C082900000E0FF3395E0FEC3E499
:10158E009FFFE49EFED082D08375F003EF12337579
:10159E00EE75F003A42583F583E0FBA3E0FAA3E048
:1015AE00F912C181900000E0903906F0301109C2A5
:1015BE00057F0812C1FE8007D2057F0812C1FE907A
:1015CE000204E0FF7004C211C215EFB4010520152C
:1015DE0002D211900000E0B40114C2057F0112C1C5
:1015EE00FEC2057F0212C1FED215C211800ED205B7
:1015FE007F0112C1FED2057F0212C1FE4387100287
:02160E00069D37
:0116100022B7
:108AAE00C205E4FDFCFFFE12B8A19036CBE0FEA39A
:108ABE00E0FFC39405EE94004009D3EF943CEE948E
:108ACE000040347BFF7AA079FF12C1819036CBE44F
:108ADE00F0A37414F09039957401F0A37436F0A3DA
:108AEE0074CBF0A3E4F0A37402F07B107D137C0C26
:108AFE007F50128D97D2059036C9E0FEA3E0FFC3DA
:108B0E009428EE94004009D3EF940EEE9401403475
:108B1E007BFF7AA1790512C1819036C9E4F0A37466
:108B2E00D2F09039957401F0A37436F0A374C9F0A5
:108B3E00A3E4F0A37402F07B107D097C0C7F50122D
:108B4E008D97D2059036C7E0FEA3E0FFC3EE9400EA
:108B5E004009D3EF9405EE940040347BFF7AA1795F
:108B6E000B12C1819036C7E4F0A37404F0903995CE
:108B7E007401F0A37436F0A374C7F0A3E4F0A374E9
:108B8E0002F07B107D117C0C7F50128D97D20590D8
:108B9E000204E0FFC394004006EFD39401402E7B05
:108BAE00FF7AA1790E12C1819002047401F09039FE
:108BBE0095F0A37402F0A37404F0A3E4F0A304F000
:108BCE007B107D087C0C7F50128D97D20590021D74
:108BDE00E0FFC394324006EFD3946440307BFF7ABB
:108BEE00A1791312C18190021D7432F090399574DF
:108BFE0001F0A37402F0A3741DF0A3E4F0A304F03B
:108C0E007B107D157C0C7F50128D97D20530051090
:108C1E001291BF12B2FCEF7003EE640170F57F008B
:018C2E002223
:10BAA10020202020202020202020002020202D2D9B
:10BAB10020202000202020202020202020202000C5
:10BAC10052554E200053544F50002020202020205A
:10BAD100202020202020003A002500202053454628
:10BAE10020202000204E2E200020742020002054F1
:10BAF100202000203534382E303420002020202012
:10BB0100202020200020205B6D696E5D20005B43BA
:05BB11005D0020200092
:10B6F800903927EEF0A3EFF08EF01233C7B725008C
:10B7080002B71D0008B72D0010B7350040B73D013E
:10B71800000000B782126F79126209805D12458EAF
:10B7280012620980551264E7126209804D127D2A5F
:10B738001262098045D2147F017E0012BEBFC21476
:10B748009000B7E0B40105E4F012C0E2900204E012
:10B75800700404F08005E4900204F09039957401B7
:10B76800F0A37402F0A37404F0A3E4F0A304F07B44
:10B77800107D087C0C7F50128D97E4903927F0A338
:02B78800F022AD
:106F7900128103E4903929F0A3F07F9E12C2EA7DC1
:106F8900057C007F0C7E0012B8A19036C9E0FEA3F3
:106F9900E0FF7D037C0012A21D7D047C007F0E7E34
:106FA9000012B8A19036C7E0FEA3E0FF7D017C0086
:106FB90012AB7E7D037C007F0C7E0012B8A1903657
:106FC900CBE0FEA3E0FF7D037C0012A21D7F9C1293
:106FD900C2EA903929E07002A3E060030271F91254
:106FE900B2FC903929EEF0A3EFF08EF01233C7719D
:106FF9001B00027010000871B9001071CA004071BD
:10700900E90800000071EF7D057C007F0C7E00120D
:10701900B8A19036C9E0FEA3E0FF7D037C0012A26F
:107029001D7F9F12C2EA9036C9E0FEA3E0FF9039A6
:107039003F7403F07B0E7A017D287C001278F3906F
:1070490036C9EEF0A3EFF07D047C007F0E7E0012BE
:10705900B8A19036C7E0FEA3E0FF7D017C0012AB2A
:107069007E9036C7E0FEA3E0FF90393F7403F07BC2
:10707900057A00E4FDFC1278F39036C7EEF0A3EF31
:10708900F07F9C12C2EAE4900000F0D21190021441
:10709900E07004A3E06428700A900214F0A3741449
:1070A900F08007E4900214F0A3F0E49036BDF07B81
:1070B9000190399504F0A37436F0A374C9F0A3E4E0
:1070C900F0A37402F07B107D097C0C7F50128D9720
:1070D9009039957401F0A37436F0A374C7F0A3E452
:1070E900F0A37402F07B107D117C0C7F50128D97F8
:1070F9009039957401F0A37436F0A374BDF0A3E43C
:10710900F0A304F07B107D177C0C7F50128D970241
:1071190071EF7D037C007F0C7E0012B8A19036CB05
:10712900E0FEA3E0FF7D037C0012A21D7F9F12C237
:10713900EA9036CBE0FEA3E0FF90393F7403F07B81
:107149003C7A007D057C001278F39036CBEEF0A3F3
:10715900EFF0127B1C9036CBE0FFA3E09000B8CF94
:10716900F0A3EFF07F9C12C2EAE49036BDF07B01F8
:1071790090399504F0A37436F0A374CBF0A3E4F02E
:10718900A37402F07B107D137C0C7F50128D9790B5
:1071990039957401F0A37436F0A374BDF0A3E4F03B
:1071A900A304F07B107D177C0C7F50128D978036DD
:1071B90012ADDB126A659039297408F0A3E4F080F6
:1071C900259036BDE0FF128C2F12B4627F1E7E001F
:1071D9007D007C0012BF56E4903929F0A3F08006A7
:1071E9007F9C12C2EA22E4903929F0A3F0026FDBF6
:0171F9002273
:10458E00E4903929F0A3F09036BDE090392DF01269
:10459E00AC4B9036BDE0FF12B022903929E0640892
:1045AE007002A3E070030249D212B2FC903929EED8
:1045BE00F0A3EFF08EF01233C748500002466300AE
:1045CE000848E40010498300404625020045E704F0
:1045DE000049C20800000049C890392DE004F0E0FF
:1045EE00D3941040037401F090392DE0FF12B022E5
:1045FE00E490392BF0A3F043871090392CE004F0AF
:10460E00700690392BE004F090392BE0B413E8A338
:10461E00E0B488E30249C890392DE014F0E0C39469
:10462E000150037410F090392DE0FF12B022E49087
:10463E00392BF0A3F043871090392CE004F070066C
:10464E0090392BE004F090392BE0B413E8A3E0B4DA
:10465E0088E30249C87B017A39793090392DE0FD23
:10466E0090394B7450F012A51090392FEFF0C364AF
:10467E00809480500302476090392DE0FF7B017AD1
:10468E003679BD90394FE4F0A37411F012BD741257
:10469E008AAEEF702290392DE0FF7B017A3679BD1C
:1046AE0090393DE4F0A37411F012947812AC4B9053
:1046BE00392DE0FF12B0229039957401F0A37436B3
:1046CE00F0A374BDF0A3E4F0A304F07B107D057C91
:1046DE000C7F50128D977D047C007F1B7E0012B8DC
:1046EE00A19003F8E075F003A42454F582E5F034AC
:1046FE0037F583E0FBA3E0FAA3E0F912C18190360F
:10470E00CBE0FEA3E0FF127B1C9036CBE0FFA3E0D4
:10471E009000B8CFF0A3EFF0E490392BF0A3F04364
:10472E00871090392CE004F0700690392BE004F0DD
:10473E0090392BE0B475E8A3E0B430E37D047C003F
:10474E007F1B7E0012B8A17BFF7ABA79A112C181BC
:10475E0080607D047C007F1B7E0012B8A19003F860
:10476E00E075F003A4240CF582E5F03437F583E010
:10477E00FBA3E0FAA3E0F912C181E490392BF0A378
:10478E00F043871090392CE004F0700690392BE03E
:10479E0004F090392BE0B475E8A3E0B430E37D0467
:1047AE007C007F1B7E0012B8A17BFF7ABA79A11222
:1047BE00C181E4900000F0900214F0A3F07B019010
:1047CE00399504F0A37436F0A374C9F0A3E4F0A3F2
:1047DE007402F07B107D097C0C7F50128D979039FE
:1047EE00957401F0A37436F0A374C7F0A3E4F0A39C
:1047FE007402F07B107D117C0C7F50128D979039D6
:10480E00957401F0A37436F0A374CBF0A3E4F0A377
:10481E007402F07B107D137C0C7F50128D979039B3
:10482E00957401F0A37436F0A374BDF0A3E4F0A365
:10483E0004F07B107D177C0C7F50128D97D21102E5
:10484E0049C87D047C007F0F7E0012B8A17B017ADF
:10485E003679BE7D087C0012905D90392EEFF0BF48
:10486E00FF107F9C12C2EA90392DE0FF12B0220297
:10487E0049C890392EE070147B017A3679BE903992
:10488E002DE0FD90394B7450F012A51090392DE0AB
:10489E00FF9036BDF07B017A3679BD90393DE4F05C
:1048AE00A37411F012947890392DE0FF12B022E427
:1048BE0090392BF0A3F043871090392CE004F07060
:1048CE000690392BE004F090392BE0B475E8A3E0A4
:1048DE00B430E30249C890392DE0F4049036BDF0AF
:1048EE0078BE7C367D017BFF7ABA79AC1236659044
:1048FE00392DE0FF7B017A3679BD90393DE4F0A386
:10490E007411F01294787F9C12C2EA7D047C007FB1
:10491E001B7E0012B8A19003F8E075F003A4243CAE
:10492E00F582E5F03437F583E0FBA3E0FAA3E0F976
:10493E0012C181E490392BF0A3F043871090392CEB
:10494E00E004F0700690392BE004F090392BE0B4BF
:10495E0075E8A3E0B430E37D047C007F1B7E00127B
:10496E00B8A17BFF7ABA79B512C18190392DE0FFDB
:10497E0012B02280457B017A39793090392DE0FDD5
:10498E0090394B7450F012A51090392FEFF0C3648C
:10499E00809480401290392DE0FF128C2FE49039D4
:1049AE0029F0A3F012B4627F1E7E007D007C0012FF
:1049BE00BF5680067F9C12C2EA22E4903929F0A3EA
:0449CE00F00245A806
:0149D20022C2
:10B02200EF24FE90393DF090393BE4F0A37406F032
:10B03200E4903939F0A3F090393DE0FFC364809485
:10B04200815004EF2410F090393DE0D36480949055
:10B052004004E024F0F090393BE0FCA3E0FD7F0BDC
:10B062007E0012B8A190393DE0FF3395E0FE7D02EB
:10B072007C0012A21D7B017A39793E90393DE0FDB8
:10B0820090394B7450F012A51090393BE0FCA3E0CC
:10B09200FD7F0F7E0012B8A17B017A39793E12C181
:10B0A2008190393DE004F090393CE024FFF0903982
:10B0B2003BE034FFF090393AE004F0700690393901
:10B0C200E004F0C390393AE09404903939E06480A6
:07B0D2009480500302B03925
:01B0D9002254
:1064E700E4903929F0A3F090022EF090392DF012A4
:1064F700AD1390022EE0FF12A8DC903929E0640862
:106507007002A3E070030267A612B2FC903929EE6D
:10651700F0A3EFF08EF01233C766D2000265BF001A
:10652700086747001067840040657F0200654004E4
:1065370000679608000000679C90392DE004F0E0A2
:10654700C3648094894002E4F090392DE0FF12A8DB
:10655700DCE490392BF0A3F043871090392CE0044A
:10656700F0700690392BE004F090392BE0B413E873
:10657700A3E0B488E302679C90392DE014F0E0C3F0
:106587006480948050037408F090392DE0FF12A8BE
:10659700DCE490392BF0A3F043871090392CE0040A
:1065A700F0700690392BE004F090392BE0B413E833
:1065B700A3E0B488E302679C90392DE0FDD36480A3
:1065C700948050030266C17B017A02792F90394B80
:1065D700744DF012A510C3EF648094804079903910
:1065E7002DE0FF7B017A02792E903936E4F0A3740F
:1065F700CEF012BDCE7D047C007F1B7E0012B8A1B9
:106607009003F8E075F003A42454F582E5F03437DD
:10661700F583E0FBA3E0FAA3E0F912C181E4903926
:106627002BF0A3F043871090392CE004F07006900C
:10663700392BE004F090392BE0B475E8A3E0B430CF
:10664700E37D047C007F1B7E0012B8A17BFF7ABA32
:1066570079A112C18180637D047C007F1B7E0012BB
:10666700B8A19003F8E075F003A4240CF582E5F0D7
:106677003437F583E0FBA3E0FAA3E0F912C181E424
:1066870090392BF0A3F043871090392CE004F07079
:106697000690392BE004F090392BE0B475E8A3E0BD
:1066A700B430E37D047C007F1B7E0012B8A17BFF22
:1066B7007ABA79A112C18102679C12368212AD1390
:1066C70090392DE0FF12A8DC02679C7D047C007FD7
:1066D7000F7E0012B8A17B017A02792F7D087C001A
:1066E70012905D90392EEFF0BFFF0B90392DE0FF30
:1066F70012A8DC02679C90392EE070147B017A02A5
:10670700792F90392DE0FD90394B744DF012A5107B
:1067170090392DE0FF90022EF07B017A02792E90BE
:106727003935E4F0A374CEF0128EFA90392DE0FFDC
:1067370012A8DC7F327E007D007C0012BF56805598
:10674700E490022EF09003F8E075F003A424ECF532
:1067570082E5F03438F583E0FBA3E0FAA3E0F978AB
:106767002F7C027D011236651249D37F9C12C2EA43
:1067770012AD1390392DE0FF12A8DC801890392D47
:10678700E0FF129A9B12B4627F9C12C2EA80067FD6
:0F6797009C12C2EA22E4903929F0A3F0026501B6
:0167A60022D0
:10A8DC00EF24FE903933F0903931E4F0A37406F094
:10A8EC00E490392FF0A3F0903933E0FFC3648094E7
:10A8FC00805004EF2409F0903933E0D364809488BD
:10A90C004004E024F7F0903931E0FCA3E0FD7F0B2C
:10A91C007E0012B8A1903933E0FF3395E0FE7D0242
:10A92C007C0012A21D903931E0FCA3E0FD7F0F7E6C
:10A93C000012B8A1903933E0701F9003F8E075F065
:10A94C0003A424ECF582E5F03438F583E0FBA3E0B6
:10A95C00FAA3E0F912C18180227B017A3979349013
:10A96C003933E0FD90394B744DF012A5107B017A10
:10A97C0039793412C1817F2012B92B903933E0041C
:10A98C00F0903932E024FFF0903931E034FFF09050
:10A99C003930E004F0700690392FE004F0C39039A0
:10A9AC0030E0940490392FE064809480500302A826
:01A9BC00F3A7
:01A9BD002277
:1049D3009036D2E0FFA3E0900200CFF0A3EFF0E423
:1049E30090393DF0A3F0A3F0A3F01200037F9C12D3
:1049F300C2EAE490022EF0903937F0A3F09000B8A9
:104A0300E0FEA3E0FF7C007D031230A67D64CFCDE2
:104A1300CFCECCCE12310DEF0490023CF0E075F016
:104A2300B4A4FF900238E5F0F0A3EFF090023D74D8
:104A330004F0129DF590023CE0FF7E0012AEA190BF
:104A4300023DE0FF7E0012A7EF90023DE0FD7C00F7
:104A53007E047FD81230B890393BEEF0A3EFF0908C
:104A630001F4E0FCA3E0FDA3E0FEA3E0FF903945E1
:104A7300123338E4903933F0A3F0903937F0A3F0D0
:104A8300900200E0FEA3E0FF7C007D0A1230B890A4
:104A93003935EEF0A3EFF090393DEEF0A3EFF024BB
:104AA300E7FFEE34FFFE903939F0A3EFF0C3EE6475
:104AB3008094805007E4903939F0A3F0D390393AC9
:104AC300E094FF903939E0648094804006E4F0A3D9
:104AD30074FFF090393BE0FEA3E0FFD3903936E05A
:104AE3009FEE6480F8903935E06480984005EEF0DD
:104AF300A3EFF090393AE090023EF07D027C007F14
:104B0300017E0012B8A17BFF7ABA79C112C18190EC
:104B13003945E0F8A3E0F9A3E0FAA3E0FB9001F440
:104B2300E0FCA3E0FDA3E0FEA3E0C39BFFEE9AFE3F
:104B3300ED99FDEC98FC903941123338903941E0FE
:104B4300FCA3E0FDA3E0FEA3E0FFE47B64FAF9F835
:104B5300123271903941123338903941E0FCA3E0AD
:104B6300FDA3E0FEA3E0FFEE540FFEE4903931EE27
:104B7300F0A3EFF090023CE0FD7C0012310D903980
:104B83002FEEF0A3EFF0C3903934E09FEE6480F88A
:104B9300903933E06480984003024D04903938E043
:104BA30004F07006903937E004F0D3903938E0947C
:104BB300B5903937E0648094804006E4F0A374B57F
:104BC300F0900200E0FEA3E0FF7C007D0A1230B803
:104BD30090392FEEF0A3EFF0C390393EE09FEE64DF
:104BE30080F890393DE0648098500F90392FE0FFB2
:104BF300A3E090393DCFF0A3EFF090393BE0FEA363
:104C0300E0FFD3903930E09FEE6480F890392FE0D5
:104C13006480984005EEF0A3EFF090023DE0FB9036
:104C23003935E0FCA3E0FDCFEBCF7E001230A67C4C
:104C3300007D1412310DEEC0E0EFC0E090392FE09B
:104C4300FCA3E0FDCFEBCF7E001230A67C007D14E9
:104C530012310D903954EEF0A3EFF0903934E02483
:104C630034FF903933E03400FE903938E02434FBCC
:104C7300903937E03400FAD0E0FDD0E0FC125591D2
:104C830090392FE0FEA3E0FF903935EEF0A3EFF06B
:104C930024E7FFEE34FFFE903939F0A3EFF0C3EEC3
:104CA300648094805007E4903939F0A3F0D39039AD
:104CB3003AE094FF903939E0648094804006E4F050
:104CC300A374FFF090393AE0FF903938E0243EF5C1
:104CD30082E43402F583EFF0903937E0FFA3E090EC
:104CE3003933CFF0A3EFF07D037C007F057E001204
:104CF300B8A190392FE0FEA3E0FF7D037C0012A250
:104D03001DE490392FF0A3F0900238E0FEA3E0FFFA
:104D1300D3903932E09F903931E09E404390393748
:104D2300E0FFA3E090023ACFF0A3EFF090023D74CE
:104D33000CF090393DE0FCA3E0FDD39464EC648077
:104D43009480400C7E047FD812310D90023DEFF029
:104D530090023DE0C394044003024DFB7404F0222F
:104D630012B2FC90393FEEF0A3EFF07003EE64084B
:104D73006003024B12903937E0FFA3E090023ACF71
:104D8300F0A3EFF090023D740CF090393DE0FCA3EA
:104D9300E0FDD39464EC64809480400C7E047FD85F
:104DA30012310D90023DEFF090023DE0C3940450A8
:104DB300037404F07D027C007F017E0012B8A17BA6
:104DC300FF7ABA79C612C181E490393FF0A3F0FFAC
:104DD300FE4387100FBF00010EBE75F5BF30F29082
:104DE300393FE064087002A3E0600D12B2FC903911
:084DF3003FEEF0A3EFF080E7B2
:014DFB002295
:059A9B0090392FEFF0EF
:109AA000D3648094805003029B9D7B017A02792FBE
:109AB000E0FD90394B744DF012A510C3EF64809413
:109AC00080407990392FE0FF7B017A02792E90391E
:109AD00036E4F0A374CEF012BDCE7D047C007F1B73
:109AE0007E0012B8A19003F8E075F003A42454F5A9
:109AF00082E5F03437F583E0FBA3E0FAA3E0F91246
:109B0000C181E4903930F0A3F0438710903931E0FF
:109B100004F07006903930E004F0903930E0B4750C
:109B2000E8A3E0B430E37D047C007F1B7E0012B824
:109B3000A17BFF7ABA79A112C18180617D047C008A
:109B40007F1B7E0012B8A19003F8E075F003A424F7
:109B50000CF582E5F03437F583E0FBA3E0FAA3E0EF
:109B6000F912C181E4903930F0A3F04387109039A5
:109B700031E004F07006903930E004F0903930E0C4
:109B8000B475E8A3E0B430E37D047C007F1B7E0065
:109B900012B8A17BFF7ABA79A112C1812290020387
:109BA0007401F090392FE0FF129F0A7F017E0012AE
:0A9BB000BEBF12C245E4900203F0AC
:019BBA002288
:107D2A001271FAE4903929F0A3F012B2FC903929C1
:107D3A00EEF0A3EFF08EF01233C77D7000027D647F
:107D4A0000087E0000107E3000407E7E02007E79B0
:107D5A0004007E83080000007EA812C06612A11CDF
:107D6A001271FA027EA87D057C007F1C7E0012B883
:107D7A00A17BFF7ABA79CB12C1817D037C007F1C7B
:107D8A007E0012B8A17BFF7ABA79CB12C1817D033A
:107D9A007C007F147E0012B8A19001FCE0FEA3E0F3
:107DAA00FF7D037C0012A21D7F9F12C2EA9001FC94
:107DBA00E0FEA3E0FF90393F7402F07B1E7A00E4F4
:107DCA00FDFC1278F39001FCEEF0A3EFF0E49000D2
:107DDA00B5F0A3F07F9C12C2EA9001FCE07002A306
:107DEA00E06006127F1C1282B2E4903929F0A3F0F7
:107DFA001271FA027EA87D057C007F1C7E0012B8F3
:107E0A00A17BFF7ABA79CB12C1817D037C007F1CEA
:107E1A007E0012B8A17BFF7ABA79CB12C181129780
:107E2A00161271FA80781200037F9E12C2EA7D044C
:107E3A007C007F057E0012B8A19003F8E025E024BB
:107E4A0006F582E4342AF583E493FE740193CAEEBC
:107E5A00CAF97BFF12C181E4FF12B3AFBF01061258
:107E6A00B0DA1267A77F9C12C2EA1271FA802F1247
:107E7A00C223802A129CDA80257F9C12C2EA90399A
:107E8A00957401F0A37400F0A374B4F0A3E4F0A312
:107E9A0004F07B107D067C0C7F50128D9722903661
:107EAA00CFE0FEA3E0FF90392BE06E7003A3E06FF2
:107EBA007003027D347D047C007F0F7E0012B8A11E
:107ECA009001EAE0FEA3E0FF7D057C0012A21D7B83
:107EDA00FF7ABA79D812C181900152E0FEA3E0FF7D
:107EEA007D027C0012AB7E7BFF7ABA79D812C181FF
:107EFA009036CFE0FEA3E0FF7D027C0012AB7E90BD
:107F0A0036CFE0FFA3E090392BCFF0A3EFF0027D4C
:017F1A003432
:017F1B002243
:10A11C009003F8E0FF90392DF07E0012B24712B296
:10A12C00FC90392EEEF0A3EFF08EF01233C7A1DEC7
:10A13C000100A1940200A14E0400A2150800000029
:10A14C00A12A90392DE0C394035005E004F080055A
:10A15C00E490392DF090392DE0FF7E0012B247E4E7
:10A16C00903930F0A3F0C3903931E094109039302D
:10A17C00E0648094A750A7438710A3E004F0700616
:10A18C00903930E004F080DE90392DE0D39400401B
:10A19C0005E014F0800690392D7403F090392DE011
:10A1AC00FF7E0012B247E4903930F0A3F0C390392F
:10A1BC0031E09410903930E0648094A7400302A100
:10A1CC002A438710A3E004F07006903930E004F0C5
:10A1DC0080DB90392DE09003F8F09039957401F004
:10A1EC00A37403F0A374F8F0A3E4F0A304F07B10C1
:10A1FC007D047C0C7F50128D9712C06690392DE037
:10A20C00FF7E0012B24702A12AE490392EF0A3F08F
:01A21C00221F
:10B24700EF24FE903936F0903934E4F0A37405F01A
:10B25700E4903932F0A3F0903936E0FFC36480946C
:10B26700805004EF2404F0903936E0D3648094834F
:10B277004004E024FCF0903934E0FCA3E0FD7F10AB
:10B287007E0012B8A1903936E0FF3395E0FE903783
:10B297006C75F018EF123375EE75F018A42583F569
:10B2A70083C083C0829003F8E0D082D08375F00317
:10B2B700123375E0FBA3E0FAA3E0F912C1819039DC
:10B2C70036E004F0903935E024FFF0903934E0346B
:10B2D700FFF0903933E004F07006903932E004F063
:10B2E700C3903933E09405903932E06480948050FC
:04B2F7000302B25E3E
:01B2FB002230
:10971600900226E090392DF07D027C007F0F7E00BE
:1097260012B8A17F9F12C2EA7D027C007F0F7E00E5
:1097360012B8A112B2FC90392EEEF0A3EFF08EF023
:109746001233C79815010097B70200975D04009879
:109756004208000000972E90392DE0C39401500571
:10976600E004F08005E490392DF090392DE025E0F5
:1097760024D2F582E43429F583E493FE740193CA76
:10978600EECAF97BFF12C181E4903930F0A3F0C331
:10979600903931E09410903930E0648094A7508875
:1097A600438710A3E004F07006903930E004F0809F
:1097B600DE90392DE0D394004005E014F080069049
:1097C600392D7401F090392DE025E024D2F582E49C
:1097D6003429F583E493FE740193CAEECAF97BFF3C
:1097E60012C181E4903930F0A3F0C3903931E0948E
:1097F60010903930E0648094A7400302972E438787
:1098060010A3E004F07006903930E004F080DB909D
:10981600392DE0900226F09039957401F0A3740278
:10982600F0A37426F0A3E4F0A304F07B107D077C7C
:109836000C7F50128D977F9C12C2EA22E490392E3B
:08984600F0A3F07F9C12C2EABE
:01984E0022F7
:1067A7007F017E0012BEBFE490392DF0A3F07F9EDB
:1067B70012C2EA7D057C007F157E0012B8A1900207
:1067C7001DE0FF7E007D057C0012A21D7D057C007B
:1067D7007F1A7E0012B8A17BFF7ABA79DA12C181DB
:1067E7007F9C12C2EA90392DE07002A3E060030299
:1067F7006A6412B2FC90392DEEF0A3EFF08EF0121E
:1068070033C768190008688200406A54080000000E
:106817006A5A7D057C007F157E0012B8A190021D83
:10682700E0FF7E007D057C0012A21D7F9F12C2EA59
:1068370090021DE0FF7E009039377405F0A3E4F065
:10684700A3740AF07B647A007D327C001276BF90D5
:10685700021DEFF09039957401F0A37402F0A37450
:106867001DF0A3E4F0A304F07B107D157C0C7F5092
:10687700128D977F9C12C2EA026A5A1200037F9E0A
:1068870012C2EA7D047C007F057E0012B8A1900346
:10689700F8E025E02406F582E4342AF583E493FE44
:1068A700740193CAEECAF97BFF12C1817F0112B34B
:1068B700AFEF640160030269E390021712334400EB
:1068C700000005900217E0FCA3E0FDA3E0FEA3E0B3
:1068D700FF12BF9FE47B0CFAF9F8900217E0FCA3C4
:1068E700E0FDA3E0FEA3E0FF1232719001EAEEF0B3
:1068F700A3EFF0E47B0CFAF9F8900217E0FCA3E0B1
:10690700FDA3E0FEA3E0FF123271CCE8CCCDE9CDC8
:10691700CEEACECFEBCFE47B05FAF9F81231E69059
:106927000152EEF0A3EFF07F017E0012BEBF903957
:106937002FE4F0A304F0903930E0F4049036BDF072
:1069470078BE7C367D017BFF7ABA79AC12366590CA
:106957003930E0FF7B017A3679BD90393DE4F0A309
:106967007411F0129478903930E004F07006903981
:106977002FE004F0D3903930E0941090392FE06481
:1069870080948040B190392FE4F0A304F09039301F
:10699700E0F40490022EF0782F7C027D017BFF7AD1
:1069A700BA79AC123665903930E0FF7B017A02790B
:1069B7002E903935E4F0A374CEF0128EFA90393068
:1069C700E004F0700690392FE004F0D3903930E0FE
:1069D700940890392FE06480948040B17F9C12C264
:1069E700EA12B0DA7D057C007F157E0012B8A1900F
:1069F700021BE0FEA3E0FF7D057C0012A21D7D04C3
:106A07007C007F157E0012B8A1900212E0FEA3E081
:106A1700FF7D057C0012A21D7D037C007F157E0093
:106A270012B8A190020AE0FEA3E0FF7D057C0012E8
:106A3700A21D7D027C007F157E0012B8A190021D69
:106A4700E0FF7E007D057C0012A21D80067F9C1260
:0D6A5700C2EA22E490392DF0A3F00267ECB2
:016A6400220F
:10368200E490392FF0A3F01200037F9C12C2EA12D9
:103692009DF590023CE0FF7E0012AEA190023DE05B
:1036A200FF7E0012A7EF90023DE0FD7C007E047FCA
:1036B200D81230B890393DEEF0A3EFF090023AE024
:1036C200C313FFA3E013903931CFF0A3EFF07D03D2
:1036D2007C007F047E0012B8A1903932E0243EF5CE
:1036E20082E43402F583E02419FFE433FE7D037C97
:1036F2000012A21D7D047C007F037E0012B8A190FF
:10370200023CE0FF7E00903931E0FCA3E0FD123084
:10371200A67D047C0012A21D90023AE0FEA3E0FF07
:1037220090393BEEF0A3EFF0D394C8EE648094801E
:10373200400990393BE4F0A374C8F090023CE0FFEA
:103742007E0012AEA190023DE0FF7E0012A7EF9034
:10375200023EE02419FFE433FE903937F0A3EFF084
:1037620090393DE0FCA3E0FDC39FEE6480F8EC6479
:1037720080985008903937ECF0A3EDF0903939E495
:10378200F0A304F090393BE0FEA3E0FFD390393A76
:10379200E09FEE6480F8903939E06480984003023B
:1037A2003856A3E0243EF582E43402F583E024197E
:1037B200FFE433FE903935F0A3EFF090393DE0FCA1
:1037C200A3E0FDC39FEE6480F8EC648098500890FB
:1037D2003935ECF0A3EDF090023DE0FB903937E093
:1037E200FCA3E0FDCFEBCF7E001230A67C007D145F
:1037F20012310DEEC0E0EFC0E0903935E0FCA3E0FD
:10380200FDCFEBCF7E001230A67C007D1412310D6D
:10381200903954EEF0A3EFF0903939E0FCA3E0FDCB
:103822002433FFE43CFEED2434FBE43CFAD0E0FD1B
:10383200D0E0FC125591903935E0FFA3E0A3CFF020
:10384200A3EFF090393AE004F07006903939E004C1
:10385200F0023786903933E4F0A3740AF0903933DA
:10386200E0FCA3E0FDC3943EEC648094805023907E
:103872003932E02434FF903931E03400FE7B01120A
:10388200B65F903934E02402F0903933E03400F02E
:1038920080CB90392FE064087002A3E07003023CF1
:1038A200AE12B2FC90392FEEF0A3EFF07003EE648B
:1038B200046003023AAF90393BE0FEA3E0FFC390FD
:1038C2003932E09FEE6480F8903931E064809840AC
:1038D20003023AAF903933E4F0A3740AF09039331B
:1038E200E0FCA3E0FDC3943EEC64809480502390FE
:1038F2003932E02434FF903931E03400FEE4FB1227
:10390200B65F903934E02402F0903933E03400F0AD
:1039120080CB903932E004F07006903931E004F047
:1039220090023EE02419FFE433FE903937F0A3EF12
:10393200F090393DE0FCA3E0FDC39FEE6480F8EC1B
:103942006480985008903937ECF0A3EDF090393943
:10395200E4F0A304F090393BE0FEA3E0FFD39039FA
:103962003AE09FEE6480F8903939E0648098400331
:10397200023A27A3E0243EF582E43402F583E024F0
:1039820019FFE433FE903935F0A3EFF090393DE0B2
:10399200FCA3E0FDC39FEE6480F8EC6480985008BD
:1039A200903935ECF0A3EDF090023DE0FB90393711
:1039B200E0FCA3E0FDCFEBCF7E001230A67C007DC1
:1039C2001412310DEEC0E0EFC0E0903935E0FCA3F7
:1039D200E0FDCFEBCF7E001230A67C007D141231C9
:1039E2000D903954EEF0A3EFF0903939E0FCA3E0EA
:1039F200FD2433FFE43CFEED2434FBE43CFAD0E04A
:103A0200FDD0E0FC125591903935E0FFA3E0A3CF41
:103A1200F0A3EFF090393AE004F07006903939E003
:103A220004F0023957903933E4F0A3740AF0903964
:103A320033E0FCA3E0FDC3943EEC64809480502309
:103A4200903932E02434FF903931E03400FE7B01BA
:103A520012B65F903934E02402F0903933E034003A
:103A6200F080CB7D047C007F037E0012B8A190021F
:103A72003CE0FF7E00903931E0FCA3E0FD1230A66D
:103A82007D047C0012A21D7D037C007F047E001257
:103A9200B8A1903932E0243EF582E43402F583E0A5
:103AA2002419FFE433FE7D037C0012A21D90392FFE
:103AB200E064027002A3E06003023894D3903932CA
:103AC200E09405903931E064809480500302389488
:103AD200903933E4F0A3740AF0903933E0FCA3E0A8
:103AE200FDC3943EEC648094805023903932E024EC
:103AF20034FF903931E03400FEE4FB12B65F9039B6
:103B020034E02402F0903933E03400F080CB903975
:103B120032E024FFF0903931E034FFF090023EE0D1
:103B22002419FFE433FE903937F0A3EFF090393DCA
:103B3200E0FCA3E0FDC39FEE6480F8EC6480985043
:103B420008903937ECF0A3EDF0903939E4F0A30492
:103B5200F090393BE0FEA3E0FFD390393AE09FEECC
:103B62006480F8903939E06480984003023C23A3D2
:103B7200E0243EF582E43402F583E02419FFE433C5
:103B8200FE903935F0A3EFF090393DE0FCA3E0FD63
:103B9200C39FEE6480F8EC6480985008903935EC4D
:103BA200F0A3EDF090023DE0FB903937E0FCA3E09A
:103BB200FDCFEBCF7E001230A67C007D1412310DBA
:103BC200EEC0E0EFC0E0903935E0FCA3E0FDCFEBC2
:103BD200CF7E001230A67C007D1412310D90395434
:103BE200EEF0A3EFF0903939E0FCA3E0FD2433FFBF
:103BF200E43CFEED2434FBE43CFAD0E0FDD0E0FCF2
:103C0200125591903935E0FFA3E0A3CFF0A3EFF076
:103C120090393AE004F07006903939E004F0023B42
:103C220053903933E4F0A3740AF0903933E0FCA3E3
:103C3200E0FDC3943EEC648094805023903932E0DE
:103C42002434FF903931E03400FE7B0112B65F90DC
:103C52003934E02402F0903933E03400F080CB7D37
:103C6200047C007F037E0012B8A190023CE0FF7E3C
:103C720000903931E0FCA3E0FD1230A67D047C0007
:103C820012A21D7D037C007F047E0012B8A1903930
:103C920032E0243EF582E43402F583E02419FFE4A5
:0C3CA20033FE7D037C0012A21D0238944A
:013CAE0022F3
:109DF5007D077C00E4FFFE12B8A17BFF7ABA79DC0F
:109E050012C1817D057C00E4FFFE12B8A17BFF7ABB
:109E1500BA79E512C18190022EE0FF3395E0FE7D0F
:109E2500027C0012AB7E7D047C00E4FFFE12B8A12B
:109E35007BFF7ABA79EA12C1817D037C00E4FFFEDB
:109E450012B8A17BFF7ABA79EF12C181E4FDFCFF5C
:109E5500FE12B8A17BFF7ABA79F412C18190395408
:109E6500E4F0A3743FF07B0B7A00FD7C00E4FFFE79
:109E7500125591903954E4F0A3743FF07B327A0087
:109E8500FD7C007F1F7E00125591903954E4F0A3AC
:109E9500743FF0E4FBFAFDFCFFFE12559190395436
:109EA500E4F0A3743FF07B327A00E4FDFC7F32FEE0
:109EB500125591E4903954F0A3F07B05FAFDFCFFAF
:109EC500FE125591E4903954F0A3F07B32FAFDFC73
:109ED5007F2DFE125591903954E4F0A3740CF07B5C
:109EE5002D7A00FD7C007F057E0012559190395436
:109EF500E4F0A37434F07B2D7A00FD7C007F057EB1
:059F050000125591223D
:08AEA100903949EEF0A3EFF037
:10AEA900E4903954F0A3F07B71FAFDFC7F34FE1273
:10AEB9005591E4903954F0A3F07BADFAFDFC7F790C
:10AEC900FE125591E4903954F0A3F07BE9FAFDFCA8
:10AED9007FB5FE125591903949E0FFA3E0A3CFF069
:10AEE900A3EFF0E4FDFC7F0AFE12B8A17BFF7ABA5A
:10AEF90079FD12C18190394BE0FEA3E0FF7D027C10
:10AF09000012A21D903949E0FEA3E0FF90394CE000
:10AF19002FF090394BE03EF07BFF7ABA79FD12C1F0
:10AF29008190394BE0FEA3E0FF7D027C0012A21D57
:10AF39007BFF7ABB790612C181903949E0FEA3E013
:10AF4900FF90394CE02FF090394BE03EF0E0FEA342
:09AF5900E0FF7D027C0012A21D44
:01AF620022CC
:08A7EF00903949EEF0A3EFF0F0
:10A7F700E4903954F0A3F07B34FA7D3FFC7F34FEBC
:10A8070012559190394BE4F0A304F090394AE09047
:10A81700394DF090394BE0FEA3E0FF7C007D051237
:10A82700310DED4C701BA3E0FD3395E0FC903954DE
:10A83700F0A3EDF07B397A007F347E0012559180CA
:10A847001B90394DE0FD3395E0FC903954F0A3EDB2
:10A85700F07B367A007F347E0012559190394CE0B8
:10A8670004F0700690394BE004F090394AE0FF900D
:10A87700394DE02FF0E0C3648094BF40967D067C9D
:10A88700007F0A7E0012B8A17BFF7ABB790F12C145
:10A8970081903949E0FCA3E0FD7E047FD812310D99
:10A8A700A3EEF0A3EFF07C007D6412310D7C007DF8
:10A8B700641230A690394BEEF0A3EFF07D077F0AC4
:10A8C7007E0012B8A190394BE0FEA3E0FF7D037C28
:04A8D7000012A21DAC
:01A8DB00225A
:106A6500E490392BF0A3F07B017A3979D01289189B
:106A75007D057C007F1E7E0012B8A19039D6E0FE10
:106A8500A3E0FF7D027C0012AB7E7F3A12B92B900A
:106A950039D8E0FEA3E0FF7D027C0012AB7E7F3A91
:106AA50012B92B9039DAE0FEA3E0FF7D027C0012DB
:106AB500AB7E7D057C007F087E0012B8A19039D49D
:106AC500E0FEA3E0FF7D027C0012AB7E7F2E12B9B3
:106AD5002B9039D2E0FEA3E0FF7D027C0012AB7E55
:106AE5007F2E12B92B9039D0E0FEA3E0FF7D047C08
:106AF5000012AB7E7BFF7ABB791312C18112B2FC07
:106B050090392BEEF0A3EFF08EF01233C76B1E0019
:106B1500086CEC080000006A6C9039D0E0FFA3E037
:106B250090392DCFF0A3EFF09039D2E0FFA3E0909C
:106B3500392FCFF0A3EFF09039D4E0FFA3E09039DF
:106B450031CFF0A3EFF09039D6E0FFA3E0903933D1
:106B5500CFF0A3EFF09039D8E0FFA3E0903935CF1F
:106B6500F0A3EFF09039DAE0FFA3E0903937CFF0EA
:106B7500A3EFF07F9F12C2EA7D057C007F0A7E00AD
:106B850012B8A1903931E0FEA3E0FF90393F7402BD
:106B9500F07B1F7A007D017C001278F3903931EE8D
:106BA500F0A3EFF07D057C007F0D7E0012B8A1906B
:106BB500392FE0FEA3E0FF90393F7402F07B0C7A99
:106BC500007D017C001278F390392FEEF0A3EFF0F1
:106BD5007D057C007F127E0012B8A190392DE0FE64
:106BE500A3E0FF90393F7404F07BB77A0B7DBC7C42
:106BF500071278F390392DEEF0A3EFF07D057C00B8
:106C05007F207E0012B8A1903933E0FEA3E0FF900B
:106C1500393F7402F07B177A00E4FDFC1278F3909B
:106C25003933EEF0A3EFF07D057C007F237E001263
:106C3500B8A1903935E0FEA3E0FF90393F7402F02A
:106C45007B3B7A00E4FDFC1278F3903935EEF0A336
:106C5500EFF07D057C007F267E0012B8A1903937C4
:106C6500E0FEA3E0FF90393F7402F07B3B7A00E43D
:106C7500FDFC1278F3903937EEF0A3EFF07F9C120C
:106C8500C2EA7F1E7E007D007C0012BF56E490396B
:106C95002BF0A3F090392FE0FCA3E0FDA3E0FAA3CD
:106CA500E0FBA3E0FFA3E090393FCFF0A3EFF09026
:106CB5003935E0FFA3E0903941CFF0A3EFF09039EB
:106CC50037E0FFA3E0903943CFF0A3EFF090392DE3
:106CD500E0FEA3E0FF1287827B017A3979D0128921
:0C6CE5001812ADDB026A6C7F9C12C2EA40
:016CF1002280
:10C0E200D2057F0412C1FE7F0A7E007D007C001211
:10C0F200BF56C2057F0412C1FEC2057F0812C1FEEF
:10C102007FC87E007D007C0012BF56D2057F0812D8
:08C11200C1FEE4900000F022E0
:1085E9000D0A53454620476D62482020203534380E
:1085F9002E30340A0A0D000A0D000A0A0D00F8434C
:108609000D0A000D0A0020636D2F6D696E0A0D00B9
:108619003B2020003B20003B20202020000A202571
:1086290032642C253032643B00202535643B2025FB
:1086390035643B202535643B202535643B202535B1
:10864900643B2025733B000A0D53454620476D6264
:10865900482020203534382E30340A0A0D002020D5
:1086690020202000202020000A0D2020202020206A
:1086790020202020202020202020202020202020F1
:108689002020002020202020202020202020202001
:10869900000A202573000A53454620476D62482089
:1086A90020203534382E30340A000A25732020253D
:1086B9006264000A2573202025730A000A2535649F
:1086C9003B2025356275000D090900203534382E07
:1086D9003034200A0A0D000A0A0A0D00545B0043CF
:1086E9005D0A0D001B2A74373552001B2A7031357B
:1086F90030581B2A723141001B2A62343657001B3D
:108709002A726243000A0D2020202030000920200F
:1087190020000A0D0909090909092020742F5B7332
:1087290065635D0A000D0A090900203534382E30C9
:1087390034200A0D000A0D545B0009202030002066
:108749002020202020000A0D090909090909090921
:108759002020742F5B7365635D0A0D000A0A0A0005
:108769002020202020202020202020202020202000
:09877900202020202020202000F7
:058C2F00903939EFF05F
:108C34007014783A7C397D017B017A3679BDFE7FE8
:108C4400111230068017903939E0FF7B017A3979A7
:108C54003A90394FE4F0A37411F012BD747F0A12F4
:108C6400AF639003F8E025E02402F582E43429F5AB
:108C740083E493FE740193CAEECAF97BFF12BB1618
:108C84007BFF7A8579E912BB169003F8E025E0248E
:108C940012F582E43429F583E493FE740193CAEE59
:108CA400CAF97BFF12BB1690393AE0FF3395E0FE18
:108CB4007D027C0012A6077BFF7A86790012BB1620
:108CC4009003F8E025E02422F582E43429F583E4D6
:108CD40093FE740193CAEECAF97BFF12BB167B01A3
:108CE4007A39793B12BB167BFF7A86790312BB165D
:108CF4009003F8E025E02432F582E43429F583E496
:108D040093FE740193CAEECAF97BFF12BB16903925
:108D140046E0FEA3E0FF7D037C0012A6077BFF7AFA
:108D240086790712BB169003F8E025E02452F582F9
:108D3400E43429F583E493FE740193CAEECAF97B03
:108D4400FF12BB16903944E0FEA3E0FF7D037C00D4
:108D540012A6077BFF7A86790C12BB169003F8E003
:108D640025E02472F582E43429F583E493FE74014A
:108D740093CAEECAF97BFF12BB16903948E0FEA3F2
:108D8400E0FF7D037C0012A6077BFF7A86790F1231
:028D9400BB160C
:018D960022BA
:1082B20012B81612B5BA7BFF7A86791912BB1690DC
:1082C20036C9E0FEA3E0FF7D057C0012A6077BFF16
:1082D2007A86791D12BB169000B1E0FEA3E0FF7C06
:1082E200007D0A12310D7D057C0012A6077BFF7A04
:1082F20086792012BB169036C7E0FEA3E0FF7D050B
:108302007C0012A6077BFF7A86792012BB16903674
:10831200CBE0FEA3E0FF7D057C0012A6077BFF7A7F
:1083220086791D12BB169000B8E0FEA3E0FF7D0522
:108332007C0012A6077BFF7A86791912BB1690037E
:10834200F8E075F00CA4248CF582E43438F583C08F
:1083520083C082900000E0FF3395E0FED082D0839C
:1083620075F003EF123375EE75F003A42583F583E0
:10837200E0FBA3E0FAA3E0F912BB167BFF7A867951
:108382000012BB167BFF7A8679269001EAE0FFA3F2
:10839200E0903993CFF0A3EFF0900152E0FFA3E019
:1083A200903995CFF0A3EFF0123D1A9036C9E0FF55
:1083B200A3E0903993CFF0A3EFF09000B1E0FEA3D9
:1083C200E0FF7C007D0A12310D903995EEF0A3EFAB
:1083D200F09036C7E0FFA3E0903997CFF0A3EFF01B
:1083E2009036CBE0FFA3E0903999CFF0A3EFF09065
:1083F20000B8E0FFA3E090399BCFF0A3EFF0900329
:10840200F8E075F00CA4248CF582E43438F583C0CE
:1084120083C082900000E0FF3395E0FED082D083DB
:1084220075F003EF123375EE75F003A42583F5831F
:10843200E0F9A3E0FAA3E090399DC9F0A3EAF0A322
:0C844200E9F07BFF7A867932123D1A22A5
:107F1C004387107BFF7A86790012BB169003F8E03A
:107F2C0025E02402F582E43429F583E493FE740100
:107F3C0093CAEECAF97BFF12BB167BFF7A86795087
:107F4C0012BB164387109003F8E025E02412F5824B
:107F5C00E43429F583E493FE740193CAEECAF97BE9
:107F6C00FF12BB169036BDE0FF3395E0FE7D027C20
:107F7C000012A6077BFF7A86790012BB169003F8D5
:107F8C00E025E02422F582E43429F583E493FE74A1
:107F9C000193CAEECAF97BFF12BB167B017A3679C4
:107FAC00BE12BB167BFF7A86790312BB169003F8C0
:107FBC00E025E024E2F582E43428F583E493FE74B2
:107FCC000193CAEECAF97BFF12BB167F2012AF6376
:107FDC004387109003F8E025E024D2F582E434289E
:107FEC00F583E493FE740193CAEECAF97BFF12BBCE
:107FFC00167BFF7A86796712BB169003F8E025E0B2
:10800C002442F582E43429F583E493FE740193CA87
:10801C00EECAF97BFF12BB169003F8E025E0246250
:10802C00F582E43429F583E493FE740193CAEECA15
:10803C00F97BFF12BB167BFF7A86796D12BB164358
:10804C0087109003F8E025E02472F582E43429F5DA
:10805C0083E493FE740193CAEECAF97BFF12BB163C
:10806C007BFF7A86797112BB169003F8E025E02429
:10807C0082F582E43429F583E493FE740193CAEE0D
:10808C00CAF97BFF12BB169003F8E025E02492F5A9
:10809C0082E43429F583E493FE740193CAEECAF9A1
:1080AC007BFF12BB167BFF7A86798C12BB16900372
:1080BC00F8E025E02482F582E43429F583E493FE8C
:1080CC00740193CAEECAF97BFF12BB169003F8E059
:1080DC0025E02492F582E43429F583E493FE7401BF
:1080EC0093CAEECAF97BFF12BB167BFF7A86790323
:0780FC0012BB16438710229E
:059F0A00903932EFF078
:109F0F004387109003F8E025E024A2F582E434297A
:109F1F00F583E493FE740193CAEECAF990399374F2
:109F2F00FFF0A3EAF0A3E9F07BFF7A86799A123D5E
:109F3F001A7BFF7A86799F123D1A4387109003F898
:109F4F00E025E024B2F582E43429F583E493FE742E
:109F5F000193CAEECAF990399374FFF0A3EAF0A304
:109F6F00E9F0903932E0903996F07BFF7A8679B339
:109F7F00123D1A9003F8E025E024C2F582E434295B
:109F8F00F583E493FE740193CAEECAF99039937482
:109F9F00FFF0A3EAF0A3E9F0A37401F0A37402F0B9
:109FAF00A3742FF07BFF7A8679BC123D1A90393358
:109FBF00E4F0A304F090023AE0FEA3E0FF903933FF
:109FCF00E0FCA3E0FDD39FEC9E50407BFF7A8679A7
:109FDF00C590023CE0FF7E001230A6903993EEF060
:109FEF00A3EFF0903934E0243EF582E43402F58398
:109FFF00E0903995F0123D1A438710903934E00400
:0BA00F00F07006903933E004F080AAE6
:01A01A002223
:10C02700E4FFFE438710E4FDFC9003F975F024EF6D
:10C03700123375EE75F024A42583F583E5822DF57B
:10C0470082E5833CF583E4F00DBD00010CED64242B
:0EC057004C70D60FBF00010EBE01C8BF69C5F8
:01C0650022B8
:109BBB00E4903932F0A3F0903932E0FEA3E0FFEEEF
:109BCB003395E0FDFCE47B187A01F9F8C3123311ED
:109BDB004057438710903932E0FEA3E0FFEE3395F8
:109BEB00E0FDFCE47BFB1AF81231E6E47B187A010A
:109BFB00F9F812BFE3CDEFCDCCEECCECC0E0EDC06D
:109C0B00E090393AECF0A3EDF0D0E0FDD0E0FC7B36
:109C1B00687A01E4FFFE126CF2903933E02428F0ED
:109C2B00903932E03400F0808E438710E490393263
:109C3B00F0A3F0FFFE903932E0FCA3E0FD9003F9B6
:109C4B0075F024EF123375EE75F024A42583F5839C
:109C5B00E5822DF582E5833CF5837401F00FBF009F
:109C6B00010EBE01D0BF69CD438710E4FEFFC3EFE9
:109C7B009469EE648094815055438710E490393297
:109C8B00F0A3F0903932E0FCA3E0FDC39424EC6424
:109C9B0080948050309003F975F024EF123375EEF9
:109CAB0075F024A42583F583E5822DF582E5833CAD
:109CBB00F583747FF0903933E004F07006903932FD
:0E9CCB00E004F080BE743C2FFFE43EFE80A05B
:019CD9002268
:0EB19100CBEDCBCAECCA903944EEF0A3EFF040
:10B19F00C3EE64809480500302B246D3E09468906B
:10B1AF003944E064809481400302B246C3EA64806C
:10B1BF009480500302B246D3EB94FBEA64809480F0
:10B1CF0050757C007D07CFEBCFCEEACE12310D90BC
:10B1DF003946EEF0A3EFF0CEEACECFEBCF7C007D79
:10B1EF000712310DCFEDCF7401C8EFC8088002C32D
:10B1FF0033D8FC903948F0903946E0FEA3E0FF9039
:10B20F003944E0FCA3E09003F975F024123375EC98
:10B21F0075F024A42583F583E5822FF582E5833E1F
:10B22F00F583C083C082E0FF903948E0FEEF4ED037
:07B23F0082D083F043871069
:01B2460022E5
:106CF200903934EEF0A3EFF0A3ECF0A3EDF0A3EAA9
:046D0200F0A3EBF01F
:106D0600903934E0FEA3E0FFC3EB9FFFEA9E903983
:106D16003CF0A3EFF0903936E0FEA3E0FFC39039D4
:106D26003BE09FFF90393AE09EFE90393EF0A3EF9C
:106D3600F012C287EEC0E0EFC0E090393CE0FEA35F
:106D4600E0FF12C287D0E0FDD0E0FCD3EF9DEC64FB
:106D560080F8EE6480985003026E83903934E0FE2A
:106D6600A3E0FF903939E09FEE6480F8903938E06F
:106D76006480985068903940EEF0A3EFF090393671
:106D8600E0FCA3E0FD903942ECF0A3EDF090393839
:106D9600E0FBA3E0903934CBF0A3EBF090393AE076
:106DA600FBA3E0903936CBF0A3EBF0A3EEF0A3EF14
:106DB600F0A3ECF0A3EDF0A3E0FEA3E0FFC3E49F95
:106DC600FFE49E90393CF0A3EFF0A3E0FEA3E0FFC2
:106DD600C3E49FFFE49E90393EF0A3EFF0E49039C0
:106DE60040F0A3F090393CE0FEA3E0FF903940E08C
:106DF600FCA3E0FDD39FEE6480F8EC64809840032A
:106E0600026F78903935E02DFF903934E03CFEEE84
:106E1600C0E0EFC0E090393EE0FEA3E0FFFBCAEE23
:106E2600CAEA3395E0F9F8A3E0FEA3E0FFEE339556
:106E3600E0FDFC1231E6EEC0E0EFC0E090393CE048
:106E4600FEA3E0FFFBCAEECAEA3395E0F9F8D0E00C
:106E5600FFD0E0FE12BFE3903937E02FFD903936C0
:106E6600E03EFCD0E0FFD0E0FE12B191903941E067
:106E760004F07006903940E004F0026DEA9039366D
:106E8600E0FEA3E0FFC390393BE09FEE6480F890FC
:106E9600393AE06480985070903934E0FEA3E0FF00
:106EA600903940EEF0A3EFF0903936E0FCA3E0FD18
:106EB600903942ECF0A3EDF0903938E0FBA3E09076
:106EC6003934CBF0A3EBF090393AE0FBA3E09039EC
:106ED60036CBF0A3EBF0A3EEF0A3EFF0A3ECF0A318
:106EE600EDF0A3E0FEA3E0FFC3E49FFFE49E90392C
:106EF6003CF0A3EFF0A3E0FEA3E0FFC3E49FFFE4B2
:106F06009E90393EF0A3EFF0E4903942F0A3F09062
:106F1600393EE0FAA3E0FB903942E0FCA3E0FDD362
:106F26009BEA6480F8EC648098504790393CE0FE18
:106F3600A3E0FF1230A6CDEBCDCCEACC12310D90FA
:106F46003935E02FFF903934E03EFE903942E0FCBF
:106F5600A3E0FD903937E02DFD903936E03CFC1278
:106F6600B191903943E004F07006903942E004F0A4
:026F7600809DFC
:016F780022F6
:10A9BE00E4903932F0A3F090023AE0FEA3E0FF906B
:10A9CE003932E0FCA3E0FDC39FEC9E400302AA9E39
:10A9DE00438710ED25E0FFEC33FEEEC0E0EFC0E064
:10A9EE00E0243EF582E43402F583E0FFE4EF24191F
:10A9FE00FFE433FEE433FDE433FCE47BFBFAF9F8C9
:10AA0E001231E6E47B187A01F9F812BFE3CDEFCDEF
:10AA1E00CCEECCECC0E0EDC0E0903933E02401FF89
:10AA2E00903932E03400FEEF25E0FBEE33FAEAC057
:10AA3E00E0EBC0E0A3E0243FF582E43402F583E0CE
:10AA4E00FFE4EF2419FFE433FEE433FDE433FCE4CA
:10AA5E007BFBFAF9F81231E6E47B187A01F9F81269
:10AA6E00BFE390393AEEF0A3EFF0D0E0FBD0E0FA7E
:10AA7E00D0E0FDD0E0FCD0E0FFD0E0FE126CF29012
:10AA8E003933E004F07006903932E004F002A9C5C3
:01AA9E002295
:1051F0007BFF7A8679D012BB169003F8E025E02475
:10520000A2F582E43429F583E493FE740193CAEE97
:10521000CAF97BFF12BB167BFF7A8679D412BB16C4
:105220004387109003F8E025E024E2F582E4342877
:10523000F583E493FE740193CAEECAF97BFF12BBB7
:105240001612B8167BFF7A86790012BB169003F807
:10525000E025E024D2F582E43428F583E493FE745B
:105260000193CAEECAF97BFF12BB1643871012B531
:10527000BA7BFF7A86790012BB169003F8E025E02E
:1052800024B2F582E43429F583E493FE740193CAD1
:10529000EECAF97BFF12BB1690022EE0FF3395E0B9
:1052A000FE7D017C0012A6077BFF7A86790012BB87
:1052B000164387109003F8E025E024C2F582E43419
:1052C00029F583E493FE740193CAEECAF97BFF12B9
:1052D000BB1690022EE0701F9003F8E075F003A457
:1052E00024ECF582E5F03438F583E0FBA3E0FAA383
:1052F000E0F912BB1680097B017A02792F12BB16E6
:105300007BFF7A8679E012BB164387107BFF7A8693
:1053100079E512BB167FF812AF637BFF7A8679E8D6
:1053200012BB164387107BFF7A8679ED12BB16906D
:105330003932E4F0A374FBF043871012AA9F90392E
:1053400032E0FEA3E0FFEE3395E0FDFCE47B187A4B
:1053500001F9F81231E6E47BFBFAF9F812BFE3E455
:105360007B28FAF9F812BFE3CCE8CCCDE9CDCEEA40
:10537000CECFEBCFE4FBFAF9F8C3123311703B90B8
:105380003932E0FEA3E0FFEE3395E0FDFCE47B184C
:105390000AF81231E6E47BFBFAF9F812BFE3903920
:1053A0003AEEF0A3EFF07F0D12AF6390393AE0FED2
:1053B000A3E0FF7D047C0012A6077BFF7A8679F4C8
:1053C00012BB167BFF7A87790112BB16E490393441
:1053D000F0A3F0C3903935E09470903934E06480E4
:1053E000948140030254E0438710E490393CF090EC
:1053F0003936F0A3F043871090393CE0FBEBC0E076
:10540000903932E0FEA3E0FF7C007D0712310D9061
:105410003936E0FCA3E0FD903935E02DFD903934BC
:10542000E03CFC9003F975F024ED123375EC75F057
:1054300024A42583F583E5822FF582E5833EF58359
:10544000E0FB3395E0FA903932E0FEA3E0FF7C0008
:105450007D0712310D74017E00C8EDC8088005C3B8
:1054600033CE33CED8F9FFEE5AFEEF5B4E60047FA9
:105470000180027F00903937E0FEC374079EFEEF83
:10548000C8EEC8088002C333D8FCFFD0E04F903983
:105490003CF0903937E004F07006903936E004F0C3
:1054A000903936E07004A3E0640860030253F5C34A
:1054B000903935E09468903934E0648094814007F5
:1054C00090393CE05480F090393CE0FF12AF63909B
:1054D0003935E02408F0903934E03400F00253D339
:1054E0007BFF7A87790812BB1612B2FCEF7003EECD
:1054F00064087006903936F0A3F0903933E024FF49
:10550000F0903932E034FFF0C3E0648094804003CF
:105510000253387BFF7A87790E12BB16900238E06F
:10552000FEA3E0FF7C007D061230B8903938EEF023
:10553000A3EFF0903936E4F0A304F04387107BFF2B
:105540007A87791612BB16903936E0FCA3E0FDA3EA
:10555000E0FEA3E0FF1230A67D047C0012A60790B7
:105560003937E004F07006903936E004F0C3903922
:1055700037E09407903936E06480948040BD7BFF2B
:105580007A87791B12BB167BFF7A87790812BB16C4
:0155900022F8
:08BA2B00903936EEF0A3EFF0B4
:10BA33007F1B12AF637F4B12AF637F6912AF634308
:10BA430087107F0112AF63E4903938F0A3F0903987
:10BA530038E0FEA3E0FFC39469EE64809481503D17
:10BA6300438710903936E0FCA3E0FD9003F975F0AD
:10BA730024EF123375EE75F024A42583F583E58254
:10BA83002DF582E5833CF583E0FF12AF63903939EE
:0DBA9300E004F07006903938E004F080B156
:01BAA0002283
:105C34007F1B12AF637F2112AF63E4FF12AF634394
:105C440087107BFF7A87792E12BB169003F8E02524
:105C5400E024A2F582E43429F583E493FE740193ED
:105C6400CAEECAF97BFF12BB167BFF7A877933121F
:105C7400BB164387109003F8E025E024E2F582E4A4
:105C84003428F583E493FE740193CAEECAF97BFFCA
:105C940012BB167F2012AF6312B8167BFF7A867987
:105CA4000012BB169003F8E025E024D2F582E43418
:105CB40028F583E493FE740193CAEECAF97BFF12BC
:105CC400BB167F2012AF6343871012B5BA7BFF7AED
:105CD40086790012BB169003F8E025E024B2F58221
:105CE400E43429F583E493FE740193CAEECAF97B84
:105CF400FF12BB1690022EE0FF3395E0FE7D017C7F
:105D04000012A6077BFF7A86790012BB1643871020
:105D14009003F8E025E024C2F582E43429F583E415
:105D240093FE740193CAEECAF97BFF12BB1690026C
:105D34002EE0701F9003F8E075F003A424ECF582C4
:105D4400E5F03438F583E0FBA3E0FAA3E0F912BBF5
:105D54001680097B017A02792F12BB167BFF7A86A3
:105D6400790012BB167F1B12AF637F3312AF637FC0
:105D74001512AF634387107BFF7A87793E12BB16F7
:105D84007FF812AF637BFF7A8679E812BB164387EC
:105D940010903932E4F0A37424F0903932E0FEA379
:105DA400E0FFD39400EE648094805003025E7A4353
:105DB4008710EE3395E0FDFCE47BA87A07F9F8122E
:105DC40031E6E47BFCFAF9F812BFE3903934EEF0E3
:105DD400A3EFF012AA9F903934E0FEA3E0FFEE3364
:105DE40095E0FDFCE47B28FAF9F812BFE3CCE8CC9B
:105DF400CDE9CDCEEACECFEBCFE47B08FAF9F8D3E8
:105E0400123311402C903934E0FEA3E0FFEE3395B9
:105E1400E0FDFCE47B28F812BFE3E47B28FAF9F800
:105E24001231E67D047C0012A6077F0912AF63805D
:105E3400057F0912AF63903933E024FFFF903932B4
:105E4400E034FFFE12BA2B7F0D12AF637F0A12AF4C
:105E54006343871012B2FCEF7003EE64087006907F
:105E64003932F0A3F0903933E024FFF0903932E076
:105E740034FFF0025D9E7F0A12AF637F1B12AF6393
:105E84007F3312AF634387107F2412AF637BFF7AA3
:105E940087794312BB16900238E0FEA3E0FF7C0032
:105EA4007D061230B8903934EEF0A3EFF04387103A
:105EB400903932E4F0A304F04387107BFF7A8779AA
:105EC4004812BB16903932E0FCA3E0FDA3E0FEA328
:105ED400E0FF1230A67D047C0012A607903933E05F
:105EE40004F07006903932E004F0C3903933E09442
:105EF40007903932E06480948040BD7BFF7A8779D3
:105F04004F12BB167F1B12AF637F4012AF634387F0
:0A5F1400107BFF7A87796512BB1637
:015F1E002260
:10C2450012C027129BBB12A9BE900226E0600714FC
:0AC255007007125C34221251F0222F
:10B462007D027C007F0A7E0012B8A19039E5E0B42B
:10B47200011E9003F8E025E024D6F582E43429F594
:10B4820083E493FE740193CAEECAF97BFF12C18171
:10B492007D027C007F0A7E0012B8A19039E6E0B4FA
:10B4A200011E9003F8E025E024F6F582E43429F544
:10B4B20083E493FE740193CAEECAF97BFF12C18141
:10B4C2007D027C007F0A7E0012B8A19039E4E0B4CC
:10B4D200011E9003F8E025E024E6F582E43429F524
:10B4E20083E493FE740193CAEECAF97BFF12C18111
:10B4F2009039E4E070159039E5E0700F9039E6E09C
:0CB5020070097BFF7A87796912C18122F1
:10B5BA009039747402F0A3F0A3F07B017A3979D040
:10B5CA00128918438710C39039D7E0940A9039D664
:10B5DA00E09400500B7F3012AF639039747401F01D
:10B5EA009039D6E0FEA3E0FF903974E0FD7C0012AA
:10B5FA00A6077F3A12AF63C39039D9E0940A90390B
:10B60A00D8E09400500B7F3012AF63903975740103
:10B61A00F09039D8E0FEA3E0FF903975E0FD7C0098
:10B62A0012A6077F3A12AF63C39039DBE0940A90FF
:10B63A0039DAE09400500B7F3012AF639039767498
:10B64A0001F09039DAE0FEA3E0FF903976E0FD7C64
:04B65A000012A6072D
:01B65E0022C9
:10B816009039747402F0A3F07B017A3979D01289D9
:10B8260018438710C39039D5E0940A9039D4E09430
:10B8360000500B7F3012AF639039747401F0903969
:10B84600D4E0FEA3E0FF903974E0FD7C0012A60769
:10B856007F2E12AF63C39039D3E0940A9039D2E0B9
:10B866009400500B7F3012AF639039757401F090DD
:10B8760039D2E0FEA3E0FF903975E0FD7C0012A608
:10B88600077F2E12AF639039D0E0FEA3E0FF7D0460
:0AB896007C0012A6077F2012AF63AA
:01B8A0002285
:107479004239C300004239C500004139C7004139CA
:07748900C8004239CC0000ED
:03005B0002593017
:0D593000C0E0C0F0C083C082C0D075D018A8
:10593D0020160A900153E09039C2F0D21674242536
:10594D00C9F5C975C800900229E004F090022CE059
:10595D0004F090022DE004F0C39039C4E094E89077
:10596D0039C3E09403500EA3E004F070069039C3E0
:10597D00E004F0801B900005744EF0A37420F090AD
:10598D0000B3E04410F09039C37403F0A37420F019
:10599D00C39039C6E094E89039C5E09403500EA346
:1059AD00E004F070069039C5E004F0801B90000310
:1059BD00744EF0A37420F09000B3E04410F09039D1
:1059CD00C57403F0A37420F09001F4E0FCA3E0FD96
:1059DD00A3E0FEA3E0FFE4FAF9F8EF2401FFEA3EAD
:1059ED00FEE93DFDE83CFC9001F4123338900229AC
:1059FD00E0C3946440279036D0E004F070069036F2
:105A0D00CFE004F0900229E4F030100B9001F3E0A8
:105A1D00600BE014F080069001F3740FF0900229F2
:105A2D00E0B4210590022CE4F0900229E0B4420587
:105A3D0090022DE4F0900229E075F00A84E5F070F3
:105A4D00139039C0E0FF900229E06F60079000B31A
:105A5D00E04401F09036D0E020E0179039C1E0FF2E
:105A6D009036CFE07003A3E06F60079000B3E04481
:105A7D0004F0900152E0FEA3E0FF7C007D051230A2
:105A8D00B8ED4C701F9039C2E0FF900152E07003E9
:105A9D00A3E06F600F9000B3E04440F0900153E03D
:105AAD009039C2F07F107EC08F828E83E030E70385
:105ABD00D38001C39200A200E433FF9036DEE06F85
:105ACD00605C9039C7E004F0E0D394034055740353
:105ADD00F09036DEEFF09001F3740FF030001D9072
:105AED0039C5E0FFA3E0900003CFF0A3EFF09039AC
:105AFD00C5E4F0A3F09000B3E04410F02000249032
:105B0D0039C3E0FFA3E0900005CFF0A3EFF090398B
:105B1D00C3E4F0A3F09000B3E04410F08005903999
:105B2D00C7E4F0900229E0FF9039C0E06F60089063
:105B3D000229E09039C0F09039C1E0FF9036CFE0F6
:105B4D007003A3E06F7003025BDAC39036D0E0946C
:105B5D003C9036CFE09400404BE4F0A3F09001531D
:105B6D00E004F07006900152E004F09001FCE0FEBC
:105B7D00A3E0FFD39400EE940040299000B6E0041A
:105B8D00F070069000B5E004F0C39000B6E09F9071
:105B9D0000B5E09E400E9000B3E04480F09000B55B
:105BAD00E4F0A3F0C3900153E0943C900152E094D3
:105BBD00004012E4F0A3F09001EBE004F0700690C9
:105BCD0001EAE004F09036D0E09039C1F090020483
:105BDD00E0FFB40111900009E0FE900229E0C39EA0
:105BED005004C2C28002D2C2EFB4011190000AE08B
:105BFD00FF90022CE0C39F5004C2C38002D2C39019
:105C0D000204E0B4011190000BE0FF90022DE0C3FF
:0C5C1D009F5004C2C18002D2C175FF007C
:0B5C2900D0D0D082D083D0F0D0E03289
:03000B0002C11A15
:10C11A00C0E0C083C082C0D075D0109001FBE0247B
:10C12A000AF0E0C394644002E4F090021DE0FF903C
:10C13A0001FBE0C39F5004C2928002D292D0D0D0B9
:06C14A0082D083D0E03238
:10AA9F004387109000B3E030E0031299799000B330
:10AAAF00E030E208125F1F900000EFF09000B3E07B
:10AABF0030E4139036CBE0FEA3E0FF127B1C900036
:10AACF00B8EEF0A3EFF09000B3E030E63D90021740
:10AADF00E0FCA3E0FDA3E0FEA3E0FFE4FAF9F8EF4A
:10AAEF002401FFEA3EFEE93DFDE83CFC900217120F
:10AAFF003338900217E0FCA3E0FDA3E0FEA3E0FFD4
:10AB0F0012BF9F9000B3E054BFF09000B3E030E766
:10AB1F0010900203E070031282B29000B3E0547FF2
:10AB2F00F07F4012C299500E9039C8E0C3940A507A
:10AB3F000AE004F08005E49039C8F09039C8E0C30A
:10AB4F00940A4013C2C690000074FFF0E490020410
:10AB5F00F090022004F022201402D2C6900220E0CE
:0EAB6F00B4010B9000B77401F0E4900220F0E6
:01AB7D0022B5
:05B50E00903974EFF01C
:10B5130012BD1ACCEECCCDEFCDE4122CCA7BA07AAF
:10B523001679BC7845122B0EE4FBFA797A7844122B
:10B533002C17122D03903975EEF0A3EFF0903974A8
:10B54300E0FF12BD1ACCEECCCDEFCDE4122CCA7BBA
:10B553004E7A1279127844122B0EECC0E0EDC0E063
:10B56300EEC0E0EFC0E0903974E0FF12BD1ACCEEFC
:10B57300CCCDEFCDE4122CCAD0E0FBD0E0FAD0E082
:10B58300F9D0E0F8122B0E7B2A7A5079FE784B1211
:10B593002C17122CB4122D03903976E02FFF90391B
:10B5A30075E03EFE9036D3E02FFF9036D2E03ECFDB
:06B5B30024FDCF34FFFE71
:01B5B900226F
:109979009039C9E0146077147003029A29147003AE
:10998900029A5D24036003029A8E7F0712BD1ACCE6
:10999900EECCCDEFCDE4122CCA7B687AB3791A7874
:1099A90040122B0EECC0E0EDC0E0EEC0E0EFC0E0ED
:1099B9009036D3E025E0FD9036D2E033FCE4122C5A
:1099C900CAD0E0FBD0E0FAD0E0F9D0E0F8122A1DC5
:1099D900E4FBFA79407840122C17122D039036D205
:1099E900EEF0A3EFF09039C97401F0029A93E4FF05
:1099F90012B50ECCEECCCDEFCD900008E025E0FFFE
:109A0900900007E033FEED2FFFEC3EFE7C007D0366
:109A19001230B8EEF0A3EFF09039C97402F0806A01
:109A2900E4FF12B50ECAEECACBEFCB9000B1E0FE4F
:109A3900A3E0FF7C007D091230A6EB2FFFEA3EFE72
:109A49000D1230B89000B1EEF0A3EFF09039C9745F
:109A590003F080367F0312B50ECCEECCCDEFCD905E
:109A69000201E025E0FF900200E033FEED2FFFEC5C
:109A79003EFE7C007D031230B8EEF0A3EFF0E490D7
:109A890039C9F08005E49039C9F09000B3E054FE7B
:019A9900F0DC
:019A9A0022A9
:105F1F00903974E4F0A304F09036C9E0FEA3E0FFDB
:105F2F007C007D0A1230A6900002E02FFF90000146
:105F3F00E03EFE900007E0FCA3E0FDC3EF9DFFEE07
:105F4F009CFE903976F0A3EFF07C007D0A12310DA4
:105F5F00CCEECCCDEFCDD3ED9400EC6480948040AB
:105F6F001E903975E025E0FF903974E033FE74051B
:105F7F002FF58274023EF583E475F001123143C3AD
:105F8F00EC64809480501E903975E025E0FF9039C5
:105F9F0074E033FE74052FF58274023EF58374FFAF
:105FAF00F5F0123143900212E0FCA3E0FD7E037F77
:105FBF00E812310DCCEECCCDEFCD903975E025E068
:105FCF00FB903974E033FA74052BF58274023AF5BD
:105FDF0083E0FEA3E0D39DEC6480F8EE64809840EC
:105FEF001E900212E0FCA3E0FD7E037FE812310D4C
:105FFF0074052BF58274023AF583EEF0A3EFF0905F
:10600F003975E025E0FF903974E033FE74052FF504
:10601F008274023EF583E0FCA3E0C3EC64809480BD
:10602F00500E74052FF58274023EF583E4F0A3F051
:10603F00903976E0FCA3E0FD903975E025E0FF9004
:10604F003974E033FE740E2FF58274023EF583EC43
:10605F00F0A3EDF0900007E0FCA3E0FDC39039CB77
:10606F00E09DFD9039CAE09CFC74ED2FF582740120
:10607F003EF583ECF0A3EDF0903975E025E0FF904D
:10608F003974E033FE740E2FF58274023EF583E00F
:10609F00FCA3E0FD90021BE0FEA3E0FF1230A67C04
:1060AF00007D0A12310DCAEECACBEFCB903975E0E5
:1060BF0025E0FF903974E033FE74052FF5827402EA
:1060CF003EF583E0FCA3E0FD900212E0FEA3E0FFAB
:1060DF001230A67C007D0A12310DEF2BFBEE3AFA3F
:1060EF00903975E025E0FF903974E033FE74ED2FA1
:1060FF00F58274013EF583E0FCA3E0FD90020AE017
:10610F00FEA3E0FF1230A67C007D0A12310DEF2BAB
:10611F00FFEE3AFED3EF9400EE648094805003E4D8
:10612F00FEFFD3EF9464EE6480948040047E007F82
:10613F0064900009EFF090000AF09036C7E0FEA3DC
:10614F00E0FF7C007D641230A67D051230B8900010
:10615F000BEFF0900007E0FFA3E09039CACFF0A358
:10616F00EFF09000B3E054FBF0900000E0FEC3644A
:10617F008094805003026205900204E07002FF22B7
:10618F00903976E0FCA3E0FDD39432EC64809480E8
:10619F005033C3ED94CEEC6480947F402890021569
:1061AF00E004F07006900214E004F0C3900215E0D2
:1061BF009428900214E064809480403AE4F0A37431
:1061CF0028F07F0122900215E024FFF0900214E0E6
:1061DF0034FFF0E0FCA3E0FDC39414EC64809480E2
:1061EF005014ED9400EC648094805007E4900214F6
:0961FF00F0A3F07F0022CFEECFE7
:016208002273
:087B1C00903974EEF0A3EFF0C4
:107B24009039CCE06E7003A3E06F6016E49001FE20
:107B3400F0A3F0903974E0FFA3E09039CCCFF0A328
:107B4400EFF09000B3E020E403027CE0900003E057
:107B5400FEA3E0FF900006E02FFF900005E03EFE4C
:107B6400CBEFCBFAE4F9F87F207E4B7D0DFC12BFFE
:107B7400E3EF2432FFE43EFEE43DFDE43CFCE47B21
:107B84000AFAF9F812BFE3903976EEF0A3EFF09019
:107B940000B8E0FEA3E0FF7C007D141230A690390B
:107BA40077E02FFF903976E03EFE7D0312310DEE33
:107BB400F0A3EFF0903974E0FAA3E0FB900221E027
:107BC400FEA3E0FFCDEBCDCCEACC1230A67C007D49
:107BD400641230B890022BE02FFF90022AE03E900E
:107BE40039CEF0A3EFF07E007F0ACDEBCDCCEACC0A
:107BF4001230A6903974EEF0A3EFF0A3E0FEA3E0F8
:107C0400FFC3903975E09FFF903974E09EFE903970
:107C140078F0A3EFF012C2877C007D1412310DEFCF
:107C24002401FFE43EFED3EF9405EE64809480408B
:107C3400047E007F05C3903979E094FB903978E0A5
:107C44006480947F502B9001FEE0FCA3E0FD90390A
:107C5400CFE02DFD9039CEE03CFCD3ED9400EC64F4
:107C6400809480400C9001FFE09FF09001FEE09E24
:107C7400F0D3903979E09405903978E06480948069
:107C8400402B9001FEE0FCA3E0FD9039CFE02DFDF8
:107C94009039CEE03CFCC3ED94FFEC6480948050BA
:107CA4000C9001FFE02FF09001FEE03EF0D3900134
:107CB400FFE0943C9001FEE0648094804006E4F090
:107CC400A3743CF0C39001FFE094C49001FEE0640F
:107CD40080947F500774FFF0A374C4F09001FEE019
:107CE400FEA3E0FF9039CFE02FFF9039CEE03EFEB7
:107CF400C3EF94FFEE6480948040047E007FFFD342
:107D0400EF9400EE648094805003E4FEFF8FFC90B7
:107D140000B3E054EFF0903976E0FEA3E0FF7C007E
:057D24007D0A12310D83
:017D29002237
:101611005568727A6569743A200054696D652020B5
:1016210020203A200048657572652020203A20006C
:101631005A656761722020203A2000446174756DFB
:1016410020203A200044617465202020203A2000A7
:1016510044617461202020203A2000454348545AB7
:10166100454954554852202020005245414C544987
:101671004D45434C4F434B200054454D5053205250
:1016810045454C20005A45474152006465757473C5
:1016910063682020006765726D616E202020006103
:1016A1006C6C656D616E6420006E69656D69656362
:1016B1006B69002020352031202020200020203699
:1016C1002031202020200020203720312020202000
:1016D1000020203820312020202000656E676C69B1
:1016E1007363682000656E676C6973682020006110
:1016F1006E676C616973202000616E6769656C7348
:101701006B69002020352032202020200020203647
:1017110020322020202000202037203220202020AD
:1017210000202038203220202020006672616E7A4D
:101731002E202020006672656E63682020200066DE
:1017410072616E6361697320006672616E637573A5
:101751006B690020203520332020202000202036F6
:10176100203320202020002020372033202020205B
:101771000020203820332020202000706F6C6E69FB
:101781007363682000706F6C69736820202000709B
:101791006F6C6F6E6169732000706F6C736B692081
:1017A1002020002020352034202020200020203639
:1017B1002034202020200020203720342020202009
:1017C1000020203820342020202000202031203506
:1017D1002020202000202032203520202020002021
:1017E10020332035202020200020203420352020C7
:1017F10020200020203520352020202000202036E8
:1018010020352020202000202037203520202020B6
:1018110000202038203520202020002020312036B3
:1018210020202020002020322036202020200020CF
:101831002033203620202020002020342036202074
:101841002020002020352036202020200020203696
:101851002036202020200020203720362020202064
:101861000020203820362020202000202031203761
:10187100202020200020203220372020202000207E
:101881002033203720202020002020342037202022
:101891002020002020352037202020200020203645
:1018A1002037202020200020203720372020202012
:1018B100002020382037202020200020203120380F
:1018C100202020200020203220382020202000202D
:1018D10020332038202020200020203420382020D0
:1018E10020200020203520382020202000202036F4
:1018F10020382020202000202037203820202020C0
:10190100002020382038202020200067656C616489
:10191100656E006C6F616465640063686172678203
:10192100007A616C61646F77616E6F000067656C4E
:101931006F65736368740064656C657465640073D6
:1019410075707072696D82006B61736F77616E691A
:1019510065006765737065696368657274007361BA
:1019610076656400656E7265676973746572007A85
:101971006170616D696574616E6F00414B545545CD
:101981004C4C200043555252454E54200041435483
:1019910055414C00414B5455414C4E494500205353
:1019A10050524143484520004C414E47554147451F
:1019B10020004C414E4755450020204A455A594B7D
:1019C100006C65657200656D707479007669646597
:1019D10000776F6C6E65004E494348542042455272
:1019E1004549542000202020424552454954202099
:1019F1002000204D414E2E204245524549542000A1
:101A01004D414E2E4E2E4245524549540020204E06
:101A11004F54205245414459202000202020524556
:101A21004144592020202000204D414E2E20524576
:101A31004144592020004D414E2E4E2E52454144E5
:101A4100592000202070617320707288742020203A
:101A51000020202020707288742020202000202067
:101A610070728874206D616E2E2020006E6F6E2062
:101A710070728874206D616E00204E494520474F79
:101A8100544F5759202000202020474F544F575979
:101A910020202000204D414E2E20474F544F5759B2
:101AA10020004D414E2E4E2E474F544F575900485E
:101AB100415542452F4E4F5441555320002020207F
:101AC1004645484C455232202000202020464548BA
:101AD1004C455233202020002020204645484C45CB
:101AE10052342020002020454D455247454E435950
:101AF1002020002020204552524F52203220200029
:101B01002020204552524F522033202020002020F7
:101B1100204552524F522034202000202055524758
:101B2100454E43452020202000202020455252458B
:101B31005552203220002020204552524555522036
:101B41003320200020202045525245555220342078
:101B51000020204552524F52203120202020005099
:101B61004152414D45544552415553445255434BC1
:101B7100200A00504152414D455445525345545459
:101B8100494E4753200A00504152414D4554524558
:101B9100200A00504152414D455452590A00507299
:101BA1006F6772616D6D2D4E722E2020203A2000DC
:101BB10050726F6772616D2D4E6F2E202020203A7A
:101BC100200050726F6772616D6D652D4E6F2E2012
:101BD100203A200050726F6772616D7920202020B9
:101BE1002020203A20004B656E6E7A656963686E2D
:101BF100756E6720203A20004E616D6520202020FF
:101C0100202020202020203A20005369676E616C3B
:101C110069736174696F6E20203A004F7A6E616357
:101C21007A656E696520202020203A20004C756677
:101C31007474656D70657261747572203A2000412B
:101C4100697274656D7065726174757220203A20D5
:101C51000074656D702E20706F77696574727A619A
:101C61003A200054656D706572617475726520412A
:101C710069723A20004C75667474656D702E20206F
:101C8100203A200041697274656D702E2020202059
:101C91003A200054656D702E204169722020203A4F
:101CA100200074656D702E20706F772E20203A20F1
:101CB1000049522D5374656C6C7765727420202035
:101CC1003A200049522D70726573657420202020DE
:101CD10020203A20004952206E617374617761209F
:101CE100202020203A200049522020202020203A84
:101CF100200049522D7072652E203A2000547261E5
:101D01006E73666572202020202020203A20004337
:101D11006F6E7665796F7220202020202020203A76
:101D210020007472616E73706F7274202020202005
:101D3100203A2000536F6C6C203A2000707265735A
:101D41002E3A20006E6173742E3A2000497374207C
:101D5100203A2000637572722E3A20006A6573740E
:101D61003A200054656D706572617475726B75729D
:101D71007665200054656D706572617475726520B9
:101D81004D6561737572656D656E742000436F7585
:101D9100726265206465206D657375726520004B04
:101DA100727A79776520506F6D6961727520004E86
:101DB100722E2020202020203A20004E6F2E20203D
:101DC100202020203A20004B656E6E7A2E202020A4
:101DD1003A20005469746C65202020203A20004E7E
:101DE1006F6D6272652020203A20006F7A6E616308
:101DF1007A656E69653A2000485020202020202015
:101E0100202020004550534F4E202020202020200C
:101E11002000447275636B65726665686C6572005B
:101E21005072696E746572204572726F72004572EC
:101E31007265757220496D7072696D6575720062A7
:101E41006C61642077796472756B75004B65696E9E
:101E510020506170696572202000506170657220A8
:101E61004572726F7220200070617320646520706A
:101E71006170696572006272616B20706170696581
:101E810072750054696D656F7574202020202020C3
:101E91000050617373776F7274202020203A200004
:101EA10050617373776F7264202020203A200035CF
:101EB10034382E303400202020004300204845498A
:101EC1005A2020202020202056203D202020202084
:101ED100636D2F6D696E20205072672E3A202000AD
:101EE1002020506172616D2E20202050726F677228
:101EF100616D6D2020204D657373656E202020205B
:101F010053797374656D2020200020484541542089
:101F110020202020202056203D2020202020636DDD
:101F21002F6D696E20205072672E3A2020002020EC
:101F3100506172616D2E20202050726F6772616D49
:101F41002020204D65617375726520202020537912
:101F51007374656D202020004348415546202020A0
:101F61002020202056203D2020202020636D2F6D31
:101F7100696E20205072672E3A2020002020506187
:101F810072616D2E20202050726F6772616D2E205C
:101F910020204D657375726520202020537973745C
:101FA100656D65202000204F47525A2020202020B7
:101FB100202056203D2020202020636D2F6D696E4A
:101FC10020205072672E3A202000506172616D65A9
:101FD100747279202050726F6772616D79202020B0
:101FE100506F6D6961722020202053797374656D83
:101FF10020202000504152414D45544552004C751E
:10200100667420202020203A20202020202020201B
:1020110020202020202020202020202020202020BF
:102021002020004952203120202020203A20202049
:102031002020202020005472616E73666572203A60
:102041002020202020636D2F6D696E200054656D66
:1020510070657261747572205472616E7366657217
:102061002020202055687220202020447275636B47
:10207100656E200041697274656D702E203A2020D2
:10208100202020202020202020202020202020204F
:10209100202020202020202000436F6E7665796F5C
:1020A10072203A2020202020636D2F6D696E200060
:1020B10054656D7065726174757220436F6E7665DB
:1020C100796F722020436C6F636B202020202020C9
:1020D1005072696E74202000504152414D45545256
:1020E10045004169722020202020203A2020202014
:1020F10020202020202020202020202020202020DF
:10210100202020202020005472616E736665727455
:102111003A2020202020636D2F6D696E2000202041
:1021210054656D702E20202020205472616E732E14
:1021310020202020202020202020202020496D70D8
:1021410072696D657200504152414D4554525900BA
:10215100506F77696574727A653A202020202020BB
:10216100202020202020202020202020202020206E
:102171002020202000202054656D702E202020205A
:102181005472616E73666572202020202020202009
:102191002020202020204472756B2020003E3E200C
:1021A100202020202020202020202020203C3C0016
:1021B10050524F4752414D4D450020204C616465BE
:1021C1006E20202020205370656963682E20204CEA
:1021D10094736368656E202020447275636B656E2D
:1021E1002020200050524F4752414D0020204C6F7B
:1021F100616420202020202020536176652020204A
:102201002044656C65746520202020205072696E21
:1022110074202020200050524F4752414D4D4553CC
:10222100002043686172676572202020456E7265E7
:10223100676973742E5375707072696D65722020B1
:10224100496D7072696D657220200050524F47527E
:10225100414D59004C61646F77616E6965205A6127
:1022610070616D6965742E204B61736F77616E6962
:1022710065202020204472756B20202020004D45D0
:1022810053534B555256454E0020416E7A6569674E
:10229100656E2020205370656963682E2020204DD3
:1022A100657373656E202020447275636B656E20C3
:1022B1002020004D4541535552454D454E54002077
:1022C100446973706C617920202020205361766508
:1022D100202020204D6561737572652020202050DB
:1022E10072696E742020202000434F55524245539D
:1022F100204445204D4553555245002041666669AD
:10230100636865722020456E7265676973742E205B
:10231100204D6573757265722020496D7072696D0B
:1023210065722020004B525A59574520504F4D4954
:1023310041525500577973776965746C2E20205A84
:102341006170616D6965742E2020506F6D696172D5
:1023510020202020204472756B202020200053591A
:102361005354454D45494E5354454C4C554E4745A4
:102371004E0053707261636865202020203A20204E
:102381002020202020202020202020204B6F6E7430
:1023910072617374202B00426574722E2D53746424
:1023A1002E203A20202020202020202020206820BC
:1023B1000050726F746F6B6F6C6C20203A2020207C
:1023C1002020202020206D696E20204B6F6E7472BA
:1023D100617374202D00447275636B65727479703A
:1023E100203A2020202020202020202020202000F2
:1023F1002053707261636865202050726F746F6B37
:102401006F6C6C2020447275636B657220202053C1
:1024110065727669636520200053595354454D53C5
:10242100455454494E4753004C616E677561676569
:102431002020203A20202020202020202020202081
:102441002020436F6E7472617374202B004F70658E
:102451007261742E2D682E203A2020202020202009
:10246100202020206820005265706F727420202087
:1024710020203A2020202020202020206D696E205D
:1024810020436F6E7472617374202D005072696EF7
:10249100746572202020203A202020202020202036
:1024A1002020202020004C616E6775616765202027
:1024B100205265706F7274202020205072696E74F2
:1024C1006572202020536572766963652020005370
:1024D100595354454D45004C616E67756520202068
:1024E10020203A20202020202020202020202020D1
:1024F10020436F6E747261737465202B00436F6D9E
:1025010074657572202020203A2020202020202070
:102511002020202068200050726F746F636F6C65FB
:1025210020203A2020202020202020206D696E20AC
:1025310020436F6E747261737465202D00496D7054
:1025410072696D616E7465203A2020202020202060
:1025510020202020202000204C616E6775652020FE
:102561002050726F746F636F6C6520496D70726972
:102571006D616E74652053657276696365200053E1
:10258100595354454D004A657A796B20202020200B
:1025910020203A2020202020202020202020202020
:1025A100204B6F6E7472617374752B004C69637A82
:1025B1006E696B20712E502E3A2020202020202081
:1025C100202020206820200050726F746F6B6F6C88
:1025D100202020203A2020202020202020206D694A
:1025E1006E20204B6F6E7472617374752D0044728E
:1025F100756B20202020202020203A202020202020
:1026010020202020202020200020204A657A796B7C
:102611002020202050726F746F6B6F6C202020205F
:102621004472756B202020205365727669736500B2
:10263100205354454C4C454E202020202020202062
:102641002020202020202020202020202020202089
:10265100202020202020002053455454494E47205B
:102661002020202020202020202020202020202069
:102671002020202020202020202020202000205247
:1026810045474C4147452020202020202020202064
:102691002020202020202020202020202020202039
:1026A10020202020002055535441574941432020E8
:1026B1002020202020202020202020202020202019
:1026C1002020202020202020202020004765626C2F
:1026D10061657365203A2020202020200020474595
:1026E100424C4145534520202020202020202020FD
:1026F100202020202020202020200046616E203A2A
:102701002020202020202020202020002046414E73
:1027110020202020202020202020202020202020B8
:1027210020202020202020202000536F7566666C19
:1027310065726965203A202020200020534F5546BC
:10274100464C455249452020202020202020202091
:1027510020202020202020200057656E74796C6194
:10276100746F72203A202020202020002057454EEF
:1027710054594C41544F5220202020202020202009
:1027810020202020202020202000444154454E4676
:1027910045484C4552202100506172616D65746558
:1027A10072207769726420617566005374616E648A
:1027B100617264776572742065696E6765737465AB
:1027C1006C6C7400426573746165746967656E2031
:1027D100647572636820454E54455200444154412A
:1027E1004552524F52202100506172616D657465EE
:1027F100722077696C6C20736574006F6E2073743E
:10280100616E6461726476616C75650050726573A6
:102811007320454E54455220746F20636F6E666974
:10282100726D00426C61642064616E7963682C0092
:1028310070727A796A6D756A6520706172616D6511
:102841007472007374616E646172646F77792C00C5
:10285100706F7477696572647A6E69652070727AD7
:10286100657A20454E5445520045525245555220F5
:10287100444520444F4E4E4545532021004C65733D
:1028810020706172616D657472657320766F6E740C
:1028910020657472652072616D616E65730064619B
:1028A1006E73206C6120636F6E6669677572617407
:1028B100696F6E20696E697469616C6500436F6E42
:1028C1006669726D65722070617320454E54455280
:1028D100001611161B16261631000000000000001C
:1028E10000163C1646164616510000000000000076
:1028F10000165C166B167A168600000000000000B8
:10290100001B601B741B881B94192D192D192D197F
:102911002D1B9F1BB11BC31BD5192D192D192D194A
:102921002D1BE71BF91C0B1C1C192D192D192D1919
:102931002D1C2E1C401C521C64192D192D192D19EA
:102941002D1C761C851C941CA3192D192D192D19CC
:102951002D1CB21CC41CC41CD6192D192D192D19DE
:102961002D1CE81CF31CF31CE8192D192D192D1928
:102971002D1CFE1D101CFE1D23192D192D192D199D
:102981002D1D351D3D1D3D1D45192D192D192D19C6
:102991002D1D4D1D551D551D5D192D192D192D1956
:1029A1002D1D641D751D8E1DA0192D192D192D1993
:1029B1002D1DB01DBC1DBC1DB0192D192D192D19B2
:1029C1002D1DC81DD41DE01DEC192D192D192D1912
:1029D1002D1DF91E051E131E211E2F1E40192D1916
:1029E1002D192D192D1E4D1E5B1E691E77192D19CE
:1029F1002D192D192D1E841E841E841E84192D1936
:102A01002D192D192D1E921EA11EA11EA1192D19C0
:052A11002D192D192D07
:1074900060C0376CFF168CFF1696FF16A0FF16AA69
:1074A000FF16B4FF16BEFF16C8FF16D2FF16DCFF8C
:1074B00016E6FF16F0FF16FAFF1704FF170EFF1768
:1074C00018FF1722FF172CFF1736FF1740FF174A28
:1074D000FF1754FF175EFF1768FF1772FF177CFF37
:1074E0001786FF1790FF179AFF17A4FF17AEFF1715
:1074F000B8FF17C2FF17CCFF17D6FF17E0FF17EA38
:10750000FF17F4FF17FEFF1808FF1812FF181CFFE3
:107510001826FF1830FF183AFF1844FF184EFF18BE
:1075200058FF1862FF186CFF1876FF1880FF188A42
:10753000FF1894FF189EFF18A8FF18B2FF18BCFF91
:1075400018C6FF18D0FF18DAFF18E4FF18EEFF186E
:10755000F8FF1902583754FF190CFF1914FF191BB3
:10756000FF1922FF192DFF192DFF192DFF192D5875
:10757000373CFF192EFF1938FF1940FF1949FF1931
:107580002DFF192DFF192DFF192D5836F4FF195312
:10759000FF195FFF1965FF1970FF192DFF192DFFE6
:1075A000192DFF192D5838ECFF197CFF1985FF198B
:1075B0008EFF1995FF192DFF192DFF192DFF192D7C
:1075C000583724FF199FFF19A9FF19B3FF19BAFFF4
:1075D000192DFF192DFF192DFF192D58370CFF19E3
:1075E000C2FF19C7FF19CDFF19D2FF192DFF192DA1
:1075F000FF192DFF192D6060388CFF19D8FF19E68F
:10760000FF19F3FF1A01FF1A0EFF1A1CFF1A29FFB8
:107610001A37FF1A44FF1A52FF1A5FFF1A6DFF1A3A
:107620007AFF1A88FF1A95FF1AA3FF19D8FF19E6E7
:10763000FF19F3FF1A01FF19D8FF19E6FF19F3FF2D
:107640001A01FF19D8FF19E6FF19F3FF1A01FF19F4
:10765000D8FF19E6FF19F3FF1A016060382CFF1AF2
:10766000B0FF1ABEFF1ACBFF1AD9FF1AE6FF1AF4B1
:10767000FF1B01FF1B0FFF1B1CFF1B2AFF1B37FFFC
:107680001B45FF1B52FF1AF4FF1B01FF1B0FFF19C5
:10769000D8FF19E6FF19F3FF1A01FF19D8FF19E601
:1076A000FF19F3FF1A01FF19D8FF19E6FF19F3FFBD
:0E76B0001A01FF19D8FF19E6FF19F3FF1A019E
:106209001200037F9C12C2EA7D077C007F1F7E007B
:1062190012B8A17BFF7A1E79B012C1817D077C007B
:106229007F037E0012B8A19003F8E075F00CA42456
:106239008CF582E43438F583C083C082900000E095
:10624900FF3395E0FED082D08375F003EF123375EA
:10625900EE75F003A42583F583E0FBA3E0FAA3E040
:10626900F912C1817D067C007F077E0012B8A17BEF
:10627900FF7A1E79B712C1817D047C007F137E00ED
:1062890012B8A17BFF7A1E79BB12C1817D027C0005
:106299007F027E0012B8A19003F8E0146026146012
:1062A9003F1460582403706E7BFF7A1E79BD12C1BA
:1062B90081E4FDFCFFFE12B8A17BFF7A1E79E11291
:1062C900C18180527BFF7A1F790B12C181E4FDFCE9
:1062D900FFFE12B8A17BFF7A1F792F12C181803688
:1062E9007BFF7A1F795912C181E4FDFCFFFE12B8C8
:1062F900A17BFF7A1F797D12C181801A7BFF7A1FEA
:1063090079A712C181E4FDFCFFFE12B8A17BFF7AD7
:106319001F79CB12C1817F0412A6FD7D027C007F0B
:10632900087E0012B8A1900204E0B401077F31127F
:10633900B92B80057F3012B92B900204E09036D139
:10634900F07D027C007F127E0012B8A19000B8E0B7
:10635900FEA3E0FF7D037C0012A21D7D067C007F69
:10636900067E0012B8A19036C7E0FEA3E0FF7D03C8
:106379007C0012A21D7D047C007F0F7E0012B8A153
:106389009000B1E0FEA3E0FF7C007D0A12310D7D93
:10639900037C0012A21D7D027C007F227E0012B8C0
:1063A900A19036BDE0FF3395E0FE7D027C0012A28C
:1063B9001D903954E4F0A37419F07BE57A00FD7C53
:1063C900007F0A7E00125591903954E4F0A37414A9
:1063D900F07B087A007D177C007F087E00125591BA
:1063E900903954E4F0A37414F07BE77A007D177CAC
:1063F900007FE77E001255917B017D187C007F09A3
:106409007E0012B65F7B017D187C007FE67E00125C
:10641900B65F903954E4F0A3742CF07B287A007DA0
:10642900267C007F287E00125591903954E4F0A310
:10643900742CF07BAC7A00FD7C007F287E0012551D
:1064490091903954E4F0A3742CF07BC87A00FD7C58
:10645900007FB67E00125591903954E4F0A374265A
:10646900F07BC87A007D2C7C007FC87E0012559194
:10647900903954E4F0A37426F07BAF7A007D2B7C2D
:10648900007FB17E00125591903954E4F0A374262F
:10649900F07BAA7A007D2B7C007FAC7E001255919F
:1064A900903954E4F0A37426F07BB47A007D2B7CF8
:1064B900007FB67E001255917D267C007F2D7E00DF
:1064C90012984F7B017A007D367C007FB37E0012E3
:0E64D90041327D257C007F6E7E0012B9B42218
:10984F00903929EEF0A3EFF0A3ECF0A3EDF09039EF
:10985F0029E0FAA3E0FB2401FFE43AFEEFC0E0EBBE
:10986F00240CFBE43AFAA3E0FFA3E0903954CFF0C5
:10987F00A3EFF0D0E0FF125591903929E0FAA3E061
:10988F00FBFFCEEACEEEC0E090392CE02401FD9034
:10989F00392BE03400FCA3E02403FE90392BE03495
:1098AF0000903954F0A3CEF0D0E0FE1255919039CC
:1098BF002AE0240DFB903929E03400FACFEBCFFEDC
:1098CF00EEC0E090392CE02401FD90392BE03400FC
:1098DF00FCA3E02403FE90392BE03400903954F0C0
:1098EF00A3CEF0D0E0FE12559190392AE02401FF6B
:1098FF00903929E03400FE90392CE02404FD903992
:10990F002BE03400FC7B0112B65F90392AE0240C67
:10991F00FF903929E03400FE90392CE02404FD90AB
:10992F00392BE03400FC7B0112B65F903929E0FA45
:10993F00A3E0FB2402FFE43AFEEEC0E090392CE0F6
:10994F002405FD90392BE03400FCEB240BFBE43AAB
:10995F00FAA3E02405FE90392BE03400903954F03F
:0A996F00A3CEF0D0E0FE12559122C5
:10413200903929EEF0A3EFF0A3ECF0A3EDF0CEEA74
:10414200CECFEBCFEA600302458DEF24FE7003026F
:1041520042921470030244102402600302458D90BF
:104162003929E0FAA3E0FB24FBFFEA34FFFEEEC0AC
:10417200E090392CE02402FD90392BE03400FCEB76
:104182002404FBE43AFAA3E024FEFE90392BE03447
:10419200FF903954F0A3CEF0D0E0FE125591903941
:1041A20029E0FAA3E0FB24FBFFEA34FFFEEEC0E0C5
:1041B20090392CE024FEFD90392BE034FFFCEB24F7
:1041C20004FBE43AFAA3E02402FE90392BE0340027
:1041D200903954F0A3CEF0D0E0FE125591903929D7
:1041E200E0FAA3E0FB24FAFFEA34FFFEEEC0E0901F
:1041F200392CE02401FD90392BE03400FCEB24053E
:10420200FBE43AFAA3E024FFFE90392BE034FF905E
:104212003954F0A3CEF0D0E0FE125591903929E046
:10422200FAA3E0FB24FAFFEA34FFFEEEC0E0903985
:104232002CE024FFFD90392BE034FFFCEB2405FB3E
:10424200E43AFAA3E02401FE90392BE034009039DD
:1042520054F0A3CEF0D0E0FE125591903929E0FA45
:10426200A3E0FB24FAFFEA34FFFEEFC0E0A3E0FC88
:10427200A3E0FDEB2405FBE43AFA90392BE0FFA31F
:10428200E0903954CFF0A3EFF0D0E0FF1255912225
:10429200903929E0FAA3E0FB24FAFFEA34FFFEEEAC
:1042A200C0E090392CE024FAFD90392BE034FFFC79
:1042B200EB2406FBE43AFAA3E02406FE90392BE055
:1042C2003400903933F0A3CEF0E4A3F0D0E0FE1234
:1042D200A31E903929E0FAA3E0FB24FCFFEA34FF95
:1042E200FEEEC0E090392CE02402FD90392BE03440
:1042F20000FCEB2404FBE43AFAA3E024FEFE90392E
:104302002BE034FF903954F0A3CEF0D0E0FE1255EA
:1043120091903929E0FAA3E0FB24FCFFEA34FFFE86
:10432200EEC0E090392CE02403FD90392BE03400FC
:10433200FCEB2404FBE43AFAA3E024FDFE90392BC3
:10434200E034FF903954F0A3CEF0D0E0FE12559144
:10435200903929E0FAA3E0FB24FCFFEA34FFFEEEE9
:10436200C0E090392CE02404FD90392BE03400FCAD
:10437200EB2404FBE43AFAA3E024FCFE90392BE0A0
:1043820034FF903954F0A3CEF0D0E0FE1255919054
:104392003929E0FAA3E0FB24FDFFEA34FFFEEEC078
:1043A200E090392CE02404FD90392BE03400FCEB42
:1043B2002403FBE43AFAA3E024FCFE90392BE03418
:1043C200FF903954F0A3CEF0D0E0FE12559190390F
:1043D20029E0FAA3E0FB24FEFFEA34FFFEEEC0E090
:1043E20090392CE02404FD90392BE03400FCEB24BE
:1043F20002FBE43AFAA3E024FCFE90392BE034FFFE
:10440200903954F0A3CEF0D0E0FE125591229039AB
:1044120029E0FAA3E0FB24FAFFEA34FFFEEEC0E053
:1044220090392CE024FAFD90392BE034FFFCEB2488
:1044320006FBE43AFAA3E02406FE90392BE03400AE
:10444200903933F0A3CEF0E4A3F0D0E0FE12A31E25
:10445200903929E0FAA3E0FB2402FFE43AFEEEC021
:10446200E090392CE02404FD90392BE03400FCEB81
:1044720024FEFBEA34FFFAA3E024FCFE90392BE091
:1044820034FF903954F0A3CEF0D0E0FE1255919053
:104492003929E0FAA3E0FB2403FFE43AFEEEC0E090
:1044A20090392CE02404FD90392BE03400FCEB24FD
:1044B200FDFBEA34FFFAA3E024FCFE90392BE03442
:1044C200FF903954F0A3CEF0D0E0FE12559190390E
:1044D20029E0FAA3E0FB2404FFE43AFEEEC0E090F8
:1044E200392CE02404FD90392BE03400FCEB24FC51
:1044F200FBEA34FFFAA3E024FCFE90392BE034FF00
:10450200903954F0A3CEF0D0E0FE125591903929A3
:10451200E0FAA3E0FB2404FFE43AFEEEC0E09039A7
:104522002CE02403FD90392BE03400FCEB24FCFB4F
:10453200EA34FFFAA3E024FDFE90392BE034FF9029
:104542003954F0A3CEF0D0E0FE125591903929E013
:10455200FAA3E0FB2404FFE43AFEEEC0E090392C1B
:10456200E02402FD90392BE03400FCEB24FCFBEA52
:1045720034FFFAA3E024FEFE90392BE034FF903999
:0C45820054F0A3CEF0D0E0FE12559122C0
:108103001200039003F8E01460771470030281E80F
:1081130014700302824B240360030282AC7D077C4C
:10812300007F0F7E0012B8A17BFF7A1F79F512C181
:10813300817D057C007F017E0012B8A17BFF7A1F41
:1081430079FF12C1817D047C007F017E0012B8A1FA
:108153007BFF7A20792412C1817D037C007F017E1D
:108163000012B8A17BFF7A20793712C181E4FDFCAC
:10817300FFFE12B8A17BFF7A20794E12C1810282E1
:10818300AC7D077C007F0F7E0012B8A17BFF7A1FB6
:1081930079F512C1817D057C007F017E0012B8A1B3
:1081A3007BFF7A20797512C1817D047C007F017E7B
:1081B3000012B8A17BFF7A20792412C1817D037C50
:1081C300007F017E0012B8A17BFF7A20799A12C149
:1081D30081E4FDFCFFFE12B8A17BFF7A2079B11286
:1081E300C1810282AC7D077C007F0F7E0012B8A1A3
:1081F3007BFF7A2079D912C1817D057C007F017EC6
:108203000012B8A17BFF7A2079E312C1817D047C3F
:10821300007F017E0012B8A17BFF7A20792412C16E
:10822300817D037C007F017E0012B8A17BFF7A2150
:10823300790812C181E4FDFCFFFE12B8A17BFF7A2D
:1082430021791F12C18180617D077C007F0F7E0031
:1082530012B8A17BFF7A21794712C1817D057C0089
:108263007F017E0012B8A17BFF7A21795112C1816F
:108273007D047C007F017E0012B8A17BFF7A207908
:108283002412C1817D037C007F017E0012B8A17B93
:10829300FF7A20793712C181E4FDFCFFFE12B8A1F9
:0F82A3007BFF7A21797612C1817F0412A6FD221A
:10AC4B001200037D047C007F087E0012B8A17BFFFD
:10AC5B007A21799E12C1817F0412A6FD9003F8E040
:10AC6B001460331460561460792403600302AD1230
:10AC7B007D077C007F0E7E0012B8A17BFF7A2179C5
:10AC8B00B112C181E4FDFCFFFE12B8A17BFF7A215A
:10AC9B0079BB12C181227D077C007F0E7E0012B82A
:10ACAB00A17BFF7A2179E512C181E4FDFCFFFE1245
:10ACBB00B8A17BFF7A2179ED12C181227D077C003F
:10ACCB007F0E7E0012B8A17BFF7A22791712C18109
:10ACDB00E4FDFCFFFE12B8A17BFF7A22792212C1A0
:10ACEB0081227D077C007F0E7E0012B8A17BFF7A4C
:10ACFB0022794C12C181E4FDFCFFFE12B8A17BFF4F
:08AD0B007A22795512C1812260
:10AD13001200037D047C007F087E0012B8A17BFF34
:10AD23007A21799E12C1817F0412A6FD9003F8E077
:10AD33001460331460561460792403600302ADDA9F
:10AD43007D077C007F0E7E0012B8A17BFF7A2279FB
:10AD53007F12C181E4FDFCFFFE12B8A17BFF7A22C2
:10AD6300798A12C181227D077C007F0E7E0012B892
:10AD7300A17BFF7A2279B412C181E4FDFCFFFE12AC
:10AD8300B8A17BFF7A2279C012C181227D077C00A2
:10AD93007F0A7E0012B8A17BFF7A2279EA12C18171
:10ADA300E4FDFCFFFE12B8A17BFF7A2279FC12C1FD
:10ADB30081227D077C007F0E7E0012B8A17BFF7A83
:10ADC30023792612C181E4FDFCFFFE12B8A17BFFAB
:08ADD3007A23793512C18122B7
:1071FA001200039003F8E0147003027292147003F1
:10720A0002730A147003027381240360030273F683
:10721A007D077C007F0A7E0012B8A17BFF7A237962
:10722A005F12C1817D057C007F027E0012B8A17BBE
:10723A00FF7A23797312C1817D047C007F027E006C
:10724A0012B8A17BFF7A23799812C1817D037C0051
:10725A007F027E0012B8A17BFF7A2379B212C18124
:10726A007D027C007F027E0012B8A17BFF7A23791F
:10727A00D712C181E4FDFCFFFE12B8A17BFF7A237D
:10728A0079F112C1810273F67D077C007F0A7E00C4
:10729A0012B8A17BFF7A24791A12C1817D057C007C
:1072AA007F027E0012B8A17BFF7A24792912C1815C
:1072BA007D047C007F027E0012B8A17BFF7A2479CC
:1072CA004E12C1817D037C007F027E0012B8A17B31
:1072DA00FF7A24796812C1817D027C007F027E00D8
:1072EA0012B8A17BFF7A24798D12C181E4FDFCFFDB
:1072FA00FE12B8A17BFF7A2479A712C1810273F624
:10730A007D077C007F0F7E0012B8A17BFF7A24796B
:10731A00D012C1817D057C007F027E0012B8A17B5C
:10732A00FF7A2479D812C1817D047C007F027E0015
:10733A0012B8A17BFF7A2479FE12C1817D037C00F9
:10734A007F027E0012B8A17BFF7A25791812C181CB
:10735A007D027C007F027E0012B8A17BFF7A25792C
:10736A003E12C181E4FDFCFFFE12B8A17BFF7A2523
:10737A00795812C18180757D077C007F0F7E0012CB
:10738A00B8A17BFF7A25798012C1817D057C007FB7
:10739A00017E0012B8A17BFF7A25798712C1817D0F
:1073AA00047C007F017E0012B8A17BFF7A2579ADAB
:1073BA0012C1817D037C007F017E0012B8A17BFF90
:1073CA007A2579C912C1817D027C007F017E001273
:1073DA00B8A17BFF7A2579EF12C181E4FDFCFFFE9B
:1073EA0012B8A17BFF7A26790A12C1817D057C0039
:1073FA007F0F7E0012B8A19003F8E0FF75F018A481
:10740A00246CF582E43437F58375F003EF12337593
:10741A00E0FBA3E0FAA3E0F912C1817D037C007FBF
:10742A00147E0012B8A19001FCE0FEA3E0FF7D03E8
:10743A007C0012A21D7D027C007F0F7E0012B8A183
:10744A00900226E0FF3395E0FEEF25E0FFEE33FEE3
:10745A0074D22FF58274293EF583E493FE74019366
:0F746A00CAEECAF97BFF12C1817F0412A6FD2270
:10C066001200037D077C007F0F7E0012B8A19003AB
:10C07600F8E075F003A42424F582E43437F583E070
:10C08600FBA3E0FAA3E0F912C1817D037C007F0CDB
:0FC096007E0012B8A17BFF7A21799E12C1812210
:10ADDB001200037D077C007F0F7E0012B8A1900349
:10ADEB00F8E025E024F2F582E43428F583E493FEC1
:10ADFB00740193CAEECAF97BFF12C1817D057C00F9
:10AE0B00E4FFFE12B8A19003F8E025E024E2F582FE
:10AE1B00E43428F583E493FE740193CAEECAF97BFC
:10AE2B00FF12C1817D057C007F147E0012B8A190BA
:10AE3B0003F8E025E024D2F582E43428F583E4938B
:10AE4B00FE740193CAEECAF97BFF12C181E4FDFCCB
:10AE5B00FFFE12B8A19003F8E014601514601D14E6
:10AE6B0060252403702A7BFF7A26793112C18180F9
:10AE7B001F7BFF7A26795812C18180147BFF7A26BB
:10AE8B00797F12C18180097BFF7A2679A612C18155
:06AE9B007F0412A6FD2257
:10B0DA001200039003F8E014603414605814607C82
:10B0EA002403600302B18B7D057C007F0A7E001277
:10B0FA00B8A17BFF7A2679CD12C181E4FDFCFFFE5F
:10B10A0012B8A17BFF7A2679DE12C18180737D0590
:10B11A007C007F0A7E0012B8A17BFF7A2679FC1296
:10B12A00C181E4FDFCFFFE12B8A17BFF7A27790DED
:10B13A0012C181804C7D057C007F0A7E0012B8A175
:10B14A007BFF7A27792B12C181E4FDFCFFFE12B83E
:10B15A00A17BFF7A27793C12C18180257D057C007D
:10B16A007F0A7E0012B8A17BFF7A27795A12C18121
:10B17A00E4FDFCFFFE12B8A17BFF7A27796D12C1AC
:07B18A00817F0412A6FD22E3
:1091BF001200039003F8E01460641470030292CF5E
:1091CF0014700302927E2403600302931F7D067CBA
:1091DF00007F0F7E0012B8A17BFF7A27798B12C117
:1091EF00817D047C007F047E0012B8A17BFF7A276B
:1091FF00799912C1817D037C007F047E0012B8A192
:10920F007BFF7A2779AC12C1817D017C007F047EC0
:10921F000012B8A17BFF7A2779C512C181227D0682
:10922F007C007F0F7E0012B8A17BFF7A2779DD12B9
:10923F00C1817D047C007F047E0012B8A17BFF7A80
:10924F002779E912C1817D037C007F047E0012B86B
:10925F00A17BFF7A2779FC12C1817D017C007F04FD
:10926F007E0012B8A17BFF7A28790D12C181227D71
:10927F00067C007F0F7E0012B8A17BFF7A2879242D
:10928F0012C1817D047C007F047E0012B8A17BFF98
:10929F007A28793112C1817D037C007F047E001210
:1092AF00B8A17BFF7A28794412C1817D017C007FB0
:1092BF00047E0012B8A17BFF7A28795112C1812256
:1092CF007D067C007F0A7E0012B8A17BFF7A287989
:1092DF006A12C1817D047C007F047E0012B8A17BDD
:1092EF00FF7A28797E12C1817D037C007F047E0086
:1092FF0012B8A17BFF7A28799F12C1817D017C0072
:10930F007F047E0012B8A17BFF7A2879BE12C1813B
:01931F00222B
:10A6FD00903939EFF0903954E4F0A3740BF07BEFFF
:10A70D007A00FD7C00E4FFFE125591903939E0246A
:10A71D00F9604A2403600302A7EE903954E4F0A3D4
:10A72D00740BF07B3B7A00E4FDFC7F3BFE125591F0
:10A73D00903954E4F0A3740BF07B777A00E4FDFCC0
:10A74D007F77FE125591903954E4F0A3740BF07B92
:10A75D00B37A00E4FDFC7FB3FE125591229039547B
:10A76D00E4F0A3740BF07B227A00E4FDFC7F22FE63
:10A77D00125591903954E4F0A3740BF07B447A0098
:10A78D00E4FDFC7F44FE125591903954E4F0A3741E
:10A79D000BF07B667A00E4FDFC7F66FE125591900E
:10A7AD003954E4F0A3740BF07B887A00E4FDFC7F50
:10A7BD0088FE125591903954E4F0A3740BF07BAAE6
:10A7CD007A00E4FDFC7FAAFE125591903954E4F015
:10A7DD00A3740BF07BCC7A00E4FDFC7FCCFE12550C
:02A7ED009122B7
:10BD1A00EF5407FFE5C520E3FB8FC5E4FDFC0DBD2D
:10BD2A0000010CED64C84C70F5EF2408F5C5E4FC7D
:10BD3A00FD0DBD00010CED64054C70F5E5C520E371
:10BD4A00FBAFC57C00CDEFCDED7E007806CEC313E8
:10BD5A00CE13D8F9FDCCEECCAFC6EF75F004A42D06
:09BD6A00FDE5F03CFCFECFEDCF3D
:01BD730022AD
:054DFC00903927EFF0E3
:104E0100E4A3F0A3F0903927E024BBF582E4340059
:104E1100F583E0FF643A6012EF643B600D90021F7E
:104E2100E04402F0903927E0FF22903927E004F0B6
:104E3100E0C394964002E4F0E4903928F0903928D8
:104E4100E0FFD394045052903927E024BBF582E46B
:104E51003400F583E0FE74DF2FF582E43436F58308
:104E6100EEF0903927E004F0E024BBF582E4340051
:104E7100F583E0FF643D6004EFB43B15903928E011
:104E810024E0F582E43436F583E4F09039287404A3
:104E9100F0903928E004F080A4903928E024DFF56F
:104EA10082E43436F583E4F0903928F0903928E033
:104EB100FFD39415503DA37401F0EF75F00CA424B9
:104EC100FCF582E43402F583E0FBA3E0FAA3E0F809
:104ED100CCEACCCDEBCD7B017A3679DF12357CEF94
:104EE10070099039287415F0E4A3F0903928E00492
:104EF100F080B9903929E0600D90021FE04404F080
:104F0100903927E0FF229002FCE0FBA3E0FAA3E046
:104F1100F8CCEACCCDEBCD7B017A3679DF12357C4A
:104F2100EF70059001EC04F0900308E0FBA3E0FAB8
:104F3100A3E0F8CCEACCCDEBCD7B017A3679DF1258
:104F4100357CEF70069001EC7402F0900314E0FBE5
:104F5100A3E0FAA3E0F8CCEACCCDEBCD7B017A3625
:104F610079DF12357CEF70069001EC7403F0900349
:104F710020E0FBA3E0FAA3E0F8CCEACCCDEBCD7BBB
:104F8100017A3679DF12357CEF70069001EC7404FA
:104F9100F090032CE0FBA3E0FAA3E0F8CCEACCCD3F
:104FA100EBCD7B017A3679DF12357CEF700690010B
:104FB100EC7405F0900338E0FBA3E0FAA3E0F8CC31
:104FC100EACCCDEBCD7B017A3679DF12357CEF70FF
:104FD100069001EC7406F0900344E0FBA3E0FAA311
:104FE100E0F8CCEACCCDEBCD7B017A3679DF123516
:104FF1007CEF70069001EC7407F0900350E0FBA386
:10500100E0FAA3E0F8CCEACCCDEBCD7B017A36799E
:10501100DF12357CEF70069001EC7408F090035CB0
:10502100E0FBA3E0FAA3E0F8CCEACCCDEBCD7B0129
:105031007A3679DF12357CEF70069001EC7409F055
:10504100900368E0FBA3E0FAA3E0F8CCEACCCDEB57
:10505100CD7B017A3679DF12357CEF70069001EC59
:10506100740AF0900374E0FBA3E0FAA3E0F8CCEA41
:10507100CCCDEBCD7B017A3679DF12357CEF700632
:105081009001EC740BF0900380E0FBA3E0FAA3E045
:10509100F8CCEACCCDEBCD7B017A3679DF12357CC9
:1050A100EF70069001EC740CF090038CE0FBA3E030
:1050B100FAA3E0F8CCEACCCDEBCD7B017A3679DFEF
:1050C10012357CEF70069001EC740DF0900398E0BE
:1050D100FBA3E0FAA3E0F8CCEACCCDEBCD7B017ADF
:1050E1003679DF12357CEF70069001EC740EF0908A
:1050F10003A4E0FBA3E0FAA3E0F8CCEACCCDEBCD2E
:105101007B017A3679DF12357CEF70069001EC7401
:105111000FF09003B0E0FBA3E0FAA3E0F8CCEACCF7
:10512100CDEBCD7B017A3679DF12357CEF700690BD
:1051310001EC7410F09003BCE0FBA3E0FAA3E0F8EB
:10514100CCEACCCDEBCD7B017A3679DF12357CEF21
:1051510070069001EC7411F09003C8E0FBA3E0FA33
:10516100A3E0F8CCEACCCDEBCD7B017A3679DF1226
:10517100357CEF70069001EC7412F09003D4E0FBE3
:10518100A3E0FAA3E0F8CCEACCCDEBCD7B017A36F3
:1051910079DF12357CEF70069001EC7413F0900307
:1051A100E0E0FBA3E0FAA3E0F8CCEACCCDEBCD7BC9
:1051B100017A3679DF12357CEF70069001EC7414B8
:1051C100F09003ECE0FBA3E0FAA3E0F8CCEACCCD4D
:1051D100EBCD7B017A3679DF12357CEF70069001D9
:0E51E100EC7415F0E4903929F0903927E0FFC6
:0151EF00229D
:06932000903927EFF0FB7D
:1093260090392A12334400000000903928E4F0A353
:1093360004F0EBFF3395E0FE74BB2FF58274003E1C
:10934600F583E0643D60057EFF7FFF22903927E0CC
:109356002407FF903927E0FEFD3395E0FC74BB2D12
:10936600F58274003CF583E0B43B0BC3EF6480F8F0
:10937600EE648098401B903927E004F0E0FD3395B9
:10938600E0FCC3ED9496EC6480948040C6E4F080E3
:10939600C2903927E014F0903927E0FF3395E0FEBC
:1093A60074BB2FF58274003EF583E0FF643D7003C5
:1093B60002944FC3EF648094B04008D3EF64809466
:1093C600B940057EFF7FFF22903927E0FF3395E005
:1093D600FE74BB2FF58274003EF583E0FF3395E003
:1093E600FEEF24D0FFEE34FFFE903928E0FCA3E028
:1093F600FD1230A6E4FCFD90392E12333890392A3E
:10940600E0FCA3E0FDA3E0FEA3E0FFA3E0F8A3E0F9
:10941600F9A3E0FAA3E0FBEF2BFFEE3AFEED39FDF0
:10942600EC38FC90392A123338903928E0FEA3E054
:10943600FF7C007D0A1230A6903928EEF0A3EFF0EB
:10944600903927E014F002939DE47FFF7E7FFDFCB8
:1094560090392AE0F8A3E0F9A3E0FAA3E0FBD312DF
:10946600332740057EFF7FFF2290392CE0FEA3E0E4
:01947600FFF6
:0194770022D2
:0300230002A4191B
:10A41900C0E0C083C082C0D0ECC0E0EDC0E0EEC0B7
:04A42900E0EFC0E0C0
:10A42D0020980302A4FBAF99C298EF640D601690BB
:10A43D000202E0FE04F074192EF582E43400F58377
:10A44D00EFF002A4F0900202E0FF04F074192FF572
:10A45D0082E43400F583E4F0FF74542FF582E43484
:10A46D0001F583E4F074BB2FF582E43400F583E449
:10A47D00F00FBF96E49001F2E4F09001FAE0241998
:10A48D00F582E43400F583E0FF60569001F2E0FDC3
:10A49D003395E0FC74BB2DF58274003CF583EFF031
:10A4AD009001F2E004F0E0FFFD3395E0FC74BB2D6C
:10A4BD00F58274003CF583E4F09001FAE004F0E0DD
:10A4CD00C394964002E4F0EF3395E0FEC3EF94960B
:10A4DD00EE6480948040059001F2E4F04387108093
:0EA4ED0099D212900202E0C394964002E4F06D
:10A4FB00D0E0FFD0E0FED0E0FDD0E0FCD0D0D082A9
:05A50B00D083D0E03216
:10C0A500E49039E7F0EF602020981143871012B231
:10C0B500FCEF7003EE640870EF7FAA22E599547FC8
:10C0C5009039E7F0C298800D30980AE599547F9031
:0CC0D50039E7F0C298C2989039E7E0FF0C
:01C0E100223C
:10C1FE00CDEFCD200508900209E04FF0800E3005FE
:10C20E000BC374FF9DFF900209E05FF0900209E0FE
:05C21E0090C060F02259
:10C299007D107CC08D828C83E05F6F7002D322C3D6
:01C2A9002272
:09C2D8002020202D2D2020200043
:0AC2BA00E4F5D8D2DFD2D8D2DE229C
:0B8D9700903991EFF0A3ECF0A3EDF099
:108DA200E490399CF0A3F075D8C1C2DCD2DDD208C0
:108DB200D20990399AF0A3F0EBB41004D20A8002DF
:108DC200C20A200803028EEE438710E4FFFE20DB76
:108DD2000E438710EF1F70011EEF4E70F1C2092083
:108DE2000903028EE9AFD9EF24F8604D24F0605FE9
:108DF20024F8605424F8607224F8606E24F870033A
:108E0200028EDB24286003028EE2C390399DE09437
:108E12001E90399CE064809480501AA3E004F070A4
:108E22000690399CE004F0903991E025E0F5DAC231
:108E3200DCC2DB808DE4FEFF22903991E025E0F573
:108E4200DAC2DCC2DB028DC4D2DDC2DB028DC4C257
:108E5200DDC2DC300A09903992E0A3F5DA8006908F
:108E62003993E0F5DAC2DB028DC4200A5B903998AF
:108E7200E0FEA3E0FFA3E0FCA3E0FDC39FEE64805D
:108E8200F8EC6480984016D3EF9400EE64809480EE
:108E92004006C2DDD2DCC2DBC208028DC4C2DDC222
:108EA200DC903995E0FBA3E0FAA3E0F98D828C8394
:108EB200123045F5DA90399BE004F0700690399A49
:108EC200E004F0C2DB028DC4C20AC2DDC2DC90390A
:108ED20093E0F5DAC2DB028DC4D2DDC2DB028DC4BF
:108EE200C209C208028DC4C208028DC43009057EBF
:078EF200007F0122E4FEFFF6
:018EF9002256
:0595C900903986EFF06F
:1095CE0090398AE0F9A3E0FAA3E0903995C9F0A3A7
:1095DE00EAF0A3E9F0E4A3F0A3F0128D97EF4E703A
:1095EE0003FEFF2275D8C1C2DAD2DDD206D207E45D
:1095FE0090398FF0A3F020060302970A438710E4F8
:10960E00FFFE20DB0E438710EF1F70011EEF4E7022
:10961E00F1C207200703029705AFD9EF24F0601EB1
:10962E0024D870030296F724F8602024F8601C24D6
:10963E00F8605D24F86033245060030296FE903982
:10964E0086E025E004F5DAC2DB80ABD390398EE0FC
:10965E00940190398DE0648094804004D2DA8002C7
:10966E00C2DAC2DDC2DCC2DB808C90398AE0FBA399
:10967E00E0FAA3E0F990398FE0FEA3E0F5828E8345
:10968E00E5DA123084C2DDD2DCC2DBC206029604F9
:10969E0090398AE0FBA3E0FAA3E0F990398FE0FE5F
:1096AE00A3E0F5828E83E5DA123084903990E004DF
:1096BE00F0700690398FE004F090398EE024FFFFB1
:1096CE0090398DE034FFFEC3903990E09FEE6480B8
:1096DE00F890398FE06480984004C2DA8002D2DAC2
:1096EE00C2DCC2DDC2DB029604D2DDC2DB0296040E
:1096FE00C207C206029604C2060296043007057E11
:07970E00007F0122E4FEFFD1
:019715002231
:10878200903939EEF0A3EFF0A3ECF0A3EDF0A3EAF9
:04879200F0A3EBF075
:10879600E490394EF0A3F07B01A304F0A37439F002
:1087A600A374D0F0E4903945F0903943E0FEA3E09D
:1087B600FF7C007D0A12310DEFC454F0FB90394363
:1087C600E0FEA3E0FF7C007D0A12310DEB2D90390F
:1087D60046F0903941E0FEA3E0FF7C007D0A1231AD
:1087E6000DEFC454F0FB903941E0FEA3E0FF7C009E
:1087F6007D0A12310DEB2D903947F090393FE0FE9E
:10880600A3E0FF7C007D0A12310DEFC454F0FB900B
:10881600393FE0FEA3E0FF7C007D0A12310DEB2D0F
:10882600903948F090393DE0FEA3E0FF7C007D0AD8
:1088360012310DEFC454F0FF90393AE0540375F04D
:1088460040A42FFB90393DE0FEA3E0FF7C007D0AAB
:1088560012310DEB2D903949F090393BE0FEA3E043
:10886600FF7C007D0A12310DEFC454F0FB90393BBA
:10887600E0FEA3E0FF7C007D0A12310DEB2D90395E
:108886004AF0A37401F0A37439F0A37439F0903957
:1088960039E0F9A3E0FF903950E0FBA3E0FAA3E04A
:1088A600C98FF012319A9039957401F0A37439F09A
:1088B600A37445F0A3E4F0A37406F07B087D017C65
:1088C600007F51128D97EF4E700E90394FE004F0F5
:1088D600700690394EE004F090394BE0F9A3E0FAC7
:1088E600A3E0903995C9F0A3EAF0A3E9F0A3E4F078
:1088F600A37402F07B107D257C0C7F50128D97EFC0
:108906004E700E90394FE004F0700690394EE00438
:01891600F070
:01891700223D
:0B891800903977EBF0A3EAF0A3E9F040
:108923009039837401F0A37439F0A37480F0E49058
:108933003982F090398A7401F0A37439F0A3747A00
:10894300F0A3E4F0A37406F07B087D017C007F5163
:108953001295C9EF64014E600C903982E004F0E097
:10896300C3940440CE90397BE0FD54F0FFC4540F10
:1089730075F00AA4FFED540F7C002FFFEC35F0FED9
:10898300903977E0FBA3E0FAA3E0F990000AEE8FB9
:10899300F01231B990397CE054F0FFC4540F75F0F4
:1089A3000AA4FFE0540F2FFFEC35F09000088FF07E
:1089B3001231B990397DE054F0FFC4540F75F00AB9
:1089C300A4FFE0540F2FFFEC35F09000068FF01258
:1089D30031B990397EE05430FFC4540F75F00AA4C6
:1089E300FFE0540F2FFFEC35F09000048FF01231AD
:1089F300B990397FE05410FFC4540F75F00AA4FFF7
:108A0300E0540F2FFFEC35F09000028FF01231B9D4
:108A130012316FFFAEF05403FD90397EE054C0FB7A
:108A2300C4131354036D7001EC6008900223E00437
:108A3300F08005E4900223F0900223E0C394064003
:108A430069EF2401FFE43E903980F0A3EFF0903901
:108A5300837401F0A37439F0A37480F0903983E038
:108A6300F9A3E0FAA3E0903995C9F0A3EAF0A3E9EA
:108A7300F0A3E4F0A37402F07B107D257C0C7F50FF
:108A8300128D97EF4E7006903982E004F090398092
:108A9300E0F9A3E0FF903977E0FBA3E0FAA3E0C994
:0A8AA3008FF012319AE4900223F0E4
:018AAD0022A6
:0E947800903939EFF0A3EBF0A3EAF0A3E9F08E
:10948600A3E0FAA3E0FB7C007D20FFCEEACE1231FA
:109496000D903941EEF0A3EFF07C007D20CFEBCFAD
:1094A600CEEACE12310D903945ECF0A3EDF0E49002
:1094B6003943F0A3F0903941E0FEA3E0FFA3E0FCBE
:1094C600A3E0FDC39FEE6480F8EC64809850799029
:1094D6003939E0FF3395E0FEEF7806C333CE33CE5D
:1094E600D8F924C0FBEE34FFFAEDCEECCE7805C3F6
:1094F60033CE33CED8F92BFFEA3EFE90393FF0FC4F
:10950600A3EFF0FD90393AE0F9A3E0FAA3E0903931
:1095160095C9F0A3EAF0A3E9F0A3E4F0A37420F060
:109526007B107F50128D97EF4E7002FF2290393BD1
:10953600E475F020123143903944E004F07006904F
:109546003943E004F00294BB903945E07002A3E091
:10955600606E903939E0FF3395E0FEEF24FFFFEEB1
:1095660034FFFEEF7806C333CE33CED8F9FDCCEE0A
:10957600CC903941E0FEA3E07805C333CE33CED894
:10958600F92DFFEC3EFE90393FF0FCA3EFF0FD9085
:10959600393AE0F9A3E0FAA3E0903995C9F0A3EAD5
:1095A600F0A3E9F0903945E0FFA3E0903998CFF0B9
:1095B600A3EFF07B107F50128D97EF4E7002FF22C3
:0295C6007F0024
:0195C8002280
:10BD740090394CEBF0A3EAF0A3E9F0EF3395E0FE41
:10BD8400EF24FFFFEE34FFFEEF7806C333CE33CE4D
:10BD9400D8F9FDCCEECC90394CE0F9A3E0FAA3E05D
:10BDA40090398AC9F0A3EAF0A3E9F090394FE0FF93
:10BDB400A3E090398DCFF0A3EFF07B107F50129564
:0ABDC400C9EF4E7002FF227F01223A
:0BA51000903947EBF0A3EAF0A3E9F05C
:10A51B0090394BE0FCB4501DEDFF3395E0FEEF7826
:10A52B0006C333CE33CED8F924C0FFEE34FF9039B7
:10A53B004CF0A3EFF0ECB44D17CFEDCFEF3395E02C
:10A54B00EFFEE42400FFEE340390394CF0A3EFF060
:10A55B0090394CE0FCA3E0FD90398A7401F0A374B0
:10A56B0039F0A3744EF0A3E4F0A304F07B107F50FA
:10A57B001295C9EF4E7002FF2290394EE0FFC39443
:10A58B00014059EFD39410505390394DE004F070C3
:10A59B000690394CE004F090394CE0FCA3E0FD90C0
:10A5AB003947E0F9A3E0FAA3E090398AC9F0A3EAAE
:10A5BB00F0A3E9F0A3E4F0A37409F07B107F501231
:10A5CB0095C9EF4E7002FF22903947E0FBA3E0FAEA
:10A5DB00A3E0F9900008E4123084801A903947E028
:10A5EB00FBA3E0FAA3E0F8CCEACCCDEBCD7BFF7A72
:0BA5FB00C279D812366590394EE0FF9F
:01A606002231
:0E8EFA00903931EFF0A3EBF0A3EAF0A3E9F01A
:108F0800A3E0FAA3E0FB7C007D20FFCEEACE12317D
:108F18000D903939EEF0A3EFF07C007D20CFEBCF38
:108F2800CEEACE12310DED24FFFEEC34FF90393D30
:108F3800F0A3CEF0E490393BF0A3F0903939E0FE8D
:108F4800A3E0FFA3E0FCA3E0FDC39FEE6480F8EC80
:108F58006480984003028FE7903931E0FF3395E051
:108F6800FEEF24FFFFEE34FFEFFEE42400FBEE34B7
:108F780004FAEDCEECCE7805C333CE33CED8F92B38
:108F8800FFEA3EFE903937F0FCA3EFF0FD9039324E
:108F9800E0F9A3E0FAA3E0903995C9F0A3EAF0A3B9
:108FA800E9F0A3E4F0A37420F07B107F50128D97B2
:108FB800EF4E7002FF22903933E475F020123143EE
:108FC800E4FFFE0FBF00010EEF64644E70F59039A8
:108FD8003CE004F0700690393BE004F0028F4390C7
:108FE800393DE07002A3E06069903931E0FF3395C4
:108FF800E0FEEF24FFFFEE34FFEFFEE42400FDEE79
:109008003404FC903939E0FEA3E07805C333CE334D
:10901800CED8F92DFFEC3EFE903937F0FCA3EFF0E7
:10902800FD903932E0F9A3E0FAA3E0903995C9F050
:10903800A3EAF0A3E9F090393DE0FFA3E090399866
:10904800CFF0A3EFF07B107F50128D97EF4E700298
:04905800FF227F0074
:01905C0022F1
:10BDCE00903933EBF0A3EAF0A3E9F0EF3395E0FE00
:10BDDE00EF24FFFFEE34FFEFFEE42400FDEE34040B
:10BDEE00FC903933E0F9A3E0FAA3E090398AC9F068
:10BDFE00A3EAF0A3E9F0903936E0FFA3E090398D85
:10BE0E00CFF0A3EFF07B107F501295C9EF4E70026A
:05BE1E00FF227F01225C
:06BF9F00903974123338E2
:10BFA5009039787401F0A37439F0A37474F0903962
:10BFB50078E0F9A3E0FAA3E0903995C9F0A3EAF097
:10BFC500A3E9F0A3E4F0A37404F07B107D007C0CDE
:0DBFD5007F50128D97EF4E7002FF227F000B
:01BFE200223C
:10BE72009039277401F0A37439F0A3742AF0903931
:10BE820027E0F9A3E0FAA3E090398AC9F0A3EAF027
:10BE9200A3E9F0A3E4F0A37404F07B107D007C0C12
:10BEA2007F501295C9EF4E7005FFFEFDFC229039BE
:0CBEB2002AE0FCA3E0FDA3E0FEA3E0FFFB
:01BEBE002261
:0AC2C400759852758850758DFD22A3
:10C27500758922758C47D28C75EA8175C9DCE4F520
:02C28500A922EC
:0AC2CE00C2AF75A802D2ECD2AF2275
:10C25F00E4FF7F96900019E4F0A3DFFCE490020264
:05C26F00F09001FAF05F
:01C2740022A7
:10C2AA0039303930003231303600C2AAC2AAC2AFA0
:10BF56009001F4E0F8A3E0F9A3E0FAA3E02FFFEAEA
:10BF66003EFEE93DFDE83CFC90396E1233389039CF
:10BF76006EE0FCA3E0FDA3E0FEA3E0FF9001F4E089
:10BF8600F8A3E0F9A3E0FAA3E0FBC31233275008B5
:08BF960043871012AA9F80D618
:01BF9E002280
:10B2FC00E490396EF0A3F0A3F0A3F0A3F0A3F07DDB
:10B30C00107CC08D828C83E044F07F00FE903972FB
:10B31C00F0A3EFF0FDF5828C83E0FDEEEDFF9039AC
:10B32C0072EEF0A3EFF0F4FFEEF4903972F0A3EFAD
:10B33C00F043871012AA9F903972E0FEA3E0FF4EF3
:10B34C00700122903970E0FCA3E0FDA3E0FEA3E0C5
:10B35C00FF6D7002EE6C70047B0180027B00ED4C83
:10B36C0060047D0180027D00ED5B600890396FE028
:10B37C0004F08005E490396FF090396FE0D3941E9F
:10B38C00400122903970EEF0A3EFF090396EE0049A
:10B39C00F0E0C394FA500302B30B903972E0FEA3B1
:02B3AC00E0FFC0
:01B3AE00227C
:1078F30090393BECF0A3EDF0A3EAF0A3EBF0903961
:0679030039EEF0A3EFF0E5
:10790900903940EEF0A3EFF0E4A3F0A3F012B2FC3B
:10791900903944EEF0A3EFF08EF01233C77AA80144
:107929000079F10200793A04007AC0080000007B6E
:1079390011903943E004F07006903942E004F09068
:10794900393AE004F07006903939E004F090393D95
:10795900E0FEA3E0FFC390393AE09FEE6480F8901F
:107969003939E06480984005EEF0A3EFF090393F93
:10797900E0FF3395E0FEC39039E1E09FFF9039E0E5
:10798900E09EFEF0A3EFF09039E2E0FCA3E0FD12E7
:10799900B8A1903939E0FEA3E0FF90393FE0FD330B
:1079A90095E0FC12A21D903942E0FEA3E0FFC394CA
:1079B9000AEE94004024EF9428EE9400400E7F02D2
:1079C9007E007D007C0012BF560279167F0A7E0078
:1079D9007D007C0012BF560279167F147E007D005F
:1079E9007C0012BF56027916903943E004F0700604
:1079F900903942E004F090393AE024FFF0903939A7
:107A0900E034FFF090393BE0FEA3E0FFD390393A30
:107A1900E09FEE6480F8903939E06480985005EE73
:107A2900F0A3EFF090393FE0FF3395E0FEC39039C2
:107A3900E1E09FFF9039E0E09EFEF0A3EFF090397E
:107A4900E2E0FCA3E0FD12B8A1903939E0FEA3E021
:107A5900FF90393FE0FD3395E0FC12A21D903942B9
:107A6900E0FEA3E0FFC3940AEE94004024EF9428BB
:107A7900EE9400400E7F027E007D007C0012BF560E
:107A89000279167F0A7E007D007C0012BF560279BA
:107A9900167F147E007D007C0012BF56027916E421
:107AA900903944F0A3F07F1EFEFDFC12BF569039B9
:107AB90039E0FEA3E0FF22E4903944F0A3F07F1EF1
:107AC900FEFDFC12BF5690393FE0FF3395E0FEC33F
:107AD9009039E1E09FFF9039E0E09EFEF0A3EFF0DE
:107AE9009039E2E0FCA3E0FD12B8A1903940E0FE34
:107AF900A3E0FF90393FE0FD3395E0FC12A21D9011
:107B09003940E0FEA3E0FF22E4903942F0A3F002FD
:027B19007916DB
:017B1B002247
:1076BF00903933ECF0A3EDF0A3EAF0A3EBF090399F
:0676CF0031EEF0A3EFF024
:1076D50090393AEEF0A3EFF0E4A3F0A3F012B2FC78
:1076E50090393EEEF0A3EFF08EF01233C7787F01AC
:1076F5000077C30200770604007897080000007839
:10770500E890393DE004F0700690393CE004F090D3
:107715003938E0FEA3E0FF903932E02FF09039319F
:10772500E03EF0903935E0FEA3E0FFC3903932E04A
:107735009FEE6480F8903931E06480984005EEF062
:10774500A3EFF0903937E0FF3395E0FEC39039E1C0
:10775500E09FFF9039E0E09EFEF0A3EFF09039E264
:10776500E0FCA3E0FD12B8A1903931E0FEA3E0FFF3
:10777500903937E0FD3395E0FC12A21D90393CE0CD
:10778500FEA3E0FFC3940AEE94004024EF9428EE94
:107795009400400E7F027E007D007C0012BF5602E1
:1077A50076E27F0A7E007D007C0012BF560276E2FB
:1077B5007F147E007D007C0012BF560276E2903970
:1077C5003DE004F0700690393CE004F0903938E073
:1077D500FEA3E0FFC3903932E09FFF903931E09E70
:1077E500FEF0A3EFF0A3E0FCA3E0FDC39FEE6480F1
:1077F500F8EC6480984008903931ECF0A3EDF090F6
:107805003937E0FF3395E0FEC39039E1E09FFF9003
:1078150039E0E09EFEF0A3EFF09039E2E0FCA3E052
:10782500FD12B8A1903931E0FEA3E0FF903937E0B1
:10783500FD3395E0FC12A21D90393CE0FEA3E0FF6C
:10784500C3940AEE94004024EF9428EE9400400E71
:107855007F027E007D007C0012BF560276E27F0A21
:107865007E007D007C0012BF560276E27F147E000A
:107875007D007C0012BF560276E2E490393EF0A30B
:10788500F07F1EFEFDFC12BF56903931E0FEA3E0ED
:10789500FF22E490393EF0A3F07F1EFEFDFC12BFEF
:1078A50056903937E0FF3395E0FEC39039E1E09F0C
:1078B500FF9039E0E09EFEF0A3EFF09039E2E0FCA6
:1078C500A3E0FD12B8A190393AE0FEA3E0FF90399C
:1078D50037E0FD3395E0FC12A21D90393AE0FEA396
:0D78E500E0FF22E490393CF0A3F00276E2CF
:0178F2002273
:10905D00903939EBF0A3EAF0A3E9F0A3ECF0A3ED1E
:01906D00F012
:10906E007F9F12C2EA7FA012C2EAE4903967F0A392
:10907E00F090393CE0FEA3E0FFC3903968E09FEE2C
:10908E006480F8903967E0648098501EA3E0243F16
:10909E00F582E43439F5837420F0903968E004F0F9
:1090AE007006903967E004F080C790393DE0243FA8
:1090BE00F582E43439F583E4F0903967F0A3F0904B
:1090CE00393CE0FEA3E0FFC3903968E09FEE648078
:1090DE00F8903967E064809840030291BE12844E86
:1090EE0090393EEFF09039E1E004F070069039E0EF
:1090FE00E004F09039E0E0FEA3E0FF9039E2E0FCFE
:10910E00A3E0FD12B8A190393EE0B4FF087F9C1297
:10911E00C2EA7FFF2290393EE0FF903968E0243F9B
:10912E00F582E43439F583EFF0EF6420601A90395C
:10913E003DE024FFFF90393CE034FFFE903967E0BC
:10914E006E7003A3E06F7057903967E07002A3E072
:10915E0070087F9C12C2EA7F0022E4FFFED3903992
:10916E003DE09FEE6480F890393CE06480984027A3
:10917E00743F2FF582E43439F583E0FD903939E000
:10918E00FBA3E475F001123159A9F0FAED12307219
:10919E000FBF00010E80C67F9C12C2EA7F01229093
:1091AE003968E004F07006903967E004F00290CD63
:0191BE00228E
:10844E0090396D7420F0E4903969F0A3F012B2FC0B
:10845E0090396BEEF0A3EFF08EF01233C785B701B3
:10846E0000851B0200847F040085CC080000008577
:10847E00DE90396DE004F0E0FFD3648094A0400AF2
:10848E00EF648094B050037430F090396DE0FFD3F8
:10849E00648094B9400AEF648094C150037441F033
:1084AE0090396DE0D3648094DA40037430F09039E3
:1084BE006AE004F07006903969E004F090396DE0DE
:1084CE00FF12B92B9039E1E024FFF09039E0E0344F
:1084DE00FFF0E0FEA3E0FF9039E2E0FCA3E0FD1226
:1084EE00B8A1C390396AE0940A903969E0940040CB
:1084FE000E7F0A7E007D007C0012BF5602845B7FD9
:10850E00147E007D007C0012BF5602845B90396D94
:10851E00E014F0E0C3648094A05003745AF09039D4
:10852E006DE0FFC3648094C1500AEF648094B9403B
:10853E00037439F090396DE0FFC3648094B0500A33
:10854E00EF648094A04003745AF090396AE004F00E
:10855E007006903969E004F090396DE0FF12B92B86
:10856E009039E1E024FFF09039E0E034FFF0E0FED6
:10857E00A3E0FF9039E2E0FCA3E0FD12B8A1C390A6
:10858E00396AE0940A903969E09400400E7F0A7EC1
:10859E00007D007C0012BF5602845B7F147E007D3E
:1085AE00007C0012BF5602845BE490396BF0A3F09E
:1085BE007F1EFEFDFC12BF5690396DE0FF22E49047
:1085CE00396BF0A3F07F1EFEFDFC12BF567FFF221B
:0A85DE00E4903969F0A3F002845B19
:0185E8002270
:05B3AF00903931EFF0C0
:10B3B400E4903937F07B017A3979327D04FC1290BC
:10B3C4005DE4FDFC903931E0FF3395E0FEEF25E0CC
:10B3D400FFEE33FE74B62FF58274C23EF583E49318
:10B3E400FE740193F5828E832DF582E5833CF5830B
:10B3F400E493FF74322DF582E43439F583E06F6011
:10B4040007E4903937F08006903937E004F00DBD39
:10B4140000010CED64044C70AB903937E0C36480D8
:10B4240094845032E4FCFD90C2B4E493FE7401931E
:10B434002DF582EE3CF583E493FF74322DF582E41E
:10B444003439F583E06F60037FFF220DBD00010CEA
:0DB45400ED64044C70D1E4903931F07F01BB
:01B4610022C8
:08BEBF00903932EEF0A3EFF020
:10BEC700E4A3F0A3F0903932E0FEA3E0FFC390397A
:10BED70035E09F903934E09E502AC2C67F147E0019
:10BEE7007D007C0012BF56D2C67F147E007D007C89
:10BEF7000012BF56903935E004F07006903934E0EF
:04BF070004F080C101
:01BF0B002213
:05002600903975EFF0B8
:10002B00E4F97D217CC07B64FA4387108D828C833D
:10003B00E05401F9EB1B70011AEB4A70037F0122AC
:0E004B00E960E9903975E08D828C83F07F00CA
:010059002284
:03BE2300CCEFCC95
:10BE2600E4FD90397574C0F0A37420F0A374C0F0DB
:10BE3600A37421F07B647A00438710903977E0FE83
:10BE4600A3E0F5828E83E05402FDEB1B70011AEB32
:10BE56004A70037F0122ED60E2CFECCF903975E0A6
:0BBE6600FCA3E0F5828C83EFF07F006E
:01BE710022AE
:10BC57007F80120026E4FF12BE23E4FF12BE237F7B
:10BC6700421200267F2812BE23E4FF12BE237F4321
:10BC7700120026E4FF12BE237F1012BE237F40125C
:10BC870000267F2812BE23E4FF12BE237F41120045
:10BC970026E4FF12BE23E4FF12BE237F24120026F0
:10BCA700E4FF12BE237F1012BE237F211200267FDE
:05BCB7009C1200262292
:04C2EA0012002622F6
:0700030012BBF112BF0C2239
:10BBF1007D3F7C00E4FFFE12BCBCE4903949F0A318
:10BC0100F0438710E4F5FF90394BF0A3F0E4FF1205
:10BC1100BE237FC012002690394CE004F0700690DC
:10BC2100394BE004F0C390394CE0944090394BE03B
:10BC31006480948040D790394AE004F070069039CE
:10BC410049E004F0C390394AE09428903949E0640E
:05BC510080948040AC6E
:01BC560022CB
:10BF0C007D077C00E4FFFE12B8A1E4903949F0A350
:10BF1C00F0438710E4F5FFFF12BE237FC01200260A
:10BF2C0090394AE004F07006903949E004F0C3906F
:10BF3C00394AE09440903949E06480948140D27D44
:09BF4C00077C00E4FFFE12B8A11D
:01BF550022C9
:0EBCBC0090394DECF0A3EDF0CBEFCBCAEECA01
:10BCCA007C007D061230B8CAEECACBEFCB90394D54
:10BCDA00E0FEA3E0FFC3743F9FFFE49EFE7C007D6D
:10BCEA00281230A6EF2BFFEE3ACBEFCBFA0C7D00F1
:10BCFA00FE12310DA3EEF0A3EFF07A00CFEBCF12D4
:0FBD0A00BE23903950E0FF12BE237F2412002683
:01BD19002207
:0EB8A10090396FEEF0A3EFF0A3ECF0A3EDF002
:10B8AF0090396FE0FAA3E0FB9039E0EAF0A3EBF0F8
:10B8BF00903971E0FEA3E0FF9039E2EEF0A3EFF0D4
:10B8CF00C374079FFFE49EFE7C007D281230A6EB19
:10B8DF002FFFEA3ECBEFCBFA0C7D00FE12310DEFBE
:10B8EF002410FFE43E903973F0A3EFF07A00CFEB12
:10B8FF00CF12BE23903974E0FF12BE237F241200B3
:10B90F0026903970E0FF12BE23903972E0FFC374A6
:0BB91F00079FFF12BE237F21120026AD
:01B92A0022FA
:10B65F00903960EEF0A3EFF0A3ECF0A3EDF0A3EBC5
:01B66F00F0EA
:10B67000903960E0FEA3E0FF7C007D061230B8CB7D
:10B68000EFCBCAEECA903960E0FEA3E0FF7C007DFC
:10B69000061230B8C374059D903967F0903962E0A6
:10B6A000FEA3E0FFC3743F9FFFE49EFE7C007D2865
:10B6B0001230A6CCEACCCDEBCDEF2DFFEE3C90398D
:10B6C00065F0A3EFF0903964E05401F0903966E042
:10B6D000FF12BE23903965E0FF12BE237F241200C3
:10B6E00026903964E0FF33333354F8FF903967E034
:07B6F00024F02FFF120026D9
:01B6F7002230
:1055910090394EEEF0A3EFF0A3ECF0A3EDF0A3EA07
:0455A100F0A3EBF098
:1055A50090394EE0FEA3E0FFC3EB9FFFEA9EFE901D
:1055B5003958F0A3EFF0C3EE64809480501590390C
:1055C50058E0FEA3E0FFC3E49FFFE49E903958F046
:1055D500A3EFF0903950E0FCA3E0FDC3903955E00E
:1055E5009DFF903954E09CFE90395AF0A3EFF0C32B
:1055F500EE64809480501590395AE0FEA3E0FFC315
:10560500E49FFFE49E90395AF0A3EFF0903958E0FB
:105615007002A3E0701A90395AE07002A3E070108E
:1056250090394EE0FEA3E0FF7B0112B65F7F0022BA
:1056350090395AE0FEA3E0FFD3903959E09FEE641C
:1056450080F8903958E064809850030257C190392A
:1056550052E0FEA3E0FF90394EE0FCA3E0FDD39FAE
:10566500EC9E4045903958ECF0A3EDF0903952E0AE
:10567500A3E090394EEEF0A3EFF0903952ECF0A391
:10568500EDF0903950E0FEA3E0FF903958EEF0A31D
:10569500EFF0903954E0FDA3E0903950CDF0A3ED43
:1056A500F0903954EEF0A3EFF090394EE0FFA3E00F
:1056B500903956CFF0A3EFF0903952E0FEA3E0FF0A
:1056C500D3903957E09F903956E09E400302592FF9
:1056D50090394EE0FAA3E0FBC3903953E09BFE906E
:1056E5003952E09A90395CF0A3CEF0903950E0FE43
:1056F500A3E0FFC3903955E09FFF903954E09E9099
:10570500395EF0A3EFF0C3903957E09BFF9039560F
:10571500E09AFE90395EE0FCA3E0FD1230A69039D8
:1057250058EEF0A3EFF0D39400EE64809480401D12
:1057350090395CE0FEA3E0FF7C007D0212310D9004
:105745003959E02FF0903958E03EF0801C90395CD3
:10575500E0FEA3E0FF7C007D0212310DC3903959B4
:10576500E09FF0903958E09EF0903958E0FEA3E0B4
:10577500FF90395CE0FCA3E0FD12310D903958EE45
:10578500F0A3EFF0903950E0FEA3E0FF903959E027
:105795002FF0903958E03EF0903956E0FEA3E0FF37
:1057A500A3E0FCA3E0FD7B0112B65F903957E0044E
:1057B500F07006903956E004F00256BD903954E079
:1057C500FEA3E0FF903950E0FCA3E0FDD39FEC9EE3
:1057D500404690394EE0FEA3E0FF903958EEF0A325
:1057E500EFF0903952E0FBA3E090394ECBF0A3EBFC
:1057F500F0903952EEF0A3EFF0903958ECF0A3EDAC
:10580500F0903954E0FFA3E0903950CFF0A3EFF0CA
:10581500903954ECF0A3EDF0903950E0FFA3E090FF
:105825003956CFF0A3EFF0903954E0FEA3E0FFD353
:10583500903957E09F903956E09E400302592F90CA
:10584500394EE0FEA3E0FFC3903953E09FFF903946
:1058550052E09E90395CF0A3EFF0903950E0FAA346
:10586500E0FBC3903955E09BFE903954E09A90399E
:105875005EF0A3CEF0C3903957E09BFF903956E018
:105885009AFE90395CE0FCA3E0FD1230A6903958F1
:10589500EEF0A3EFF0D39400EE64809480401D9069
:1058A500395EE0FEA3E0FF7C007D0212310D9039E8
:1058B50059E02FF0903958E03EF0801C90395EE0B9
:1058C500FEA3E0FF7C007D0212310DC3903959E043
:1058D5009FF0903958E09EF0903958E0FEA3E0FF24
:1058E50090395EE0FCA3E0FD12310D903958EEF0E1
:1058F500A3EFF090394EE0FEA3E0FF903959E02F79
:10590500F0903958E03EF0E0FEA3E0FF903956E014
:10591500FCA3E0FD7B0112B65F903957E004F070FF
:0A59250006903956E004F002582CF9
:01592F002255
:10A31E0090392FECF0A3EDF090392DEEF0A3EFF085
:08A32E00903931EAF0A3EBF0D5
:10A33600D3EF9BEE9A402790392DE0FEA3E0FF90E5
:10A34600393AEEF0A3EFF0903931E0FDA3E0903911
:10A356002DCDF0A3EDF0903931EEF0A3EFF090396A
:10A3660033E0FEA3E0FF90392FE0FCA3E0FDD39F8E
:10A37600EC9E401E90393AECF0A3EDF0903933E0B4
:10A38600A3E090392FEEF0A3EFF0903933ECF0A371
:10A39600EDF0903935E05401F090392DE0FFA3E05F
:10A3A600903936CFF0A3EFF0903931E0FEA3E0FF0D
:10A3B600D3903937E09F903936E09E505590392F2B
:10A3C600E0FFA3E0903938CFF0A3EFF0903933E007
:10A3D600FEA3E0FF903938E0FCA3E0FDD39FEC9E9E
:10A3E6005020903936E0FEA3E0FF903935E0FB12AD
:10A3F600B65F903939E004F07006903938E004F021
:10A4060080CA903937E004F07006903936E004F0DF
:02A4160080962E
:01A418002221
:10B92B0090396EEFF0BF08219039E0E0FEA3E0FF05
:10B93B00D39400EE94004011EF24FFFFEE34FFFE92
:10B94B00A3E0FCA3E0FD12B8A190396EE024E0F077
:10B95B00E0FFC39400405112BE237FC0120026901B
:10B96B0039E0E0FEA3E0FFC39427EE94005012EF02
:10B97B002401FFE43EFEA3E0FCA3E0FD12B8A1808E
:10B98B00149039E3E024FFFD9039E2E034FFFCE44E
:10B99B00FFFE12B8A1C39039E2E09400500A7D2754
:09B9AB007C00E4FFFE12B8A122A9
:10C18100903960EBF0A3EAF0A3E9F0903960E0FBAD
:10C19100A3E0FAA3E0F912302CFF600F12B92B9043
:0CC1A1003961E475F00112314380E022A6
:0EA21D0090394EEEF0A3EFF0A3ECF0A3EDF0BD
:10A22B00D39405EC94004009903950E4F0A37405E5
:10A23B00F0C3903951E09401903950E094005005EF
:10A24B00E4F0A304F0E490395EF0A3F07B107A27DE
:10A25B0090395CF0A3F0EB4A700302A2FA90394EEE
:10A26B00E0FEA3E0FFCDEBCDCCEACC12310DEF2419
:10A27B0030FD90395DE0F92452F582E43439F583F1
:10A28B00EDF0EF4E702490395EE07002A3E0701A8F
:10A29B00C3EB940AEA64809480400F745229F582D0
:10A2AB00E43439F5837420F0800890395EE4F0A330
:10A2BB0004F090394EE0FEA3E0FFCDEBCDCCEACC21
:10A2CB0012310D90394EECF0A3EDF090395DE004B6
:10A2DB00F0700690395CE004F07C007D0ACFEBCF88
:10A2EB00CEEACE12310DCAEECACBEFCB02A26190F1
:10A2FB00395DE02452F582E43439F583E4F090398A
:10A30B0051E0FF7B01C374579FF974399400FA1223
:02A31B00C181FE
:01A31D00221D
:0EAB7E00903949EEF0A3EFF0CBEDCBCAECCA54
:10AB8C00D3EB9405EA940040047A007B05C3EB9464
:10AB9C0001EA940050047A007B019039577427F035
:10ABAC00A37410F0E4903955F0A3F0903957E0708D
:10ABBC0002A3E06068903957E0FCA3E0FD903949AE
:10ABCC00E0FEA3E0FF12310DEF2430FF903956E088
:10ABDC00244BF582E43439F583EFF0903949E0FEEB
:10ABEC00A3E0FF903957E0FCA3E0FD12310D903942
:10ABFC0049ECF0A3EDF0903956E004F07006903972
:10AC0C0055E004F0903957E0FEA3E0FF7C007D0A8C
:10AC1C0012310D903957EEF0A3EFF0808E9039562B
:10AC2C00E0244BF582E43439F583E4F0CFEBCF7BB1
:0EAC3C0001C374509FF974399400FA12C1815B
:01AC4A0022E7
:10B9B400903929EEF0A3EFF0A3ECF0A3EDF024010D
:10B9C400FDE43CFC7B0112B65F90392AE02401FFC0
:10B9D400903929E03400FE90392BE0FCA3E0FD7B94
:10B9E4000112B65F90392AE02401FF903929E0342E
:10B9F40000FE90392CE02402FD90392BE03400FC49
:10BA04007B0112B65F90392AE02402FF903929E0C5
:10BA14003400FE90392CE02401FD90392BE03400F1
:07BA2400FC7B0112B65F225A
:10C15000D295D294C295D295C2949000B4E024E1D5
:10C16000FFC364809480500474402FFF7E01C3EFAE
:10C170006480F8EE6480985007D294C2940E80EEEA
:01C18000229C
:10C22300D295C294D2949000B4E004F0E0D3648039
:10C2330094BF4002E4F07F1E7E007D007C0012BFAD
:02C24300562281
:109CDA00D295C294D294C294D294C294D294C29489
:109CEA00D294C294D294C294D294C294D294C2947A
:109CFA00D294C294D294C294D294C294D294C2946A
:109D0A00D294C294D294C294D294C294D294C29459
:109D1A00D294C294D294C294D294C294D294C29449
:109D2A00D294C294D294C294D294C294D294C29439
:109D3A00D294C294D294C294D294C294D294C29429
:109D4A00D294C294D294C294D294C294D294C29419
:109D5A00D294C294D294C294D294C294D294C29409
:109D6A00D294C294D294C294D294C294D294C294F9
:109D7A00D294C294D294C294D294C294D294C294E9
:109D8A00D294C294D294C294D294C294D294C294D9
:109D9A00D294C294D294C294D294C294D294C294C9
:109DAA00D294C294D294C294D294C294D294C294B9
:109DBA00D294C294D294C294D294C294D294C294A9
:109DCA00D294C294D294C294D294C294D29490005F
:109DDA00B4E014F0E0C3648094805003743FF07FD1
:0B9DEA001E7E007D007C0012BF562290
:09C2E1000A54696D656F75740063
:10C1D60090C0437482F07403F07401F004F0E4FF3D
:10C1E600FE0FBF00010EEF64644E70F590C04374FD
:07C1F60003F07406F014F0E1
:01C1FD00221F
:03AF6300C9EFC96A
:10AF66009039927475F0A37430F090C041E0FF7E82
:10AF7600007C005408FD640860089039E57401F00F
:10AF86008005E49039E5F0E4903990F0A3F0FCEF09
:10AF96005404FD640470079039E404F08005E490DD
:10AFA60039E4F0E4903990F0A3F0FCEF5410FD641E
:10AFB6001060089039E67401F08005E49039E6F0F7
:10AFC6009039E5E06401600F9039E4E064016007C0
:10AFD6009039E6E0B401037FFF2290C040E9F0908B
:10AFE600C043E4F0903990F0A3F090C04304F043DE
:10AFF600871090C041E05402FD7C00903993E02414
:10B00600FFF0903992E034FFF0E07002A3E07003A5
:0BB016007FFE22ED64024C60D67F003C
:01B02100220C
:0BBB1600903989EBF0A3EAF0A3E9F0FE
:10BB210012000E90398CEEF0A3EFF0E4A3F0A3F035
:10BB310090398CE0FEA3E0FFC390398FE09FEE6463
:10BB410080F890398EE06480985039903989E0FB13
:10BB5100A3E0FAA3E0F912302CFF12AF63EFB4FEB9
:10BB6100097BFF7AC279E1123D1A90398AE475F0B6
:10BB71000112314390398FE004F0700690398EE064
:04BB810004F080ACA0
:01BB8500229D
:0EA60700903977EEF0A3EFF0A3ECF0A3EDF0A6
:10A61500D39405EC94004009903979E4F0A37405CE
:10A62500F0C390397AE09401903979E094005005AF
:10A63500E4F0A304F0E4903987F0A3F07B107A27C7
:10A64500903985F0A3F0EB4A700302A6D9903977CB
:10A65500E0FEA3E0FFCDEBCDCCEACC12310DEF242B
:10A6650030FD903986E0F9247BF582E43439F583B1
:10A67500EDF0EF4E7019903987E07002A3E0700F8E
:10A68500747B29F582E43439F5837420F0800890D1
:10A695003987E4F0A304F0903977E0FEA3E0FFCD1D
:10A6A500EBCDCCEACC12310D903977ECF0A3EDF07F
:10A6B500903986E004F07006903985E004F07C005E
:10A6C5007D0ACFEBCFCEEACE12310DCAEECACBEF63
:10A6D500CB02A64B903986E0247BF582E43439F52C
:10A6E50083E4F090397AE0FF7B01C374809FF974AD
:07A6F500399400FA12BB16B4
:01A6FC00223B
:10C1AD00EFB40A11740D30D0052013024480F599B7
:10C1BD003099FDC299EF547F30D005201302448091
:09C1CD00FFF5993099FDC2992299
:102A1600022D6FE86480F8E933E83360110460F052
:102A2600ED33EC337009E8FCE9FDEAFEEBFF220426
:102A360060DED3EB9FEA9EE99DE8C2E78CF0C2F721
:102A460095F0400CE8CCF8E9CDF9EACEFAEBCFFBED
:102A5600122D3A85D0F05804700320D5B3E80470DF
:102A6600075002B2D5022D7992D5EC0460F7E4CC7A
:102A7600C0E0C398F8603B94186008400DD0E0FBB6
:102A8600022D51E4FBFAC9FC8028E830E406E4C9CB
:102A9600FBE4CAFCE830E305E4C9CACBFCE854070A
:102AA6006010F8C3E913F9EA13FAEB13FBEC13FC15
:102AB600D8F130F52FC3E49CFCEF9BFFEE9AFEEDB8
:102AC60099FDD0E0FBEF4E4D4C701222DB03022D38
:102AD60076EC2CFCEF33FFEE33FEED33FDED30E705
:102AE600EB022D51EF2BFFEE3AFEED39FDD0E0FB68
:102AF60050130BBB0003022D79ED13FDEE13FEEF11
:082B060013FFEC13FC022D513A
:102B0E00EC4D6011E8497017ED33EC3304600DE4C1
:102B1E00FCFFFEFD22E933E8330470F8022D6F123C
:102B2E002D3A58046009E4CC24815006285009023D
:102B3E002D79284003022D76C0E0EB4A7044B9800F
:102B4E0006D0E0FB022D65EF4E701CBD8008EBFF3A
:102B5E00EAFEE9FD80EBE98DF0A4FEE5F0022BF72D
:102B6E00E9CDF9EAFEEBFFEF89F0A4FCE5F0CE89A2
:102B7E00F0A42EFFE435F0CD89F0A42DFEE435F05F
:102B8E008067EF4E7005BD80D780C3EF8BF0A4AC8D
:102B9E00F0EE8BF0A42CFCE435F0F8EF8AF0A42CC8
:102BAE00E5F038FCE433CB8DF0A42CFCE5F03BF8DB
:102BBE00EE8AF0A42CFCE5F038F8E433CF89F0A4CB
:102BCE002CFCE5F038CF3400CE89F0A42FFFE5F0D1
:102BDE003EFEE433C98DF0A42EFEE5F039CD8AF029
:102BEE00A42FFFE5F03EFEE43DFD33D0E0FB5007A1
:102BFE000BBB000F022D79EC2CFCEF33FFEE33FEF6
:062C0E00ED33FD022D5123
:102C1400022D79EC5D046005E859047003022D6F00
:102C2400122D3A580460F6EC4860F2EC7004FDFE94
:102C3400FF22C860DB2481C85009C3986002500693
:102C4400022D769850CAF582E9294B4A7005AB8269
:102C5400022D6575F0007C1A7880C3EF9BEE9AED27
:102C640099400DC3EF9BFFEE9AFEED99FDE842F00B
:102C7400DC23ACF0D0E0FFD0E0FED0E0FDAB82205E
:102C8400E7101BEB60BAEC2CFCEF33FFEE33FEEDE8
:102C940033FD022D51E803F830E705C0F075F0006C
:102CA400EF2FFFEE33FEED33FD40B830E7C280AACC
:102CB400ED33EC33600A047003BD8004ECB2E7FC2E
:012CC40022ED
:102CC50075F020800E75F010800575F0087D007E8A
:102CD500007F003392D530D503123303EC33401017
:102CE500EF33FFEE33FEED33FDEC33FCD5F0ED2293
:0E2CF500E5F0247EA2D513CC92E7CDCEFF22CF
:102D0300EDD2E7CD33EC3392D524814006E4FFFEC8
:102D1300FDFC22FCE4CFCECDCC24E0501174FF8027
:102D2300EDC3CC13CCCD13CDCE13CECF13CF0470C4
:072D3300F030D5DE0233038E
:103CAF00E5082493F582E43439F583E00508229082
:103CBF003990300D03903993E475F001123381027E
:103CCF00302C2006E97F2ED2068018EF540F249057
:103CDF00D43440D4FF300A0BEF24BFB41A00500382
:103CEF002461FFE50960021509050CE50C7002055A
:103CFF000B300D0E903990E475F001123381EF0205
:103D0F00307202C1AD7403D20D8003E4C20DF50809
:103D1F00903990123398E4F509F50BF50CE509602D
:103D2F00077F20123CF280F5750AFFC207C206C258
:103D3F0008C209C20BC20CC20E123CBEFF700D307E
:103D4F000D057F00123D03AF0CAE0B22B4255FC2F1
:103D5F00D5C20A123CBEFF24D0B40A00501A75F027
:103D6F000A780930D50508B6FF0106C6A426F62045
:103D7F00D5047002D20980D924CFB41A00EF5004B1
:103D8F00C2E5D20A023FF5D20780C6D20680C0D262
:103D9F000880BCD2D580BAD20B80B47F20123CF2FF
:103DAF002008077401B5090040F1123CAFFF123C27
:103DBF00F2023D2CD20ED20C8095123CAFFB123C7E
:103DCF00AFFA123CAFF94A4B700679F37A407BFF9A
:103DDF0020082EE509602A7E008E8275830012303E
:103DEF004560060EEE650A70F0C2D5EBC0E0EAC082
:103DFF00E0E9C0E0EE124056D0E0F9D0E0FAD0E0B2
:103E0F00FB12302CFF60AAEBC0E0EAC0E0E9C0E093
:103E1F00123CF2D0E02401F9D0E03400FAD0E0FBFC
:103E2F00E50A0460DCD50AD98087D20880A2124047
:103E3F003860F7E50A700104122D84A90A600DE5B8
:103E4F000A600914F50A1240E0EF60F3EA30E70266
:103E5F00F404C3995079EAF4250A0430E701E40425
:103E6F00F50A800D12403860C1EA050A250A122DA5
:103E7F0084EA9039BFF030E701E4250A04D50A043B
:103E8F00200B0114124056E4C0E01240E09039BFFD
:103E9F00E0601320E70714F0123CDA802204F0D020
:103EAF00E014C0E07F00123CDAE50A6007123CD153
:103EBF00150A800B300B03123CD1D0E0023D2CD001
:103ECF00E00480C4124038609EE50A04122D8490ED
:103EDF0039BFEAF0E50A200B026001042404124006
:013EEF00567C
:103EF00074FF04C0E01240E0123CDAE50A200B0235
:103F00006003123CD1D0E0B50AE87F45123CE49052
:103F100039BFE07F2B30E7047F2DF404C0E0123C72
:103F2000F2D0E075F00A84C0F0123CDBD0E0123C25
:103F3000DB023D2C791080027908C20CC20E800889
:103F4000D2D5790A8004790AC2D5E50A047002F54F
:103F50000AE4FAFDFEFF123CAFFC7B0820071312B7
:103F60003CAFFD7B1030060A123CAFFE123CAFFFA7
:103F70007B20EC3382D592D55013C3E43006069FE4
:103F8000FFE49EFEE42007039DFDE49CFCE4CBF8E7
:103F9000C207EC700CCFCECDCCE824F8F870F380DB
:103FA00017C3EF33FFEE33FEED33FDEC33FCEB33A1
:103FB000FB994002FB0FD8E9EB300705F8D0E0C4CD
:103FC00048B207C0E00AEC4D4E4F78207B0070C22B
:103FD000EAB50A0040BCC0E0124058D0F0D0E02062
:103FE0000704C4C0E0C4B207C0F0123CDBD0F0D577
:103FF000F0EB023D2C1233A13DC9533F34583D9A9A
:104000004C3D96423F384F3F40443F40493DAF43CF
:104010003F46553E73463ED3453E3D474113503DD6
:104020009E2D3DA22E3DC52B3DA6233DC32040FC29
:104030002A3D5E4800003DBDE50AB4FF03750A064F
:10404000123CAFFC123CAFFD123CAFFE123CAFFF86
:104050009039B8022DC1790AA2D5200914300B0974
:10406000B910020404B9080104A2D5200C025001C1
:10407000042008689208B509005034C0E07F203061
:1040800009197F30A208720C720B500F1240AFC298
:1040900008C20CC20BC20E7F30800F300B03E9C088
:1040A000E0123CF2300B03D0E0F9D0E0B509CC309F
:1040B0000B177F30B9100C123CF27F58300A077F83
:1040C000788003B90803123CF23008057F2D023CCA
:1040D000F27F20200EF87F2B200CF322920880CF55
:1040E0007F00B40700500B24B8F582E43439F5831F
:1040F000E0FF22286E756C6C2900D207123CAF30AD
:1041000007F8C207780930D50108F6023D5E2D5048
:10411000434958123CAF2403B405004001E49041E8
:104120000E93123CE3743A123CE3D209750904027F
:024130003F341A
:102D3A00E9D2E7C933E833F892D5EDD2E7CD33ECDF
:072D4A0033FC5002B2D52258
:102D5100EC30E7100FBF000C0EBE00080DBD0004E3
:102D61000BEB6014A2D5EB13FCED92E7FD2274FF8F
:102D7100FCFDFEFF22E480F8A2D574FF13FC7D80E8
:032D8100E480EFFC
:102D8400F920E73624F950037907E4F42402FBE53B
:102D940082158270021583DBF6E024FB501BE96088
:102DA40014E4F0E582158270021583E004F0B40A9D
:0D2DB40008E4F0D9EE7401F00A22C2D52225
:102DC100ED33EC3392D5FA602AB4FF33EDC2E77BE1
:102DD100FF60067A2D79E6E4227A2D79EF20D50479
:102DE1007A2D79EA224E614E002B494E46002D493B
:102DF1004E4600E47A08F0A3DAFC7B00740722C097
:102E010083C082ECC0E0EDC0E0EEC0E0EFC0E0EADC
:102E110075F010A4CAABF075F04DA42BFBE435F0AE
:102E2100FCEA2410FAEB34C5FBEC34D9FCEDC2E723
:102E3100FF75F056A4F42411C5F0F434C58FF0A445
:102E41002AE5F03BE43CF020E714122EF6D0E0FF37
:102E5100D0E0FED0E0FDD0E0FC122C178014F40489
:102E6100122EF6D0E0FFD0E0FED0E0FDD0E0FC1263
:102E71002B0ED082D083E0FAEDD2E7CD33EC3324B0
:102E810082FBE4C3CF33CFCE33CECD33CD33DBF3AF
:102E91007B0775F00A846004F0A31B0AE5F0F0A338
:102EA1008FF0740AA4FFACF08EF0740AA42CFEAC6F
:102EB100F050010C8DF0740AA42CFDE435F0F0A360
:052EC100DBDE740722B6
:102EC6003F8000004120000042C80000447A000014
:102ED600461C400047C35000497424004B18968096
:102EE6004CBEBC205A0E1BCA6753C21C749DC5AE8D
:102EF600FB60065407601C2323122F24EB54386012
:102F060009122F10122F1F122B0EECF8EDF9EEFA04
:102F1600EFCB22EB122F1F80F1543803241C902E86
:102F2600C6FE93FC0EEE93FD0EEE930ECE93FF229D
:0300000002B78ABA
:0CB78A00787FE4F6D8FD75812202B7D16B
:102F3600E709F608DFFA8046E709F208DFFA803E7D
:102F460088828C83E709F0A3DFFA8032E309F6086A
:102F5600DFFA8078E309F208DFFA807088828C83D2
:102F6600E309F0A3DFFA806489828A83E0A3F60886
:102F7600DFFA805889828A83E0A3F208DFFA804C60
:102F860080D280FA80C680D4806980F28033801037
:102F960080A680EA809A80A880DA80E280CA8033A0
:102FA60089828A83ECFAE493A3C8C582C8CCC58318
:102FB600CCF0A3C8C582C8CCC583CCDFE9DEE780E8
:102FC6000D89828A83E493A3F608DFF9ECFAA9F067
:102FD600EDFB2289828A83ECFAE0A3C8C582C8CCBD
:102FE600C583CCF0A3C8C582C8CCC583CCDFEADED6
:102FF600E880DB89828A83E493A3F208DFF980CC38
:1030060088F0EF60010E4E60C388F0ED2402B40430
:103016000050B9F582EB2402B4040050AF232345D7
:063026008223902F867347
:10302C00BB010689828A83E0225002E722BBFE02A2
:09303C00E32289828A83E49322D5
:10304500BB010CE58229F582E5833AF583E0225040
:1030550006E92582F8E622BBFE06E92582F8E2228A
:0D306500E58229F582E5833AF583E49322A4
:10307200BB010689828A83F0225002F722BBFE013D
:02308200F32237
:10308400F8BB010DE58229F582E5833AF583E8F082
:10309400225006E92582C8F622BBFE05E92582C82E
:0230A400F22216
:1030A600EF8DF0A4A8F0CF8CF0A428CE8DF0A42E3E
:0230B600FE22F8
:1030B800BC000BBE0029EF8DF084FFADF022E4CCFC
:1030C800F875F008EF2FFFEE33FEEC33FCEE9DECC5
:1030D800984005FCEE9DFE0FD5F0E9E4CEFD22ED0B
:1030E800F8F5F0EE8420D21CFEADF075F008EF2F55
:1030F800FFED33FD4007985006D5F0F222C398FD46
:053108000FD5F0EA22E2
:10310D00C2D5EC30E709B2D5E4C39DFDE49CFCEEDD
:10311D0030E715B2D5E4C39FFFE49EFE1230B8C36D
:10312D00E49DFDE49CFC80031230B830D507C3E468
:06313D009FFFE49EFE224C
:10314300C5F0F8A3E028F0C5F0F8E5821582700217
:063153001583E038F022B4
:10315900A3F8E0C5F025F0F0E58215827002158329
:06316900E0C838F0E82286
:10316F00BB010A89828A83E0F5F0A3E0225006872B
:10317F00F009E71922BBFE07E3F5F009E3192289ED
:0B318F00828A83E493F5F07401932220
:10319A00BB010A89828A83F0E5F0A3F0225006F780
:0F31AA0009A7F01922BBFE06F3E5F009F319227D
:1031B900F8BB0111E58229F582E5833AF583E8F048
:1031C900E5F0A3F0225009E92582C8F608A6F02205
:0D31D900BBFE09E92582C8F2E5F008F222EC
:1031E600E88FF0A4CC8BF0A42CFCE98EF0A42CFC88
:1031F6008AF0EDA42CFCEA8EF0A4CDA8F08BF0A406
:103206002DCC3825F0FDE98FF0A42CCD35F0FCEB64
:103216008EF0A4FEA9F0EB8FF0A4CFC5F02ECD3929
:0F322600FEE43CFCEAA42DCE35F0FDE43CFC2296
:1032350075F008758200EF2FFFEE33FECD33CDCC50
:1032450033CCC58233C5829BED9AEC99E5829840D3
:103255000CF582EE9BFEED9AFDEC99FC0FD5F0D6B0
:10326500E4CEFBE4CDFAE4CCF9A88222B800C1B9DA
:103275000059BA002DEC8BF084CFCECDFCE5F0CB18
:10328500F97818EF2FFFEE33FEED33FDEC33FCEB51
:1032950033FB10D703994004EB99FB0FD8E5E4F90C
:1032A500FA227818EF2FFFEE33FEED33FDEC33FCF9
:1032B500C933C910D7059BE99A4007EC9BFCE99AED
:1032C500F90FD8E0E4C9FAE4CCFB2275F010EF2F32
:1032D500FFEE33FEED33FDCC33CCC833C810D70732
:1032E5009BEC9AE899400AED9BFDEC9AFCE899F86D
:0E32F5000FD5F0DAE4CDFBE4CCFAE4C8F92200
:10BFE300C2D5E830E70FB2D5E4C39BFBE49AFAE489
:10BFF30099F9E498F8EC30E717B2D512C019123268
:10C0030071E4C39BFBE49AFAE499F9E498F880039A
:10C0130012327130D50DE4C39FFFE49EFEE49DFD13
:04C02300E49CFC227B
:0E330300C3E49FFFE49EFEE49DFDE49CFC22DB
:10331100EB9FF5F0EA9E42F0E99D42F0EC6480C833
:0633210064809845F022D3
:10332700EB9FF5F0EA9E42F0E99D42F0E89C45F0FC
:013337002273
:0C333800ECF0A3EDF0A3EEF0A3EFF02208
:10334400A8828583F0D083D08212335B12335B1260
:10335400335B12335BE473E493A3C583C5F0C58385
:10336400C8C582C8F0A3C583C5F0C583C8C582C8D3
:013374002236
:0C337500A42582F582E5F03583F5832263
:10338100F8E0FBA3A3E0F925F0F0E58215827002D5
:073391001583E0FA38F02279
:09339800EBF0A3EAF0A3E9F02236
:1033A100D083D082F8E4937012740193700DA3A3BB
:1033B10093F8740193F5828883E4737402936860CF
:0633C100EFA3A3A380DFCF
:1033C700D083D082F8E4937012740193700DA3A395
:1033D70093F8740193F5828883E473740293B5F0CC
:0D33E700067403936860E9A3A3A3A380D834
:10C28700C3EE6480948040028007C3E49FFFE49E6E
:02C29700FE2285
:10BB8600903927EBF0A3EAF0A3E9F090392DEBF01A
:10BB9600A3EAF0A3E9F0903927E0FBA3E475F001EE
:10BBA600123159A9F0FA12302C70EB90392874FF33
:10BBB600F5F012314390392AE0FBA3E475F0011247
:10BBC6003159A9F0FA12302CFF903927E0FBA3E493
:10BBD60075F001123159A9F0FAEF12307270D69051
:0BBBE600392DE0FBA3E0FAA3E0F922F8
:1033F400E3F5F009E208B5F06D606B80F3E3F5F0F6
:1034040009E608B5F060605E80F387F009E608B568
:10341400F054605280F487F009E208B5F048604641
:1034240080F488828C8387F009E0A3B5F038603695
:1034340080F488828C8387F009E493A3B5F0276035
:103444002580F388828C83E3F5F009E0A3B5F016B8
:10345400601480F388828C83E3F5F009E493A3B5C8
:10346400F004600280F202351F808580E7808E8040
:10347400D2803C8015806C807E809B80B5808B8060
:10348400A1804F8070803A02353589828A83ECFAB4
:10349400E493F5F0A3C8C582C8CCC583CCE493A358
:1034A400C8C582C8CCC583CCB5F070606E80E18994
:1034B400828A83E493F5F0A3E208B5F05E605C8051
:1034C400F289828A83E0F5F0A3E608B5F04D604BFB
:1034D40080F389828A83E0F5F0A3E208B5F03C60CA
:1034E4003A80F389828A83E493F5F0A3E608B5F081
:1034F4002A602880F2805D89828A83ECFAE493F55D
:10350400F0A3C8C582C8CCC583CCE0A3C8C582C813
:10351400CCC583CCB5F004600280E27F00F845F0AE
:10352400600EE863F0806480D395F01F40027F0151
:103534002289828A83ECFAE0F5F0A3C8C582C8CC5C
:10354400C583CCE0A3C8C582C8CCC583CCB5F0CBB9
:1035540060C980E389828A83ECFAE0F5F0A3C8C5E8
:1035640082C8CCC583CCE493A3C8C582C8CCC58328
:10357400CCB5F0A760A580E288F0ED2402B4040085
:103584005099F582EB2402B40400508F2323458222
:053594002390346D736B
:10359900E709F60870FA8046E709F20870FA803EF2
:1035A90088828C83E709F0A370FA807EE309F60824
:1035B90070FA8076E309F20870FA806E88828C834B
:1035C900E309F0A370FA806289828A83E0A3F6088E
:1035D90070FA805689828A83E0A3F20870FA804AD9
:1035E90080D280FA80C680D4806580F280318010D4
:1035F90080A680EA809A80A880DA80E280CA803139
:1036090089828A83ECFAE493A3C8C582C8CCC583AE
:10361900CCF0A3C8C582C8CCC583CC70E9800D891C
:10362900828A83E493A3F60870F9ECFAA9F0EDFB1A
:103639002289828A83ECFAE0A3C8C582C8CCC583F3
:10364900CCF0A3C8C582C8CCC583CC70EA80DD891B
:10365900828A83E493A3F20870F980CE88F0ED247E
:1036690002B4040050C4F582EB2402B4040050BA39
:0936790023234582239035E973F7
:10000E00E4FFFE12302C600C0FEF70010E09E97048
:05001E00F20A80EF2250
:10B7960002005EE493A3F8E493A34003F68001F26B
:10B7A60008DFF48029E493A3F85407240CC8C333B4
:10B7B600C4540F4420C8834004F456800146F6DF83
:10B7C600E4800B0102040810204080907479E47E26
:10B7D600019360BCA3FF543F30E509541FFEE49378
:10B7E600A360010ECF54C025E060A840B8E493A33F
:10B7F600FAE493A3F8E493A3C8C582C8CAC583CA6A
:10B80600F0A3C8C582C8CAC583CADFE9DEE780BE21
:0176BE0000CB
:00000001FF
